:1000000000000320E57101007D6C0100716B0100AF
:10001000716B0100716B0100716B0100716B01006C
:10002000716B0100716B0100716B01007D6C01004F
:100030007D6C0100716B010079420100FD400100FF
:100040007D6C01007D6C01007D6C01007D6C010008
:100050007D6C01007D6C01007D6C01007D6C0100F8
:100060007D6C01007D6C01007D6C01007D6C0100E8
:100070007D6C01007D6C01007D6C01007D6C0100D8
:100080007D6C01007D6C01007D6C01007D6C0100C8
:100090007D6C01007D6C01007D6C01007D6C0100B8
:1000A000A1110100951101007D6C01007D6C010022
:1000B0007D6C01007D6C01007D6C0100515E0100D2
:1000C0007D6C01004D5D01007D6C0100855C0100CF
:1000D0007D6C0100BD5B01007D6C01007D6C010049
:1000E0007D6C01007D6C01007D6C01007D6C010068
:1000F0007D6C01007D6C01007D6C01007D6C010058
:100100007D6C01007D6C01007D6C01007D6C010047
:100110007D6C0100892A01007D6C01007D6C01006D
:100120007D6C01007D6C01007D6C01007D6C010027
:100130007D6C01007D6C01007D6C01007D6C010017
:10014000B54201007D6C0100F55A01007D6C010093
:100150007D6C01007D6C01007D6C01007D6C0100F7
:100160007D6C01007D6C0100891101007D6C010036
:100170007D6C01007D6C01007D6C01007D6C0100D7
:100180007D6C01007D6C01007D6C01007D6C0100C7
:100190007D6C01007D6C0100195A01007D6C01002D
:1001A0007D6C01007D6C01007D6C01007D6C0100A7
:1001B0007D6C01007D6C01007D6C01007D6C010097
:1001C0007D6C01007D6C01007D6C01007D6C010087
:1001D000FFFFFFFFFFFFFFFFFFFFFFFFFFFFFFFF2F
:10040000FFFFFFFFFFFFFFFFFFFFFFFFDEF9FFFF23
:1004100010B5054C237833B9044B13B10448AFF33E
:1004200000800123237010BD00B0FF1F00000000FA
:1004300074120F00084B10B51BB108490848AFF300
:1004400000800848036803B910BD074B002BFBD0A0
:10045000BDE81040184700BF0000000004B0FF1FB7
:1004600074120F0064A2FF1F000000002DE9F04786
:100470004DF29447C1F6FF7782B04DF298463B6843
:100480000093C1F6FF76009B32689B1AB3F5487F54
:1004900043F6105500F2B8824BF2EC14C2F200059C
:1004A000C1F6FF744DF27440C1F6FF7016F0FAFA0F
:1004B0004DF23440C1F6FF7008F076FB2368984295
:1004C000804600F33884C0F22D83434520D049F2A2
:1004D000D0295FFA88F3C1F6FF79184689F8003011
:1004E00018F006FB40F25050C0F2020017F0E4FD95
:1004F00099F800000BF048FE43F61430C2F20000F9
:100500000BF0BCFC0BF0A8FC3B680193019B336033
:100510004DF27447C1F6FF77C4F80080BB7B002B17
:1005200040F03E814DF62036C1F6FF764DF2844014
:10053000C1F6FF7016F0B6FA4DF25440C1F6FF70E6
:1005400008F032FB95F8AD3055F823305A7B03EBB9
:10055000820380465B68B34200F0A0824EF25442B0
:10056000C1F6FF72934200F0A6824EF24062C1F6DD
:10057000FF72934200F0ED834EF62C02C1F6FF723B
:10058000934200F0E5824EF61822C1F6FF729342C4
:1005900000F07D844EF60442C1F6FF72934200F0F3
:1005A000BB844EF6F052C1F6FF72934200F06F85A5
:1005B0004EF6DC72C1F6FF72934200F005844FF2F2
:1005C000C812C1F6FF72934200F0D6854FF2B432E2
:1005D000C1F6FF72934200F01D8640F25452C2F2FF
:1005E0000002934200F0668640F24072C2F20002BE
:1005F000934200F0AD8640F62C12C2F20002934204
:1006000000F0F48640F61832C2F20002934200F085
:100610003B8740F60452C2F20002934200F06C871E
:1006200040F6F062C2F20002934200F0718741F29C
:10063000DC02C2F20002934200F0A28741F2C8221B
:10064000C2F20002934200F0E28741F2B442C2F2E9
:100650000002934201F0BB8041F2A062C2F20002AC
:10066000934201F05D8041F68C02C2F20002934297
:1006700001F0E98041F67822C2F20002934201F0D3
:100680002B8141F66442C2F20002934201F07C8168
:1006900042F23C02C2F20002934201F0318141F683
:1006A0005062C2F20002934201F02F8342F22822EC
:1006B000C2F20002934201F01C8342F21442C2F2E1
:1006C0000002934201F0098342F20062C2F200028A
:1006D000934201F0F68242F2EC72C2F200029342BF
:1006E00001F0E38242F6D812C2F20002934201F016
:1006F000D08242F6C432C2F20002934200F0CE81B0
:1007000043F6AC42C2F20002934201F0B18243F2DE
:100710002412C2F20002934201F06B8243F21032C3
:10072000C2F20002934201F0198243F2FC42C2F28B
:100730000002934201F0EF8143F2E862C2F200024C
:100740009342636801F086814BF2EC199845C1F63B
:10075000FF7901F3798114DA40F29840C0F2020087
:1007600017F0AAFC40460BF041FF5FFA88F099F8B9
:1007700004100AF039FE95F8AD3055F823000AF060
:100780008BFEBA7FC4F804804DF27443C1F6FF7348
:100790001AB11F7F002F00F0128202B0BDE8F0876F
:1007A0003B7B002B7FF4BEAE40F61420C0F202006B
:1007B00017F082FC95F8AD3055F823305A7B03EBE7
:1007C00082034DF620365B68C1F6FF76B34200F037
:1007D000F6834EF26822C1F6FF72934200F04C8419
:1007E0004EF25442C1F6FF72934200F073844EF20F
:1007F0004062C1F6FF72934200F077844EF62C02FD
:10080000C1F6FF72934200F07B844EF61822C1F6C7
:10081000FF72934200F07F844EF60442C1F6FF72ED
:10082000934200F0E1844EF6F052C1F6FF7293421B
:1008300000F0E5844EF6DC72C1F6FF72934200F0E0
:1008400009834FF2C812C1F6FF72934200F01C8573
:100850004FF2B432C1F6FF72934200F0208540F2AD
:100860006832C2F20002934200F05C8540F25452BA
:10087000C2F20002934200F0608540F24072C2F280
:100880000002934200F09C8540F62C12C2F2000256
:10089000934200F0A08540F61832C2F20002934263
:1008A00000F0DC8540F60452C2F20002934200F0F0
:1008B000E08540F6F062C2F20002934200F0F0855B
:1008C00041F2DC02C2F20002934200F0F48541F2F0
:1008D000C822C2F20002934200F0038641F2B44201
:1008E000C2F20002934200F0F18541F2A062C2F22E
:1008F0000002934200F0238641F68C02C2F200020D
:10090000934200F0118641F67822C2F2000293422F
:1009100000F02B8641F66442C2F20002934200F0DE
:10092000198641F65062C2F20002934200F06486DA
:1009300042F23C02C2F20002934200F0A48642F26C
:100940002822C2F20002934200F0B38642F214421F
:10095000C2F20002934200F0A18642F20062C2F2AB
:100960000002934200F0D18642F2EC72C2F2000221
:10097000934200F0BF8642F6D812C2F200029342C0
:1009800000F0AD8642F6C432C2F20002934200F09B
:100990009B8643F6AC42C2F20002934201F01E81F4
:1009A00042F63872C2F20002934201F00C8143F227
:1009B0002412C2F20002934201F0FA8043F2103294
:1009C000C2F20002934201F0E88043F2FC42C2F21C
:1009D0000002934200F04E8743F2E862C2F2000246
:1009E000934200F03C8743F6D402C2F200029342E5
:1009F0007FF49CAD40F6C410C0F202000BF0B6FBD1
:100A000006200AF06FFC91E5C2F2000543F6C02211
:100A100095F8AD3055F82330597B03EB8103C2F2D2
:100A200000025B68934204D04BF2EC14C1F6FF74F1
:100A300038E540F6D810C0F202000BF097FB4DF2FB
:100A40005440C1F6FF7008F0AFF84BF2C018C1F681
:100A5000FF784BF2EC1488F829004DF68810C1F6A7
:100A6000FF700BF00BFA0BF099FB4DF23442C1F61C
:100A7000FF7298F90030C1F6FF7400210520636011
:100A8000906323EAE37382F83C10516372B68342A9
:100A9000A8BF03469B00D36262B603E5636898452E
:100AA0003FF46FAE49F2A423C1F6FF7383F80080D0
:100AB0000BF0D2F965E6636898453FF462AE40F208
:100AC00004305FFA88F90A21C0F2020016F012FE23
:100AD00000220A21484617F0F9FA0BF0F3F907EE65
:100AE000909A0023C4F2C62306EE903AB8EE676AE5
:100AF0000023C6EE267A07EE103A4BF22003C1F629
:100B0000FF7377EE877A18684368C3ED007A0EF0BA
:100B10008DFE49F2A823C1F6FF7383F804900BF011
:100B20009BF92EE640F24450C0F2020017F0C4FADE
:100B3000B8F1000FC0F20981404600220A2117F0E7
:100B4000C5FA0BF0BFF9236843457FF4C0ACDFE47E
:100B5000636898453FF415AE40F220305FFA88F99B
:100B60000D21C0F2020016F0C5FD00220A21484600
:100B700017F0ACFA0BF0A6F907EE909A0023C4F236
:100B8000C62306EE903AB8EE676A0023C6EE267AD0
:100B900007EE103A4BF22003C1F6FF7377EE877A27
:100BA00018684368C3ED027A0EF040FE49F2A823AC
:100BB000C1F6FF7383F806900BF04EF9E1E540F6BD
:100BC000F410C0F202000BF0D1FA95F8AD3055F8F0
:100BD00023305A7B03EB820343F610595B68B34220
:100BE000C2F2000900F0DC8142F6C432C2F2000217
:100BF000934200F0EF8143F6AC42C2F2000293420E
:100C000000F07C814EF26822C1F6FF72934200F040
:100C1000C38140F26832C2F20002934200F0D080F9
:100C200042F63872C2F20002934200F02B833E4635
:100C3000B84640F2E040C0F2020017F03DFA6068AA
:100C400030440BF0D3FA40F2FC40C0F2020017F03F
:100C500033FA60680028B6BF2D22002240420A21E4
:100C600017F034FA40F21C50C0F2020017F024FAD8
:100C700000220A21384617F029FA0BF023F995F8DB
:100C8000AD3055F823707B7B07EB830343F6105997
:100C90005A6892F8511092F850308B42C2F2000913
:100CA00000F0E380636852F8212001334344DBB253
:100CB00001334BF2EC1A52F82330C1F6FF7A002BC5
:100CC00000F0D3809847386810F074FB38460AF07B
:100CD000E3FB99F8AD3059F82340637B04EB8303C1
:100CE0005A6892F8511092F850308B420BD0DAF8D3
:100CF000043052F8212001334344DBB2013352F86F
:100D0000233003B19847206810F054FB20460AF0C6
:100D1000C3FB95F8AD3055F82330186810F04AFB46
:100D200095F8AD3055F82340206810F043FB20467D
:100D30000AF0B2FB31E540F23450C0F2020017F085
:100D4000BBF9B8F1000FBFF6F7AEC8F100002D22D5
:100D5000F4E6636898453FF414AD40F210305FFA52
:100D600088F90C21C0F2020016F0C4FC00220A210E
:100D7000484617F0ABF90BF0A5F807EE909A002360
:100D8000C4F2C62306EE903AB8EE676A0023C6EEB8
:100D9000267A07EE103A4BF22003C1F6FF7377EE86
:100DA000877A18684368C3ED017A0EF03FFD49F277
:100DB000A823C1F6FF7383F805900BF04DF8E0E42B
:100DC0000F273E46B84634E7636898453FF4D9ACF0
:100DD00040F258304FFA88F90921C0F2020016F0AB
:100DE00089FCB9F1000FB4BF2D2200224FF00A0197
:100DF0004846B8BFC9F1000017F068F90BF062F877
:100E000007EE909A0023C4F24823B8EEE77A07EE83
:100E1000903A0023C4F2C82306EE103A37EE277A40
:100E20000023C7EE067A06EE903A4BF22003C1F695
:100E3000FF7377EEA67A18684368C3ED097A0EF05F
:100E4000F5FC49F2A823C1F6FF7383F80A900BF072
:100E500003F896E440F23C60C0F202000BF086F921
:100E60000D200AF0EDF9FFF761BB386810F0A2FA27
:100E700038460AF011FB40F60020C0F2020017F0DD
:100E80001BF96068013030440BF0B0F985E4636809
:100E900098453FF476AC40F230305FFA88F90B2188
:100EA000C0F2020016F026FC00220A21484617F084
:100EB0000DF90BF007F807EE909A0023C4F2C62351
:100EC00006EE903AB8EE676A0023C6EE267A07EE81
:100ED000103A4BF22003C1F6FF7377EE877A186859
:100EE0004368C3ED037A0EF0A1FC49F2A823C1F6D2
:100EF000FF7383F807900AF0AFFF42E4B8F1010FE7
:100F000000F0148140F2CC40C0F202000BF02EF948
:100F100004200AF0E7F940E4636898453FF431ACF7
:100F200040F23C304FFA88F90B21C0F2020016F073
:100F3000E1FBB9F1000FB4BF2D2200224FF00A01EE
:100F40004846B8BFC9F1000017F0C0F80AF0BAFF70
:100F500007EE909A0023C4F2C62306EE903AB8EE4C
:100F6000E76A0023C6EE267A07EE103A4BF220031A
:100F7000C1F6FF7377EE877A18684368C3ED077A86
:100F80000EF054FC49F2A823C1F6FF7383F80890D1
:100F90000AF062FFFFF7F5BB06273E46B84648E673
:100FA00040F2A440C0F2020017F086F80AF08AFF6F
:100FB00008F0CEFA01200AF095F9FFF7EEBB40F2F7
:100FC0006050C0F202000BF0D1F801200AF08AF95B
:100FD000FFF7ACBA40F2B040C0F2020017F06CF874
:100FE0000AF070FF4DF25440C1F6FF7007F0DCFDCF
:100FF0004BF2C016C1F6FF76307143F60050C2F2D4
:1010000000000AF03BFF99F8AD3059F823E09EF854
:101010000C30D3B13D46384602240EEB85025168B0
:1010200091F850206AB1002351F823201471D07038
:101030009070013391F85020DBB29A42F4D89EF8B8
:101040000C300135EDB2AB42E7D84DF23442C1F677
:10105000FF7296F928300021012023EAE3739063A0
:1010600082F83C10516372B68342A8BF03469B00CE
:10107000D36262B6FFF791BB40F27850C0F2020033
:101080000BF074F802200AF02DF9FFF74FBA6368ED
:1010900098453FF476AB40F248304FFA88F9C0F2F9
:1010A000020017F009F8B9F1000F4846BABF2D2227
:1010B000C9F1000000220A2117F008F80AF002FF27
:1010C00049F2A823C1F6FF7383F809900AF0C4FE21
:1010D000FFF757BB40F29050C0F202000BF046F809
:1010E00007200AF0ADF8FFF721BA40F2AC50C0F289
:1010F00002000BF03BF808200AF0A2F8FFF716BA3E
:1011000040F2C850C0F202000BF030F809200AF09B
:1011100097F8FFF70BBA40F2E450C0F202000BF070
:1011200025F80A200AF08CF8FFF700BA49F2A42447
:10113000C1F6FF7440F2C040C0F2020016F0BCFFDE
:101140003A460A21207816F0C1FF0AF0BBFE40F2B1
:10115000C040C0F2020016F0AFFF20780BF014F888
:101160004BF2A4124BF21C03C1F6FF72C1F6FF73DF
:10117000217811701F70CBE6636898453FF401AB8E
:1011800040F264305FFA88F90B21C0F2020016F0D9
:10119000B1FA00220A21484616F098FF0AF092FEA2
:1011A00007EE909A0023C4F2C62306EE903AB8EEFA
:1011B000676A0023C6EE267A07EE103A4BF2200348
:1011C000C1F6FF7377EE877A18684368C3ED0A7A31
:1011D0000EF02CFB49F2A823C1F6FF7383F80B90A5
:1011E0000AF03AFEFFF7CDBA40F20060C0F202000A
:1011F0000AF0BCFF0B200AF023F8FFF797B940F282
:101200001C60C0F202000AF0B1FF0C200AF018F8CE
:10121000FFF78CB9636898453FF4B3AA40F2703089
:101220005FFA88F91321C0F2020016F063FA002277
:101230000A21484616F04AFF0AF044FE07EE909A4B
:101240000023C4F2C62306EE903AB8EE676A002384
:10125000C6EE267A07EE103A4BF22003C1F6FF7372
:1012600077EE877A18684368C3ED067A0EF0DEFAE7
:1012700049F2A823C1F6FF7383F80C900AF0ECFD45
:10128000FFF77FBA2327D2E440F25460C0F2020095
:101290000AF06CFF0E2009F0D3FFFFF747B940F2C8
:1012A0007060C0F202000AF061FF0F2009F0C8FF71
:1012B000FFF73CB9636898453FF463AA40F2843075
:1012C0005FFA88F91621C0F2020016F013FA002224
:1012D0000A21484616F0FAFE0AF0F4FD07EE909A4D
:1012E0000023C4F2C62306EE903AB8EE676A0023E4
:1012F000C6EE267A07EE103A4BF22003C1F6FF73D2
:1013000077EE877A18684368C3ED057A0EF08EFA97
:1013100049F2A823C1F6FF7383F80D900AF09CFDF3
:10132000FFF72FBA40F29460C0F202000AF01EFFED
:10133000032009F0D7FFFFF7F9B840F2A860C0F228
:1013400002000AF013FF102009F028FFFFF7EEB8A3
:10135000636898453FF415AA40F29C305FFA88F91B
:101360001321C0F2020016F0C5F900220A214846F6
:1013700016F0ACFE0AF0A6FD07EE909A0023C4F228
:10138000C62306EE903AB8EE676A0023C6EE267AC8
:1013900007EE103A4BF22003C1F6FF7377EE877A1F
:1013A00018684368C3ED047A0EF040FA49F2A823A6
:1013B000C1F6FF7383F80E900AF04EFDFFF7E1B916
:1013C00040F2CC60C0F202000AF0D0FE112009F019
:1013D000E5FEFFF7ABB840F2EC60C0F202000AF0A5
:1013E000C5FE122009F0DAFEFFF7A0B86368984541
:1013F0003FF4C7A940F2B0305FFA88F90E21C0F27D
:10140000020016F077F900220A21484616F05EFE27
:101410000AF058FD07EE909A0023C4F2C62306EEA8
:10142000903AB8EE676A0023C6EE267A07EE103AC5
:101430004BF22003C1F6FF7377EE877A1868436892
:10144000C3ED0B7A0EF0F2F949F2A823C1F6FF734F
:1014500083F80F900AF000FDFFF793B940F208708F
:10146000C0F202000AF082FE132009F097FEFFF797
:101470005DB840F22470C0F202000AF077FE14203A
:1014800009F08CFEFFF752B8636898453FF479A9DC
:101490005FFA88F017F000FA0AF0DEFCFFF771B986
:1014A00040F24470C0F202000AF060FE152009F01C
:1014B00075FEFFF73BB840F26070C0F202000AF020
:1014C00055FE162009F06AFEFFF730B840F29C7016
:1014D000C0F202000AF04AFE182009F05FFEFFF792
:1014E00025B840F28070C0F202000AF03FFE1720DB
:1014F00009F054FEFFF71AB8636898453FF441A914
:101500005FFA88F017F084F90AF0A6FCFFF739B902
:10151000636898453FF435A95FFA88F017F034F90D
:101520000AF09AFCFFF72DB940F2D870C0F2020021
:101530000AF01CFE1A2009F031FEFEF7F7BF40F258
:10154000B870C0F202000AF011FE192009F026FE60
:10155000FEF7ECBF40F61800C0F202000AF006FEEB
:101560001C2009F01BFEFEF7E1BF40F2F870C0F24C
:1015700002000AF0FBFD1B2009F010FEFEF7D6BFAB
:10158000636898453FF4FDA840F2C03049F2A829AD
:10159000C1F6FF795FFA88FA1321C0F2020016F053
:1015A000A9F800220A21504616F090FD0AF08AFCA4
:1015B00099F8153099F8122099F8111099F810003F
:1015C00001EE103A99F8143007EE903AB8EE411A4D
:1015D000F8EE677AF2EE040A81EE201AC7EEA00A4E
:1015E00007EE90AAB8EE670A0AF046FF89F813A042
:1015F0000AF032FCFFF7C5B840F63C00C0F202002A
:101600000AF0B4FD1D2009F0C9FDFEF78FBF636825
:1016100098453FF4B6A840F2D43049F2A829C1F663
:10162000FF795FFA88FA1021C0F2020016F062F822
:1016300000220A21504616F049FD0AF043FC99F8B1
:10164000153099F8122099F8111099F8100007EE4A
:1016500090AA01EE103A99F81330F8EE670A00EEFE
:10166000103AB8EE411AF2EE047A81EE271AC0EE73
:10167000A70AB8EE400A0AF0FFFE89F814A00AF0A3
:10168000EBFBFFF77EB840F65C00C0F202000AF008
:101690006DFD1E2009F082FDFEF748BF40F6A00058
:1016A000C0F202000AF062FD202009F077FDFEF78B
:1016B0003DBF40F68000C0F202000AF057FD1F2037
:1016C00009F06CFDFEF732BF40F61010C0F20200C8
:1016D0000AF04CFD042009F005FEFEF727BF40F696
:1016E000F800C0F202000AF041FD232009F056FD87
:1016F000FEF71CBF40F6E000C0F202000AF036FD23
:10170000222009F04BFDFEF711BF40F6C000C0F2E9
:1017100002000AF02BFD212009F040FDFEF706BF74
:10172000636898453FF42DA840F2F83014215FFA21
:1017300088F9C0F2020015F0DDFF00220A214846B8
:1017400016F0C4FC0AF0BEFB07EE909A0023C4F228
:10175000C623F8EE676A07EE103AC6EE877A0023D2
:1017600006EE103A77EE867AF7EE006AF4EEE67A45
:10177000F1EE10FA40F3898044F23873C2F20003AC
:1017800045F2606247F670519952F0EE667A45F67E
:101790002943C4F20F6307EE103A67EE877A4AF6E0
:1017A000D811FDEEE77AC2F2000117EE903A45F249
:1017B000606049F2A82203F5B343C1F6FF72193302
:1017C0000B5282F816900AF047FBFEF7DABF636807
:1017D00098453EF4D6AF40F2E83049F2A829C1F668
:1017E000FF795FFA88FA0F21C0F2020015F082FF3C
:1017F00000220A21504616F069FC0AF063FB99F8B2
:10180000143099F8122099F8111099F8100007EE89
:1018100090AA00EE903A99F81330B8EE671A00EEED
:10182000103AF8EE600AF2EE047AC0EEA70A81EEF2
:10183000271AB8EE400A0AF01FFE89F815A00AF030
:101840000BFBFEF79EBF636898453EF49AAF5FFAC4
:1018500088F016F00DFF0AF0FFFAFEF792BF40F68F
:10186000AC10C0F202000AF081FC272009F08CFDC8
:10187000FEF75CBE40F68C10C0F202000AF076FC67
:10188000262009F081FDFEF751BE45F62943F4EE0E
:10189000C67AC4F20F63F1EE10FA05EE903A54BF27
:1018A000B0EE677AB0EE467A27EE257A44F23872C7
:1018B000BDEEC77AC2F2000217EE103A45F260613F
:1018C00003F5B343F4EEE67A1933F1EE10FA53520E
:1018D0000EDDF0EE667A5AE7636898453EF451AF44
:1018E0005FFA88F016F046FE0AF0B6FAFEF749BF36
:1018F000F4EE467AF1EE10FA48BFF0EE467A46E78B
:10190000636898453EF43DAF40F2284015215FFAE8
:1019100088F9C0F2020015F0EDFE00220A214846C7
:1019200016F0D4FB0AF0CEFA07EE909A0023C4F228
:10193000C82306EE903AB8EE676A0023C6EE267A10
:1019400007EE103A77EE877AF4EEC77AF1EE10FAE6
:1019500058D4B7EE007AF4EE477AF1EE10FAC8BF29
:10196000F0EE477AFEEEC87A40F6B05249F2A8236C
:10197000C2F20102C1F6FF73C2ED097A83F81B902F
:101980000AF06AFAFEF7FDBE636898453EF4F9AEC8
:1019900040F2104015215FFA88F9C0F2020015F0FC
:1019A000A9FE00220A21484616F090FB0AF08AFAA6
:1019B00007EE909AF8EE676AB2EE047AC6EE877A7E
:1019C000F5EEC07AF1EE10FA37D445F2A653C4F220
:1019D000AC6307EE103AF4EEC77AF1EE10FA14DDBC
:1019E00040F6B052C2F201020023C7F6FE73D36183
:1019F00049F2A823C1F6FF7383F819900AF02CFA74
:101A0000FEF7BFBE07EE903AACE742F24B43C4F29A
:101A1000BE7307EE103A67EE877A0021FCEEE77A94
:101A200040F6B05217EE903AC7F6FE71C2F20102CC
:101A30008B42C2ED077AD7D8DAE740F6B053C2F24C
:101A400001030022DA61D3E740F28840C0F20200CD
:101A5000FEF786BE98453EF494AE40F278400D21E4
:101A60005FFA88F9C0F2020015F044FE00220A2154
:101A7000484616F02BFB0AF025FA4BF22003C1F67C
:101A8000FF73B9F1280F186800F28580B9F1000FD3
:101A900014BF4A46012249F2A823C1F6FF7347F258
:101AA000A40E02744FF0000C83F82490C3F67D7EE0
:101AB000034600F50261C3F8D0C2C3F8D4E2343360
:101AC00099424FF00002F6D100F628314FF0000E97
:101AD000C4F2203EC1F800E000F6F82E00F53161B6
:101AE000002300F52F6CC0F8DC3AC0F8EC3ACEF8D1
:101AF000002000F6F42300F60C3ECCF800200A602B
:101B00004FF07E51CEF8002019600DF08FFE0AF0E4
:101B1000A3F9FEF736BE636898453EF432AE40F254
:101B200064405FFA88F91321C0F2020015F0E2FD6B
:101B300000220A21484616F0C9FA0AF0C3F949F210
:101B4000A82319F10009C1F6FF7318BF4FF001096E
:101B500083F823900AF080F9FEF713BE6368984576
:101B60003EF40FAE40F250401121C0F2020015F0D9
:101B7000C1FD00220A215FFA88F016F0A7FA0AF0E8
:101B8000A1F949F2A823C1F6FF7383F822800AF075
:101B900063F9FEF7F6BD28227DE740F67010C0F22B
:101BA00002000AF0E3FA252009F0EEFBFEF7BEBCC6
:101BB00040F65810C0F202000AF0D8FA242009F0CA
:101BC000E3FBFEF7B3BC40F64410C0F202000AF09B
:101BD000CDFA052009F086FBFEF7A8BC40F62810D8
:101BE000C0F202000AF0C2FA042009F07BFBFEF703
:101BF0009DBC636898453EF4C4AD40F240405FFA36
:101C000088F90D21C0F2020015F074FD00220A21AE
:101C1000484616F05BFA0AF055F907EE909A002351
:101C2000C4F2C623F8EE675A06EE103A85EE867ABD
:101C3000002349F2A822C1F6FF7282F8219007EE34
:101C4000903A45F2EC13C3F6386306EE903A4BF245
:101C50002003C1F6FF7377EE277A1B6867EEA67A3A
:101C600003F63C33C3ED007A0AF0F6F8FEF789BDBF
:101C7000636898453EF485AD4BF21C0318F10002F1
:101C8000C1F6FF7318BF01221A700AF0E5F8FEF7DB
:101C900078BD636898453EF474AD5FFA88F00CF047
:101CA00005FC0AF0D9F8FEF76CBD636898453EF470
:101CB00068AD5FFA88F00CF0C7FC0AF0CDF8FEF7CB
:101CC00060BD636898453EF45CAD5FFA88F00CF047
:101CD00087FD0AF0C1F8FEF754BD636898453EF4ED
:101CE00050AD5FFA88F00CF0F3FD0AF0B5F8FEF79E
:101CF00048BD636898453EF444AD5FFA88F016F03D
:101D000001FB0AF0A9F8FEF73CBD636898453EF474
:101D100038AD5FFA88F016F0C1FB0AF09DF8FEF7C7
:101D200030BD00BF2DE98048B9B002F0CFF943F2D1
:101D300041744DF294422646C1F6FF7244F250645B
:101D4000029232462746C2F2010244F2B053019297
:101D50003A469E46C2F200024BF2200305921A4612
:101D6000C1F6FF7244F2F06300921A46C2F200021A
:101D700044F2147313921A46C2F2000248F2A553B9
:101D800012921A46C0F2000243F2357314921A46B8
:101D9000C2F2010243F2367310921A46C2F20102F5
:101DA00048F2295311921A46C0F2000243F28863A6
:101DB0001D921A46C2F2010243F2C86315921A46F6
:101DC000C2F2010248F6752317921A46C0F20002C9
:101DD00043F214730E921A46C2F2010243F2CC632C
:101DE0000C921A46C2F2010243F2CD6308921A46DF
:101DF000C2F2010243F2D06304921A46C2F2010217
:101E000043F2107307921A46C2F2010242F21923FA
:101E10000D921A46C0F2010243F2347318921A4628
:101E2000C2F2010240F6F4731E921A46C2F2010297
:101E300040F62C230B921A46C0F2020249F2A42368
:101E400016921A46C1F6FF7240F6F87319921A46B6
:101E5000C2F2010249F2D0231A921A464EF60453F6
:101E6000CEF2000340F6F07140F6FC70099348F2A0
:101E7000340343F6C05B43F6C06A41F241144EF2AC
:101E80000305C2F2000EC2F20101C2F20100C1F666
:101E9000FF72C4F20403CDF818E01C911F90C2F247
:101EA000000BC2F2000AC0F201041B920F93C4F2AD
:101EB0000705069BD3F8983044F2B056C2F20006EC
:101EC000002B00F01F86059BD3F8983044F2506633
:101ED000C2F20006002B01F00F8172B64EF2180319
:101EE000029ACEF200031B681168099A126862B662
:101EF000520102D5322B88BF0131C3F52F331C9A12
:101F000003F21F3346F6174012689B08C1F2C16006
:101F1000A0FB0303C2EB93034FF47A7202FB01337D
:101F200040F64B32934240F2568172B64EF218039D
:101F3000029ACEF200031B681168099A126862B611
:101F4000570102D5322B88BF0131029A1F981268BF
:101F50002792C3F52F3303F21F3346F61747C1F21A
:101F6000C167279E00689B084FF47A72A7FB037332
:101F700002FB01F202EB9302301A41F288331C9902
:101F80004DF2944740F6FC7698420A60C1F6FF771E
:101F9000C2F2010600F27486069BD3F89830002B3B
:101FA00000F0EA8103F10408059BD3F89820002A89
:101FB00000F0CD81043272B64EF218030299CEF2CF
:101FC00000031B680F680999096862B64E0102D5C3
:101FD000322B88BF013700990868C3F52F33066894
:101FE00003F21F3346F6174EC1F2C16E9B08AEFBDB
:101FF00003E341464FF47A7E36684FEA93080EFBBE
:1020000007F7B04772B64EF21803029A0999CEF25A
:1020100000031B681268096862B6480102D5322BBA
:1020200088BF0132C3F52F3303F21F3346F6174141
:102030009B08C1F2C161A1FB0313C8EB9303DF1B33
:102040004FF47A7303FB027340F65532934203D97F
:1020500000994A6801324A60009A11894BF22002C5
:10206000C1F6FF728B4288BF138172B6139B1A7F31
:1020700044F2F06302F0FF01C2F200030AB1002251
:102080001A7762B661B372B6139E47F6FF734FF4C8
:102090000041B6F91E20F383B6F92030318462B6D0
:1020A000002AB8BF5242002BB8BF5B429342B8BF70
:1020B000134607EE903A4FF47E43C4F2FF63F8EE06
:1020C000E77A06EE903A87EEA67AF7EE007AB4EE5B
:1020D000E77AF1EE10FA03DD009AD3680133D3609A
:1020E00072B6129B1A7F44F2147302F0FF01C2F21F
:1020F00000030AB100221A7762B661B372B6129E6B
:1021000047F6FF734FF40041B6F91E20F383B6F98A
:102110002030318462B6002AB8BF5242002BB8BFCB
:102120005B429342B8BF134607EE903A4FF47E43AA
:10213000C4F2FF63F8EEE77A06EE903A87EEA67AED
:10214000F7EE007AB4EEE77AF1EE10FA03DD009ACA
:10215000D3680133D360069FD7F8980044F2B05398
:10216000C2F20003B8B193F89C1001311F29CABF15
:102170000026CEB2314697F89D2044F2B0538A42F1
:10218000C2F20003F7D00631002243F8210083F8A1
:102190009C60C3F89820059FD7F8980044F25063DC
:1021A000C2F20003B8B193F89C1001311F29CABFD5
:1021B0000026CEB2314697F89D2044F250638A4201
:1021C000C2F20003F7D00631002243F8210083F861
:1021D0009C60C3F898209BF84C7043F6C053102FB6
:1021E000C2F2000340F23A81009B1A694BF22006CA
:1021F000C1F6FF76002A00F05B82178853889908A1
:1022000002EB81010433BB428E6880F0F58153807C
:1022100006F00F02A2F1080106294FEA162300F288
:10222000BF8003F00F03082A03F10100C6F3033354
:1022300000F05282092A00F036840A2A40F02684EF
:102240000A2B00F05287009BD3F880616EB1F768CB
:1022500047B13B68DB68A342384600D098477F68A7
:10226000002FF6D1B668002EF1D1BAF82E20BAF8B8
:10227000303043F6C0619A42C2F200014BD0898DE2
:1022800001338B4280F0E6804FEA830E9EB2DAF88B
:1022900024009AF8287050F80E90AAF8306043F69F
:1022A000C060C2F2000097B9C06880B19A4226BFF0
:1022B00001F1FF318A1AD243BAF820101344B3EB6C
:1022C000910F43F6C062C2F2000280F011844FEA1F
:1022D000192309F00F0703F00F08A7F108020A936A
:1022E00043F6C066C9F3031308F10101062A0391FE
:1022F000C2F200068AF838307CD8082FC9F30333BD
:1023000000F0E283092F00F01A840A2F40F00384C2
:102310000A2B00F06787029B0B9A1B6825931268B3
:10232000259B9B1A4DF2944140F6F472642BC1F642
:10233000FF71C2F2010200F2EE80019B1B78002BBC
:102340007FF4B7AD15F0D6F8B3E515F0D3F812F079
:10235000B3F9059BC3F8980050B9019B1B78002B7B
:10236000F3D012F0A9F9059BC3F898000028F4D027
:10237000021D20E615F0BEF812F09EF9069BC3F888
:10238000980050B9019B1B78002BF3D012F094F900
:10239000069BC3F898000028F4D000F1040803E677
:1023A000901E0128D9B240F23581052A00F02C8117
:1023B000042A00F02787501F022840F238840F2A91
:1023C0007FF441AFF72900F22581009AF029B2F895
:1023D000542002D0002A3FF436AFB2F5917FBFF40B
:1023E00032AF009801461144013281F85830A0F80C
:1023F000542028E7BB1E012B9DF8288040F229813C
:10240000052F00F01E81042F00F054847B1F022B47
:1024100040F2AE830F2F7FF47EAFB8F1F70F00F2DA
:102420001881B8F1F00FB6F8601102D000293FF41E
:1024300072AFDAF88031002B01F0BB84B1F5917FE7
:1024400081F0AD844B1C9BB25144AAF8603181F8F5
:102450003D8060E70026B646334618E7986C149A2C
:1024600003681B69934240F00684109B119A1B7805
:102470001078DBB2C0B2834238BF4033181A00284C
:102480003FF4B2AEDBF848001D9A03685B6943F67F
:10249000C0569342C2F2000640F00A86109B119A81
:1024A0001B781278D9B2D2B243F2367E9142C2F290
:1024B000010E01F03385531C3F2B40F24284159BE3
:1024C0001878179B1E680023C0B28EF8003026B122
:1024D000CB1A1A2B01DC00233370C3B203F0FB02CA
:1024E000F92A3FF481AEDBF85810002940F045840A
:1024F0009BF84D208BF84F30110601F155815AB2EF
:10250000002AC1F2A7810023CBF85830CBF8543011
:102510008BF84D3068E60B682493249B1360FDF71D
:10252000A5FF009B93F884214BF22003C1F6FF73B3
:10253000002A40F0DF80009B93F885314BF22002A7
:10254000C1F6FF72002B3FF4F8AE029B1A991B688C
:1025500023930968239B5B1A41F288318B427FF6F3
:10256000ECAE1368D3F8DC1A00297FF4E6AE012341
:10257000C4F2020382F885111B781B9ADB071678D8
:1025800040F12C864FF0A0531B789E4224D00123AB
:10259000C4F202031B78DF0741F199834FF0A05387
:1025A0001B789E4218D02B78802B01F07D8300226F
:1025B000C4F20202137813F0700300D013704FF0CE
:1025C000A05301221E70C4F202021378D807FCD572
:1025D0002B78012B01F0C58340F6BC202221C0F2EC
:1025E000020015F087F8169B02211B88ADF8A03079
:1025F00028A815F07FF8A0E6104614F0ABFF0AF00B
:10260000EDF8009B186103E6F02940F21083F729EA
:1026100000F00D83F82900F04A8640F23983FC2946
:1026200000F03E8600F29A84FA2900F07C85FB29AE
:102630007FF409AE009B5B6C002B3FF404AE98471F
:1026400001E6B8F1F00F40F29382B8F1F70F00F015
:102650008F82B8F1F80F01F0978340F25B83B8F1F5
:10266000FC0F01F0168300F22685B8F1FA0F01F095
:10267000EF82B8F1FB0F7FF44EAEDAF8A02143F6FB
:10268000C063C2F20003002A00F026859047C9F318
:1026900007469DF828309DF80C808AF83A304FEABA
:1026A00019678AF839808AF83B608AF83C7032E60C
:1026B0001E9B1B78002B3FF4C6AD0AF08FF8024634
:1026C000306100283FF4BFAD0788002F7FF496AD3E
:1026D00014F040FF3761B6E5082B7FF4B4AD009BE2
:1026E0005B69002B3FF4AFADC0B2320EC6F30741B9
:1026F0009847A8E51B68D3F8DC3A002B7FF41BAFA2
:1027000040F6302EC0F2020EBEE80F0028AF0FC711
:10271000BEE80F000FC7BEE80F000FC79EE80F000E
:1027200049F2AC2687E80F00C1F6FF764FF0FF3381
:1027300016F8012B82EA030138A801F00F0100EB23
:10274000810151F8401C81EA131181EA121303F050
:102750000F0300EB830353F8402C82EA111349F274
:10276000D022C1F6FF7296426FEA0303E0D140F631
:102770007420C0F20200282142F8283C14F0BAFF6D
:10278000009B93F88421002A00F0EB824CF6CD40A8
:10279000CCF6CC40A0FB0213DB0803EB8301A2EBD9
:1027A000410230328DF8C120002B01F0228321221A
:1027B000A0FB0361C90801EB8106013AA3EB4603C4
:1027C000D2B238AE1644303306F8403C0B460029EE
:1027D000EED11046C2F1220128AB184414F08AFF52
:1027E00040F6A0201121C0F2020014F083FF49F24C
:1027F000A823C1F6FF731968002900F0B8822120D0
:1028000000E0F0B201F00F03DAB2092B38AB034459
:1028100094BF30323732090900F1FF3603F8402CFB
:10282000EFD1C0F1220128AB184414F063FF40F649
:10283000B420C0F20200062114F05CFF009B93F864
:102840008431013B03EB8303DB000233212000E0F2
:10285000F0B203F00F02D1B2092A38AA024494BFA1
:10286000303137311B0900F1FF3602F8401CEFD13F
:1028700028ABC0F12201184414F03CFF169B022142
:102880001B88ADF8A03028A814F034FF009B40F658
:102890003027C0F2020793F884E10FCF28AE0FC6AD
:1028A0000FCF0FC60FCF0FC697E80F000EF1FF3EF8
:1028B00086E80F000EEB8E0E49F2AC20C1F6FF70D9
:1028C0004FEACE034FF0FF3210F8011B81EA0206F7
:1028D00038AF06F00F0607EB860656F8406C86EA1E
:1028E000121686EA111202F00F0207EB820252F86A
:1028F000401C81EA161249F2D021C1F6FF718842CC
:102900006FEA0202E0D149F2A826C1F6FF76C6F1CD
:10291000A05909F10109012701F8282C9944C4F2B2
:10292000020798460394CDF828A049F2A823C1F6DF
:10293000FF73C3F10102013642443244B2F5805FB5
:1029400023D23B7816F801ACDA0775D516F80930B2
:102950009A4506EB090418D03B78DB076FD523783E
:102960009A4512D02B78802B6CD00020C4F2020044
:10297000037813F0700300D0037084F800A03B7854
:10298000DC07FCD52B78012B6ED049F2D023C1F6A1
:10299000FF739E42C9D101230099039CDDF828A052
:1029A0000022C4F2020381F884211B78199AD80707
:1029B000167840F196840123C1F200431B789E42B1
:1029C0003FF4B9AD0123C4F202031B78D90740F1EB
:1029D00023850123C1F200431B789E423FF4ABAD37
:1029E0002B78802B01F082810022C4F2020213783E
:1029F00013F0700300D013700122C1F200420123D2
:102A00001670C4F202031A78D207FCD52B78012B7A
:102A10007FF491AD4EF20103C4F2070360221A70F5
:102A20002B78802BFCD148F24403C4F2040300222B
:102A3000C0F206221A607EE50FF06CFE86E70FF00A
:102A400069FE8CE748F24400C4F204004EF2010330
:102A50000022C4F20703C2F228220260002018708C
:102A60002B78802BFCD080E74EF20103C4F20703E1
:102A700060221A702B78802BFCD148F24403C4F2F8
:102A800004030022C0F206221A607EE70B2A40F0FF
:102A9000F6830B2B7FF4D7AB009B1B6A002B7FF4D4
:102AA00023AEFFF7D0BB092B7FF4CDAB320E009BDA
:102AB00000F007879B69002B3FF4C5ABC6F30741C5
:102AC000C0B29847FFF7BFBB082B7FF424ACD6F801
:102AD00064319DF80C80802286F83A2053B3C9F304
:102AE00007464FEA196740463A4631469847D8E5C7
:102AF00072B61346128C5969D86812F013FF62B689
:102B0000FFF7E5BB11F0D8FDC6F8980000287FF468
:102B1000DAA9FFF760BB0B2F40F065840B2B7FF425
:102B2000FAABD6F870319DF80C80B02286F83A20C6
:102B3000002BD4D14FEA1967C9F30746B1E5092B39
:102B40007FF4E9AB5FEA196700F01C86D6F86831BC
:102B50009DF80C80902286F83A20002B01F02F81FE
:102B6000C9F30746FFB23A4631464046984798E5D2
:102B7000DAF8803143F6C060C2F20000002B01F0A9
:102B8000AA80B0F86021B2F5917F80F07183511C6A
:102B900089B252449DF82830AAF8601182F83D307D
:102BA000052F00F05B83DAF8803143F6C066C2F28D
:102BB0000006002B01F05780B1F5917F81F05F8016
:102BC000481C0A4681B252444FEA194043F6C06697
:102BD000072FAAF8601182F83D00C2F2000641F00A
:102BE0004980002B00F04982B1F5917F01F08A8184
:102BF0004A1C92B2D7B2100A51444FEA196981F8BF
:102C00003D9011460026F0228AF83B708AF83C007D
:102C1000AAF860618AF83A20002B00F03D8243F662
:102C2000FD600122C2F200009847FFF774BB0099D3
:102C3000B1F854004BF2200EB0F5917FC1F6FF7E43
:102C400080F019820EEB0007411C052A87F85830E6
:102C500089B241F0FF810098D0F87C310022A0F8C1
:102C60005420002B3FF4EFAA4BF27800C1F6FF701E
:102C70009847FFF7E8BA984700283FF4B5AA01E45F
:102C800015F078FE3B682693269B3360FFF784B9E6
:102C9000F2293FF4D8AA40F21B83F32900F00E83F7
:102CA000F6297FF4D0AA009B9B6B002B7FF4C7AC66
:102CB000FFF7C9BAD6F88031002B01F02A80B6F8A8
:102CC0006011B1F5917F80F079824A1C701891B241
:102CD000B1F5917FA6F8601180F83D80C9F30747F0
:102CE00000F05C824A1C0AEB010091B2B1F5917FC1
:102CF0004FEA1969AAF8601180F83D7000F045822A
:102D00004A1C92B20B465344AAF8602183F83D90C6
:102D1000FFF701BBB8F1F20F00F0828340F2E582C9
:102D2000B8F1F30F00F08E83B8F1F60F7FF4F3AA39
:102D3000DAF89431002B00F0D4819847C9F30746A4
:102D4000A7E4159AD05C179A1668DAB2C0B28EF86A
:102D50000020002E3FF4C1AB994238BF4031FFF74D
:102D6000B7BB30238DF8C1300121212034E5302359
:102D70008DF8C1300121212055E5020600F1D082F5
:102D80009BF84F2043F6C050C2F20000F02A426D7B
:102D900000F0BA82461802F1FF3E8E4586F84F30A9
:102DA00000F2B98290F84FC0BCF1F00F3FF4ABAB2A
:102DB0001CF0800F40F0F28200238BF86630B02BBD
:102DC00000F00483A02B00F00183D02B00F0FE82E2
:102DD000E02B00F0FB82C02B00F0F882002043F6CD
:102DE000C056C2F20006032A08BF96F851209BF88D
:102DF00050108BF8650018BF002200264FF0010E1E
:102E0000B02B8BF867108BF86820CBF85860CBF8A4
:102E100054608BF8E9E000F0BC8200F2B382902BA2
:102E200000F0B782A02B00F0B482802B00F0B182BA
:102E300000238BF84D309BF86630902B75D0A3F1B2
:102E40008006F6B2602E43D9F12B47D04DD9FA2B2C
:102E500001F0F98073D8F32B01F01781C1F0B6802F
:102E6000F62B01F0AC80F82B03D1DBF8303003B146
:102E700098479BF8642043F6C056D307C2F2000679
:102E80007FF5B2A912F0FE0F3FF4AEA996F86610D6
:102E900081F08003602B6ED896F865309F4200F079
:102EA0003481002F00F031815208012A00F0928213
:102EB000032A7FF499A9084696F8682096F86710C7
:102EC00009F01AFCFFF790B980238BF866300022D6
:102ED0008742B9D0002FCCD1F12BB7D1DBF820300D
:102EE000002BC6D008469847C3E7B02B01F05980A5
:102EF00040F22081D02B01F05B8040F2E884E02B8F
:102F000001F03680F02BB4D1DBF81C3043F6C05012
:102F1000C2F20000002BACD0B0F86710802900F19D
:102F2000690028BF80219847A3E7002ACCD08742B8
:102F3000D0D1DBF80430002B9BD0984799E7FC2BCD
:102F400000F04987C0F04087FE2B00F04B87FF2B35
:102F50008FD1DBF84430002B8AD18AE7FE2900F0BC
:102F6000F880FF297FF46FA9009B1B6D002B7FF475
:102F700066ABFFF768B9F62900F0BE8500F2B485AC
:102F8000F12900F0AF8440F2CC85F22900F0638291
:102F9000F3297FF429A9B06C0E99026896F867604E
:102FA00013688B4240F06D870F9B1B6859055CD5F9
:102FB0000C9B1B680BB101221A70089B1F7801370C
:102FC0003F2F2B4688BF4FF000084FF4204925467D
:102FD00094BF5FFA87F84746C4F206091C46049B73
:102FE0001B78BB422CD1EFF31383002B40F0B88049
:102FF000EFF31083002B40F0B380EFF3058100293D
:1030000000F0AB860F2905D94EF2F033CEF2000363
:103010000B441B78EFF3118111B18B4228BF0B4693
:10302000402B40F29D80B3F5807FD8D1019B1B7867
:10303000002BD4D114F05EFA049B1B78BB42D2D093
:1030400007990D982346F322CA552C4601211D46A7
:103050004FF420430170C4F206030899BC2281F8A2
:103060000080DA70DBF848000268D36C06F07F015C
:103070009847FFF7B9B80146EDE5B1F5917F7FF4C8
:10308000B7AD0B1200228AF83C30F0238AF83B10CF
:10309000AAF860218AF83A30DAF88431002B3FF43C
:1030A0003AA943F6FD60C2F200009847FFF733B932
:1030B0009847FFF712BAB8F1FE0F00F05983B8F144
:1030C000FF0F7FF428A9DAF8AC2143F6C063C2F2FF
:1030D0000003002A7FF4DAAAD3F8B0310BB14046DE
:1030E0009847C9F30746FFF7D4BA009BDB69002B6A
:1030F0007FF4FAAAFFF7A7B811F0DEFAC6F8980035
:1031000000287EF4EAAEFFF766B89BF86420520808
:1031100043F6C056012AC2F2000600F05B81022A83
:103120007FF462A8C7E6009B1B6C002B7FF487AA84
:10313000FFF789B8902B3FF4FCAEA02B00F09A86E5
:10314000802B7FF496AEDBF80030002B7FF4F5AED9
:103150008FE6009BDB6C002B7FF471AAFFF773B83E
:1031600099F804301B067FF53AAF049B079A1B7849
:1031700001333F2B86BF00210B46D9B2D35CDBB2B3
:1031800089F80730049B197029E743F6FD60002297
:10319000C2F20000984700230122B4E5002206F1A4
:1031A0003D009847D6F8802186F83D704FEA1969AE
:1031B0000123002A00F0CD851946A1E5002206F181
:1031C0003D009847D6F8803186F83D800122C9F34A
:1031D0000747002B00F0B085114683E50FF09AFAFF
:1031E000FFF7D0B9D6F86C319DF80C80A02286F894
:1031F0003A20002B7FF473AC4FEA1967C9F30746F6
:10320000FFF74FBA009AB2F854004BF22002B0F523
:10321000917FC1F6FF72BFF416A8411C171889B23E
:10322000B1F5917F87F85830A2F85410C6F30747DC
:103230003FF409A85318811C89B2B1F5917F83F836
:103240005870A2F854103EF4FEAF11440330360E0D
:10325000A2F8540081F85860FEF7F5BFB8F1F70FF7
:103260007FF459A8DAF88031CFB2C1F30720C9E45E
:1032700011463D30002298470022012189E40C2AA2
:1032800040F052860C2B7EF4DEAF009B5B6A002B75
:103290003EF4D9AFC6F30741C0B29847FEF7D3BF9B
:1032A000009B9B6C002B7FF4CAA9FEF7CCBF009B50
:1032B000DB6B002B7FF4C3A9FEF7C5BF009B5B6BE4
:1032C000002B3EF4C0AFC6F307409847FEF7BBBFE4
:1032D000F1297EF4B8AF009B1B6B002BF3D1FEF7F6
:1032E000B2BF0FF017FAFFF766BBB8F1F10F7FF42A
:1032F00012A8DAF88831C9F30746002B3FF4C9A9B0
:1033000030469847FFF7C5B90844013A8A4280F829
:1033100069307FF6F8A80131CBF85810FEF764BF8A
:10332000A3F1F70008283FF62BAD4FF0010E0EFA7F
:1033300000F212F4DD7F40F0AF8500287FF420AD6D
:103340009BF8693043F6C056F02BC2F200067FF4BA
:10335000DAA84A1C06EB01084FF0F70CD1B2C2F311
:10336000072286F8663086F8650086F8E9E0B065E1
:10337000706586F84D0088F869C086F8671086F891
:1033800068205CE5D02B04D0E02B02D0C02B7FF46A
:103390004FAD8BF84DC09BF866304EE50CF10C0339
:1033A000DBB2012B7FF608AD0CF0FB03F92B3FF4E9
:1033B00003ADBCF1EF0F00F282850CF0F003802B1F
:1033C00080F8663002D0902B7FF4F9AC0CF00F003F
:1033D000013004E508469BF868209BF8671009F067
:1033E0008BF9FEF701BF0C2F40F00A850C2B7EF401
:1033F00092AFD6F874319DF80C80C02286F83A203E
:10340000002B3FF497ABC9F30746404631464FEADD
:1034100019679847FFF745B90FF07CF9FFF7D9BA5C
:10342000DAF88C21002A3FF45CAE4FEA19464FEAE5
:10343000594306F07F0003F47E531843F6B29047D9
:10344000FFF727B9DAF89031C9F30746002B7FF46C
:1034500057AFFFF71EB9B06C96F8672096F8687002
:10346000D0F800E042EAC717DEF800300E9A934227
:1034700040F042850F9B1B685E055DD50C9B1B6869
:103480000BB101221A70089B1E7801363F2E2B4685
:1034900088BF4FF000084FF42049254694BF5FFADB
:1034A00086F84646C4F206091C46049B1B78B342C4
:1034B0002CD1EFF31383002B40F01581EFF3108331
:1034C000002B40F01081EFF30581002900F02081EE
:1034D0000F2905D94EF2F033CEF200030B441B78CE
:1034E000EFF3118111B18B4228BF0B46402B40F204
:1034F000FA80B3F5807FD8D1019B1B78002BD4D103
:1035000013F0F8FF049B1B78B342D2D007990D98B3
:103510002346F2228A552C4601211D464FF42043B2
:103520000170C4F206030899BC2281F80080DA70A9
:10353000DBF84800D0F800E0DEF84830189A9342F3
:1035400007F07F0140F0CF84DEF800205FFA81F8B9
:103550000E998A4240F0B6840F9A1268520562D5DD
:103560000C9B1B680BB101221A70089B03951E78F7
:1035700001363F2E4FF42043524688BF4FF00009DA
:10358000C4F20603A24694BF5FFA86F94E461D4672
:103590001446049B1A78B2422CD1EFF31382002A0E
:1035A00040F0BC80EFF31082002A40F0B780EFF3C8
:1035B0000580002800F0AF800F2805D94EF2F032C8
:1035C000CEF2000202441278EFF3118010B1824271
:1035D00028BF0246402A40F2A180B2F5807FD8D1B0
:1035E000019B1A78002AD4D113F084FF049B1A7827
:1035F000B242D2D02346079A0D9802F806800121E4
:1036000054469A464FF420430170C4F206030899C9
:10361000039D81F80090BC22DA70DBF84800D0F8F6
:1036200000E0DEF84830189A9342C7F3C61140F024
:103630005784DEF800300E9A9342CEB240F03085C7
:103640000F9B1B6858057EF5CFAD0C9B1B680BB11B
:1036500001221A70089B1F7801373F2F2B4688BF25
:103660004FF000084FF42049254694BF5FFA87F8D1
:103670004746C4F206091C46049B1B78BB4228D16E
:10368000EFF31383002B5FD1EFF31083002B5BD19B
:10369000EFF30581002954D00F2905D94EF2F033FC
:1036A000CEF200030B441B78EFF3118111B18B4272
:1036B00028BF0B46402B47D9B3F5807FDCD1019B57
:1036C0001B78002BD8D113F015FF049B1B78BB424D
:1036D000D6D02346079A2C461D464FF42043C4F209
:1036E0000603D655C7E199F8043019067FF5DDAE1B
:1036F000049B079A1B7801333F2B86BF00210B46A2
:10370000D9B2D35CDBB289F80730049B1970CCE6E0
:103710004FF48073E4E64FF4807255E72A7913067C
:103720007FF537AF049B1A78079B01323F2A86BF8B
:1037300000200246D0B29A5CD2B2EA71049B1870A3
:1037400027E74FF48073AFE799F80430190693D553
:10375000049B079A1B7801333F2B86BF00210B4641
:10376000D9B2D35CDBB289F80730049B197083E7C8
:10377000DAF8A82143F6C063C2F20003002A7EF4FF
:1037800085AFA9E4D6F864319DF80C80802286F8D4
:103790003A20C9F30746002B00F02F8331464046FC
:1037A0003A469847FEF77DBF02F10C06F1B20129B7
:1037B0007EF6A5AE02F0FB01F9293EF4A0AEEF2A99
:1037C00035D802F0F001802932D101063EF597AEDE
:1037D00001218BF84F208BF85030CBF85810F6B2FF
:1037E000012E7EF690AE02F0FB03F92B3EF48BAE79
:1037F000EF2A33D802F0F003B02B3BD040F2F48331
:10380000D02B04D0E02B35D0C02B7EF47CAE02232D
:10381000CBF854300121DBF8583043F6C0508B42CE
:10382000C2F2000032D201338365FEF7DDBC1146DF
:1038300001F0DF0EBEF1900FC7D001F0BF0EBEF158
:10384000A00FC2D001F0EF01C029BED05AB2002AA9
:10385000BEF659AE1A4603F10C06C0E7F62A00F090
:10386000D88300F2CF83F12AD1D040F21D84F22A0E
:1038700040F0E4830323CBF854300221DBF85830C6
:1038800043F6C0508B42C2F20000CCD3EF2A94BF63
:1038900002F0F003134602F00F02501C9BF8501088
:1038A0008BF86500002201268BF866308BF86710D4
:1038B0008BF86820CBF85820CBF854208BF8E960BF
:1038C000F7E25B69002B7FF4F9A8FEF7BCBCC02BC4
:1038D0007FF4CFAADBF81030002B3FF4CAAA984738
:1038E000FFF7C7BAB06C96F8672096F8687003685F
:1038F000120102F0700207F00F071B6817430E9ABF
:10390000934240F049830F9A126852055DD50C9B93
:103910001B680BB101221A70089B1E7801363F2EDE
:103920002B4688BF4FF000084FF42049254694BF2E
:103930005FFA86F84646C4F206091C46049B1B78CB
:10394000B3422CD1EFF31383002B40F09E80EFF3B2
:103950001083002B40F09980EFF30581002900F0DF
:10396000A9800F2905D94EF2F033CEF200030B44A3
:103970001B78EFF3118111B18B4228BF0B46402B0E
:1039800040F28380B3F5807FD8D1019B1B78002B58
:10399000D4D113F0AFFD049B1B78B342D2D007996A
:1039A0000D982346F1228A552C4601211D464FF4DD
:1039B00020430170C4F206030899BC2281F80080FC
:1039C000DA70DBF8480003681B680E9A934240F0F7
:1039D000DF820F9B1B6858057EF506AC0C9B1B68AD
:1039E0000BB101221A70089B1E7801363F2E2B4620
:1039F00088BF4FF000084FF42049254694BF5FFA76
:103A000086F84646C4F206091C46049B1B78B3425E
:103A100028D1EFF31383002B4FD1EFF31083002B4A
:103A20004BD1EFF3058100295BD00F2905D94EF268
:103A3000F033CEF200030B441B78EFF3118111B188
:103A40008B4228BF0B46402B37D9B3F5807FDCD1A2
:103A5000019B1B78002BD8D113F04CFD049B1B78E5
:103A6000B342D6D0079A234697552C461D464FF4AD
:103A70002043C4F206030D98012101700899BC226D
:103A800081F80080DA70FEF7AFBB99F804301B06AE
:103A90007FF554AF049B079A1B7801333F2B86BFF9
:103AA00000210B46D9B2D35CDBB289F80730049B06
:103AB000197043E74FF480735BE799F804301906F7
:103AC000A3D5049B079A1B7801333F2B86BF0021A7
:103AD0000B46D9B2D35CDBB289F80730049B19706E
:103AE00093E74FF48073A8E7FC2900F2D582FA2906
:103AF00002D2F8297EF478AB01F10803DBB2072B80
:103B00003EF672AB012202FA03F313F0DD0F3EF42E
:103B10006BAB43F60860C2F200000CF0A1F8FEF7B0
:103B200063BBF0297EF460ABB6F86730802B28BF0A
:103B30008023002B3EF458AB68334FF420473344C6
:103B4000DDF810900A9306F16808C4F20607DBF866
:103B500048000E9A036818F8011F1B68934271D140
:103B60000F9B1B685E0553D50C9B1B680BB1012294
:103B70001A70089B03911E7801363F2E8CBF0023DC
:103B8000F3B22A4688BF1E461D4611465346A2463A
:103B900099F80020B2422CD1EFF31382002A3CD1D5
:103BA000EFF31082002A38D1EFF30580002846D0C9
:103BB0000F2805D94EF2F032CEF2000202441278FC
:103BC000EFF3118010B1824228BF0246402A24D967
:103BD000B2F5807FDCD1019A1278002AD8D12191E8
:103BE000209313F087FC99F800202199209BB24282
:103BF000D2D00A4654469A462B461546079A039950
:103C000091550D99012008700899BC220B70FA702B
:103C10000A9B98459BD1FEF7E7BA3A791006B7D5CB
:103C200099F80020079C01323F2A86BF00200246F7
:103C3000D0B2A25CD2B2FA7189F80000A8E74FF4C2
:103C40008072BDE798470A9B984580D1FEF7CCBAB1
:103C5000DAF89C2143F6C063C2F20003002A7EF426
:103C600015ADFFF739BAB1F5917FFEF4A9AF072F73
:103C70003FF407AACFB2C1F30720FEF7C3BF00226B
:103C800006F13D009847D6F8803100220121FEF769
:103C90009ABFDAF8A42143F6C063C2F20003002AF7
:103CA0007EF4F4ACFFF718BA48F24402C4F20402FE
:103CB0004EF201030021C4F20703C2F22821116071
:103CC00000221A702B78802BFCD0FEF770BC0EF00F
:103CD00021FDFEF763BCB0F86011B1F5917FBEF431
:103CE0005FAF4B1C0A4699B2FEF753BF48F244023D
:103CF000C4F204024EF201030021C4F20703C2F22F
:103D00002821116000221A702B78802BFCD0FEF73E
:103D10006BBEB6F86031B3F5917FBEF4FCAA5A1CB5
:103D200092B23344B2F5917FA6F8602183F83D80CA
:103D3000C9F307473EF4EFAA531C9BB25244B3F5B4
:103D4000917F4FEA1969AAF8603182F83D703EF41C
:103D5000E2AA5A1C92B2FEF7D6BF4FF48073FFF767
:103D600059B94EF20103C4F2070360221A702B788E
:103D7000802BFCD148F24403C4F204030022C0F2B9
:103D800006221A60FEF728BCDAF8982143F6C063D1
:103D9000C2F20003002A7EF479ACFFF79DB943F626
:103DA000FD600022C2F20000984700210123FEF7C7
:103DB0004BBBB1F5917FBEF4AEAAFEF743BBFFB299
:103DC000C9F30746FEF76DBCDBF83830002B7FF4F3
:103DD0004FA8FFF74EB8DBF83C30002B7FF448A823
:103DE000FFF747B8DBF84030002B7FF441A8FFF71E
:103DF00040B801212120FEF7EFBC1F46FEF751BC61
:103E00000D2F12D10D2B7EF486AAD6F878319DF8AD
:103E10000C80D02286F83A20002B7FF4F4AA4FEAD7
:103E20001967C9F30746FEF73CBC0E2B7EF473AA54
:103E3000D6F87C31E02286F83A209BB14FEA194649
:103E40004FEA594106F07F029DF80C8001F47E5143
:103E50001143A1F5005140469847F6B24FEA196761
:103E6000FEF71FBC9DF80C804FEA1967C9F307469F
:103E7000FEF717BCDBF80830002B7FF45EA8FEF7D6
:103E8000F8BFF3219847DBF84800026806F07F018D
:103E9000D36C9847FEF7A8B9002211468BF866301C
:103EA0008BF8E9E08BF867208BF868208BF86520A9
:103EB0001046902B3FF408A80022FEF7C0BF6346CF
:103EC000FEF77BBF41469047DBF84800189AD0F8D0
:103ED00000E0DEF848309342C7F3C6113FF4A9ABC7
:103EE0009847FEF781B99847DBF84800D0F800E022
:103EF000DEF84830FFF797BB9847B06CD0F800E089
:103F0000FFF71ABB002206F13D0098470127002069
:103F1000D6F8803101463A46FEF76EBEB16DFF23FA
:103F200011B30820FFF701BA0D2A09D10D2B7EF439
:103F30008AA9009B9B6A002B7FF4ACA9FEF783B98A
:103F40000E2B7EF480A9009BDB6A002B3EF47BA93C
:103F5000720C02F47E52C6F306411143C0B2A1F5C1
:103F600000519847FEF76FB94FF0FF30FEF7C0BA27
:103F7000DBF81830002B3EF47CAFD20102F47E5205
:103F800001F07F011143A1F500519847FEF771BF81
:103F900039469847FEF728B99847B06C03681B6804
:103FA00013E5DBF80C30002B7EF4C7AFFEF761BFE2
:103FB000DBF81430002B7FF492ACFEF75ABFDBF82D
:103FC0002C30002B7EF454AFFEF753BFDBF82430C7
:103FD000002B3EF44EAFD20102F47E5201F07F007E
:103FE00010439847FEF745BF902B3FF443ACA02BFE
:103FF0003FF440AC802B7EF486AA0323CBF85430E8
:1040000002213BE4FC2A5DD8FA2A02D2F82A7EF487
:104010007AAA002001268BF86620134601468BF809
:1040200065008BF867008BF86800CBF85800CBF878
:10403000540002468BF8E960FEF701BFF32A3FF413
:10404000E6ABFEF760BADBF83430002B7EF410AF3D
:10405000FEF70FBFB1F5917F3EF4FDAD0EEB01070A
:10406000831C310C072A87F8581099B27EF4F3ADFF
:10407000B1F5917F4FEA16663EF4EDAD7144033021
:1040800081F8586081B2FEF7E6BDDBF82830002BDE
:104090007EF428AFFEF7EDBEFE29FEF4A5A82BE5C1
:1040A00031469847FEF7A0B8F02A7EF42CAA80216A
:1040B0000023CBF854108BF869208BF84D307F210A
:1040C000FFF7A9BBFE2AA4D2FEF71DBA2DE9F04FD7
:1040D00040F64C01342649F23405C4F20405C4F21A
:1040E000FE31C4F2FE3649F63C030022C1F6FF73EE
:1040F00040F203144AF24C0086F88022C4F2040015
:104100002C6081F880225969046083F8382083F894
:10411000392083F85C2083F85D2083F85E2083F8E3
:104120005F200C68486825685A6628439A662060B4
:104130001869827093F861200C680A444FF2CC50E1
:10414000157A527BC0F20E0000EBC50512026D68B5
:1041500002F4E06242F064022A6093F862200A44AA
:1041600093B0957CD27D00EBC5001202406802F44A
:10417000E06242F06402026020684A68104205D0A2
:104180001A692C2151701A69042191711A69202130
:1041900051711B694DF22445C1F6FF7580229A705A
:1041A0002B7B6B720022012BAA7184BF0822AA719B
:1041B000322012F0BDF84DF22440697BC1F6FF7049
:1041C0000DF064F84FF47A7012F0B2F84DF224401A
:1041D000C1F6FF7030210DF059F841F6B0644DF290
:1041E0002440C1F6FF703021C0F204040DF00AF83B
:1041F0002346013BFDD14DF22440C1F6FF70302132
:104200000DF044F84DF22440C1F6FF7030210CF05F
:10421000F9FF013CFDD14DF22440C1F6FF70302181
:104220000DF034F84DF22440C1F6FF7030210CF04F
:10423000E9FF42F22833013BFDD14DF22440C1F6A3
:10424000FF7020210DF022F84DF22440C1F6FF70DE
:1042500020210CF0D7FFA9794DF2244041F0200134
:10426000C1F6FF7000220DF02DF804234DF224401A
:10427000EB7100220C21C1F6FF700DF023F84DF216
:104280002440C1F6FF700DF095F802244DF2244051
:10429000C1F6FF70002206212C720DF013F84DF2CA
:1042A00024402146C1F6FF7000220DF00BF84DF2BC
:1042B000C043C0F20103013BFDD1EB794DF2244034
:1042C00003F0FE0343F00801EB71C1F6FF7000221A
:1042D0000CF0F8FFEB794DF2244003F0FD030022CF
:1042E00043F00801EB71C1F6FF700CF0EBFF0823FF
:1042F0004DF224406B730021C1F6FF700CF0C6FF35
:104300004DF22440C1F6FF700DF054F84DF22440F8
:104310000022C1F6FF7001210DF028F84EF6187149
:104320004DF22440C0F20E01C1F6FF7004F02EFCE5
:104330004DF224400122C1F6FF7000210DF016F865
:104340004EF628714DF22440C0F20E01C1F6FF7006
:104350004DF29C494DF63415C1F6FF7504F016FC7C
:10436000C1F6FF794FF47A7011F0E2FF4DF2605818
:104370004946284612F0E2FBC1F6FF784DF2E863A9
:1043800041461E46284612F0D9FB4DF224673346BB
:10439000C1F6FF73C1F6FF771E46394628464DF237
:1043A000AC7B12F0CBFBC1F6FF7B314628464DF6C5
:1043B000700AC1F6FF7A009612F0C0FB59462846F3
:1043C00012F0BCFB5146284612F0B8FB4DF688109F
:1043D0002946C1F6FF7085F852400CF005FF48F2FF
:1043E00021721046C0F2000048F2D15215460190E9
:1043F0002846019DC9F808504FF0010589F8C150C1
:1044000088F8C15087F8C150C0F20000009D0290AA
:104410004FF0010985F8C1904DF62036029DC8F88D
:104420000C50C1F6FF76009D8BF8C1904AF6910CB6
:104430004AF6693E4BF24D024AF671534DF6981119
:10444000C0F2000CC0F2000EC0F20002C0F2000385
:104450003046C1F6FF71C7F810C0C5F814E0CBF8BC
:104460001820CAF81C308AF8C19012F067FB4DF68C
:104470005C213046C1F6FF7112F060FB4DF68433CB
:104480001D464DF674304EF268274DF64843C1F68E
:10449000FF773146C1F6FF75C1F6FF73C1F6FF70B5
:1044A00086F852401E460CF09FFE4DF60C532946EE
:1044B00038460093069512F041FB009B02964DF69C
:1044C000D052C1F6FF733146384616461D4612F0EB
:1044D00035FB3246C1F6FF7216464DF69462294608
:1044E00038460095154612F029FB2A46C1F6FF72A0
:1044F0001546314638464DF6587BC1F6FF7B03968C
:104500004EF21C0A12F01AFB29463846C1F6FF7A11
:1045100004954EF2E00912F011FB5946384612F0AC
:104520000DFBC1F6FF79514638464EF2A41812F041
:1045300005FBC1F6FF784946384612F0FFFA4146BE
:10454000384612F0FBFA4EF2BC204EF25443394684
:10455000C1F6FF73C1F6FF7087F8524005930CF067
:1045600043FE4AF60D0108464AF2E9310D46C0F213
:10457000000007904AF26D3128460A46C0F200005A
:10458000089010464AF2ED12029DC0F2000201921C
:104590004FF0010285F8C120009D8BF8C12085F8FD
:1045A000C120039D8AF8C1204AF2F12785F8C12075
:1045B0003E46049D89F8C120C0F2000009903046B3
:1045C000069E85F8C120079D3562029D86F8C120B0
:1045D0002E46089D7562009D88F8C1202E46099DD3
:1045E000B562039DC0F200000A902E460A9DF56256
:1045F0004AF2857C049D0598C0F2000C4AF2692EAF
:104600004AF2F5674AF275634EF2CC21C5F830C024
:10461000C0F2000EC0F20003019ACBF834E0C0F201
:104620000007C1F6FF71C9F83C20C8F84030CAF84D
:10463000387012F083FA059D4EF290312846C1F68B
:10464000FF7112F07BFA4EF2A8402946C1F6FF70C6
:104650004EF24068C1F6FF7885F852400CF0C4FD78
:104660004EF2B8414046C1F6FF7112F067FA4EF2C1
:104670007C514046C1F6FF7112F060FA4EF2946030
:104680004146C1F6FF704EF62C07C1F6FF7788F859
:1046900052400CF0A9FD4EF2A4613846C1F6FF71FC
:1046A00012F04CFA4EF268713846C1F6FF7112F002
:1046B00045FA4EF680003946C1F6FF704EF61826D0
:1046C000C1F6FF7687F852400CF08EFD4EF6900151
:1046D0003046C1F6FF7112F031FA4EF654113046F1
:1046E000C1F6FF7112F02AFA4EF66C203146C1F67F
:1046F000FF704EF60447C1F6FF7786F852400CF083
:1047000073FD4EF67C213846C1F6FF7112F016FAA1
:104710004EF640313846C1F6FF7112F00FFA4EF6F0
:1047200058403946C1F6FF704EF6F056C1F6FF7696
:1047300087F852400CF058FD4EF668413046C1F6FD
:10474000FF7112F0FBF94EF62C513046C1F6FF71A5
:1047500012F0F4F94EF644603146C1F6FF704EF6A1
:10476000DC77C1F6FF7786F852400CF03DFD4EF63F
:1047700054613846C1F6FF7112F0E0F94EF6187137
:104780003846C1F6FF7112F0D9F94FF230003946C0
:10479000C1F6FF704FF2C816C1F6FF7687F8524097
:1047A0000CF022FD4FF240013046C1F6FF7112F0CD
:1047B000C5F94FF204113046C1F6FF7112F0BEF98F
:1047C0004FF21C203146C1F6FF704FF2B437C1F6EC
:1047D000FF7786F852400CF007FD4FF22C21384647
:1047E000C1F6FF7112F0AAF94FF2F0213846C1F676
:1047F000FF7112F0A3F94FF218424FF208404FF246
:10480000DC43C1F6FF733946C1F6FF72C1F6FF7093
:1048100087F852400093019240F268360CF0E4FCB5
:10482000019A0F92C2F200061146304612F086F944
:10483000009B0E934FF2A05B1946C1F6FF7B3046FA
:104840004FF2646A12F07AF9C1F6FF7A594630469F
:1048500012F074F94FF228795146304612F06EF991
:10486000C1F6FF794FF6B0034FF2EC78C1F6FF784E
:1048700049461D46304612F061F9C1F6FF754FF604
:104880007413414630462F461D4612F057F94FF635
:104890003822394630460097174612F04FF93A460B
:1048A000C1F6FF721746C1F6FF754FF6FC22294686
:1048B00030460195154612F041F92A46C1F6FF72BD
:1048C000394630461546029712F038F94FF6844EB5
:1048D00029463046039575464FF6C03712F02EF93B
:1048E0002946C1F6FF774FF6485EC1F6FF710D46C7
:1048F000304639460497774612F020F939464FF68C
:104900000C6EC1F6FF710F46304629460595754677
:1049100012F014F929464FF6D06EC1F6FF710D461C
:10492000304639460697774612F008F939464FF671
:10493000947EC1F6FF710F463046294607957546AD
:1049400012F0FCF8294640F2580EC1F6FF710D46F0
:10495000304639460897774612F0F0F8394640F26B
:104960001C1EC2F200010F463046294609957546C5
:1049700012F0E4F8294640F2E01EC2F200010D46B2
:10498000304639460B97774612F0D8F8394640F250
:10499000A42EC2F200010F46304629460C957546FA
:1049A00012F0CCF82946C2F200010D4630463946D5
:1049B0000D9712F0C3F8294630460A9512F0BEF85A
:1049C00040F2BC303146C2F2000086F852400CF092
:1049D0000BFC0F9A4FF0010382F8C1300E9B4FF091
:1049E000010583F8C1508BF8C1508AF8C15089F88D
:1049F000C15088F8C150009DAE464FF001058EF8B9
:104A0000C150019DAE464FF001058EF8C150029D88
:104A1000AE464FF001058EF8C150039DAE464FF0F3
:104A200001058EF8C150049DAE464FF001058EF889
:104A3000C150059DAE464FF001058EF8C150069D50
:104A4000AE464FF001058EF8C150079DAE464FF0BF
:104A500001058EF8C150089DAE464FF001058EF855
:104A6000C1504AF27111099DC0F20001AE46516475
:104A70004AF2F5064AF2790049F6FD714AF2F1521E
:104A8000C0F20006C0F200004FF00105C0F20001C4
:104A9000C0F200028EF8C1509E64CBF84C00CAF8F8
:104AA000501049F60976C9F85420009DC0F200065E
:104AB000EE6549F68D60019DC0F2000028664AF25D
:104AC0006D5E029DC0F2000EC5F864E049F6116CFF
:104AD000039DC0F2000CC5F868C049F6955A049DC4
:104AE000C0F2000AC5F86CA049F61952059DC0F243
:104AF00000022A6749F68573069D4AF2E949C0F229
:104B00000003C0F20009C8F85830C5F874904AF2A2
:104B10006548079DC0F20008C5F878804AF6F54B55
:104B2000089DC0F2000BC5F87CB04AF6C976099D15
:104B30004AF67943C0F20006C0F200030093C5F8BC
:104B400080600B9D009EC5F884604FF001024AF61C
:104B5000457085F8C1204AF6B5630C9D0D9EC0F2E4
:104B6000000001904FF00102184685F8C120C0F204
:104B700000004FF001020E9086F8C1200A9A4FF013
:104B8000010E82F8C1E02A4640F25457019DC2F856
:104B90008850C2F200070A9A0E9DC6F88C504AF659
:104BA000F13340F2CC31C0F20003C2F200013846CA
:104BB000C2F8903011F0C2FF40F290413846C2F284
:104BC000000111F0BBFF40F2A8503946C2F20000CC
:104BD00040F24078C2F2000887F852400CF004FB23
:104BE00040F2B8514046C2F2000111F0A7FF40F276
:104BF0007C614046C2F2000111F0A0FF40F29470C7
:104C00004146C2F2000040F62C16C2F2000688F8B7
:104C100052400CF0E9FA40F2A4713046C2F20001B1
:104C200011F08CFF40F668013046C2F2000111F02D
:104C300085FF40F680103146C2F2000040F618377A
:104C4000C2F2000786F852400CF0CEFA40F69011FE
:104C50003846C2F2000111F071FF40F65421384687
:104C6000C2F2000111F06AFF40F66C303946C2F220
:104C7000000040F60456C2F2000687F852400CF0DD
:104C8000B3FA40F67C313046C2F2000111F056FF13
:104C900040F640413046C2F2000111F04FFF40F6AD
:104CA00058503146C2F2000040F6F067C2F20007E9
:104CB00086F852400CF098FA40F668513846C2F235
:104CC000000111F03BFF40F62C613846C2F20001B2
:104CD00011F034FF40F644703946C2F2000041F250
:104CE000DC06C2F2000687F852400CF07DFA40F66E
:104CF00054713046C2F2000111F020FF41F2180158
:104D00003046C2F2000111F019FF41F23010314675
:104D1000C2F2000041F2C827C2F2000786F85240F2
:104D20000CF062FA41F240113846C2F2000111F073
:104D300005FF41F204213846C2F2000111F0FEFEE7
:104D400041F21C303946C2F2000041F2B446C2F2D0
:104D5000000687F852400CF047FA41F22C313046F9
:104D6000C2F2000111F0EAFE41F2F0313046C2F227
:104D7000000111F0E3FE41F208503146C2F200009A
:104D800041F2A067C2F2000786F852400CF02CFAFC
:104D900041F218513846C2F2000111F0CFFE41F243
:104DA000DC513846C2F2000111F0C8FE41F2F46055
:104DB0003946C2F2000041F68C06C2F2000687F8BE
:104DC00052400CF011FA41F204713046C2F2000177
:104DD00011F0B4FE41F2C8713046C2F2000111F088
:104DE000ADFE41F6E0003146C2F2000041F6782700
:104DF000C2F2000786F852400CF0F6F941F6F001D5
:104E00003846C2F2000111F099FE41F6B41138465D
:104E1000C2F2000111F092FE41F6CC203946C2F2F6
:104E2000000041F66446C2F2000687F852400CF0DA
:104E3000DBF941F6DC213046C2F2000111F07EFEC2
:104E400041F6A0313046C2F2000111F077FE41F682
:104E5000B8403146C2F2000041F65067C2F2000786
:104E600086F852400CF0C0F941F6C8413846C2F20B
:104E7000000111F063FE41F68C513846C2F2000188
:104E800011F05CFE41F6A4603946C2F2000042F225
:104E90003C06C2F2000687F852400CF0A5F941F634
:104EA000B4613046C2F2000111F048FE41F678715B
:104EB0003046C2F2000111F041FE42F2900031464C
:104EC000C2F2000042F22827C2F2000786F85240E0
:104ED0000CF08AF942F2A0013846C2F2000111F04A
:104EE0002DFE42F264113846C2F2000111F026FE96
:104EF00042F27C203946C2F2000042F21446C2F26D
:104F0000000687F852400CF06FF942F28C213046CF
:104F1000C2F2000111F012FE42F250313046C2F2EC
:104F2000000111F00BFE42F268403146C2F200006F
:104F300042F20067C2F2000786F852400CF054F9C2
:104F400042F278413846C2F2000111F0F7FD42F218
:104F50003C513846C2F2000111F0F0FD42F25460BB
:104F60003946C2F2000042F2EC76C2F2000687F83F
:104F700052400CF039F942F264613046C2F200014D
:104F800011F0DCFD42F228713046C2F2000111F04E
:104F9000D5FD42F640003146C2F2000042F6D81775
:104FA000C2F2000786F852400CF01EF942F650019A
:104FB0003846C2F2000111F0C1FD42F61411384624
:104FC000C2F2000111F0BAFD42F62C203946C2F2BD
:104FD000000042F6C436C2F2000687F852400CF0D8
:104FE00003F942F63C213046C2F2000111F0A6FD61
:104FF00042F600313046C2F2000111F09FFD42F648
:1050000018403146C2F2000086F8524043F6AC47E1
:105010000CF0EAF843F62433C2F20003C2F20007B0
:105020004AF64562C0F2000219464FF001053846C3
:1050300083F8C150C3F8A42011F080FD43F6E83195
:105040003846C2F2000111F079FD42F6284B43F6D2
:10505000005042F63876C2F200063946C2F2000B22
:10506000C2F2000042F6EC4A87F85240C2F2000A4F
:105070000CF0BAF842F6B0595946304611F05EFDD0
:10508000C2F200093046514642F6746811F056FDEE
:10509000C2F200083046494611F050FD3046414604
:1050A00011F04CFD42F68C703146C2F2000043F222
:1050B0002417C2F2000786F852400CF095F84AF621
:1050C00069264AF6E92E4AF6C5524AF6E11342F637
:1050D0009C71C0F2000EC0F20002C0F20003C0F2E8
:1050E0000006C2F200013846CBF894E0C9F89C20D3
:1050F000C8F8A0308BF8C1508AF8C15089F8C15067
:1051000088F8C150CAF8986011F018FD43F26001A8
:10511000C2F20001384611F011FD43F27810394611
:10512000C2F2000043F21035C2F2000587F8524087
:105130000CF05AF843F288112846C2F2000111F02F
:10514000FDFC43F24C212846C2F2000111F0F6FCAE
:1051500043F264302946C2F2000043F2FC46C2F238
:10516000000685F852400CF03FF843F274313046A7
:10517000C2F2000111F0E2FC43F238413046C2F2C3
:10518000000111F0DBFC43F250503146C2F2000046
:1051900043F2E865C2F2000586F852400CF024F8AC
:1051A00043F260512846C2F2000111F0C7FC43F2FD
:1051B00024612846C2F2000111F0C0FC43F23C70A9
:1051C0002946C2F2000043F6D406C2F2000685F872
:1051D00052400CF009F843F24C71C2F20001304623
:1051E00011F0ACFC43F61001C2F20001304611F0A0
:1051F000A5FC43F628103146C2F2000043F6C02554
:10520000C2F2000586F852400BF0EEFF43F638116B
:105210002846C2F2000111F091FC43F6FC11284629
:10522000C2F2000111F08AFC43F614302946C2F2A2
:10523000000085F852400BF0D7FF4DF68810C1F6FC
:10524000FF7006F0E1FF4DF67430C1F6FF7006F016
:10525000DBFF4EF2BC20C1F6FF7006F0D5FF40F236
:10526000BC30C2F2000006F0CFFF4EF2A840C1F6FB
:10527000FF7006F0C9FF4EF29460C1F6FF7006F0B1
:10528000C3FF4EF68000C1F6FF7006F0BDFF4EF67C
:105290006C20C1F6FF7006F0B7FF4EF65840C1F61D
:1052A000FF7006F0B1FF4EF64460C1F6FF7006F0E5
:1052B000ABFF4FF23000C1F6FF7006F0A5FF4FF2D2
:1052C0001C20C1F6FF7006F09FFF4FF20840C1F6A8
:1052D000FF7006F099FF40F2BC30C2F2000006F009
:1052E00093FF40F2A850C2F2000006F08DFF40F29A
:1052F0009470C2F2000006F087FF40F68010C2F200
:10530000000006F081FF40F66C30C2F2000006F0AB
:105310007BFF40F65850C2F2000006F075FF40F6E1
:105320004470C2F2000006F06FFF41F23010C2F28A
:10533000000006F069FF41F21C30C2F2000006F0E6
:1053400063FF41F20850C2F2000006F05DFF41F237
:10535000F460C2F2000006F057FF41F6E000C2F22E
:10536000000006F051FF41F6CC20C2F2000006F02A
:105370004BFF41F6B840C2F2000006F045FF41F68F
:10538000A460C2F2000006F03FFF42F29000C2F2B9
:10539000000006F039FF42F27C20C2F2000006F065
:1053A00033FF42F26840C2F2000006F02DFF42F2E5
:1053B0005460C2F2000006F027FF42F64000C2F23D
:1053C000000006F021FF42F62C20C2F2000006F099
:1053D0001BFF42F61840C2F2000006F015FF43F62C
:1053E0000050C2F2000006F00FFF42F68C70C2F2CD
:1053F000000006F009FF43F27810C2F2000006F048
:1054000003FF43F26430C2F2000006F0FDFE43F2F7
:105410005050C2F2000006F0F7FE43F23C70C2F2B8
:10542000000006F0F1FE43F62810C2F2000006F07C
:10543000EBFE43F61430C2F2000006F0E5FE06F083
:10544000ADFE43F61053C2F20003002593F8AD20E1
:1054500053F8224020680BF0ADFF637B04EB83031D
:105460005A6892F8513092F8500008E0834282F86E
:10547000513011D052F8231091F8C11061B9591C64
:105480008342CBB2F2D3002382F8515052F823105A
:1054900091F8C1100029F2D020684BF2C0160BF031
:1054A00089FFC1F6FF76204605F0F6FF06F0D4FC32
:1054B0002B22FF21304614F05FFA4DF27440002396
:1054C000C1F6FF70337011F0EDFA4DF28440C1F671
:1054D000FF7011F0E7FA0123C4F202031B78DB0727
:1054E00041F147804FF0A05349F2D0251A784DF290
:1054F0003443C1F6FF73C1F6FF754FF00009D2B215
:1055000063212A70996183F81C90C3F8149072B6D5
:105510008A42A8BF0A469200DA6062B64FF00508D8
:105520002A7883F83C90C3F83490F262C3F838804C
:1055300072B6C3F82C9062B64EF63C70C0F20E0004
:10554000C6F8309006F012FE4EF68070C0F20E00E3
:1055500006F00CFE4EF6B070C0F20E0006F006FE2D
:105560004EF6E070C0F20E0012F0A6FD4EF224409E
:105570000A214A46C0F20C0012F0A8FD4EF6F47063
:10558000C0F20E0006F0F2FD06F09CFC4EF6FC7038
:10559000C0F20E0006F0EAFD40F644301AF084FE38
:1055A000044645F2A65242F24B4340F6E82AC4F2C2
:1055B0002C72C3F2BE73C0F2020A8260E360302034
:1055C000C4F800A01AF070FE03464FF07C5B204642
:1055D0006360C3F800B00AF029F963682046C3F895
:1055E00004B00AF023F963682046C3F808B00AF053
:1055F0001DF963682046C3F80CB00AF017F9636818
:105600002046C3F810B00AF011F9636846F26662EA
:10561000C3F626725A6120460AF008F963684FF013
:105620007A529A6120460AF001F963682046C3F86D
:105630001CB00AF0FBF86368282222742046C3F8E5
:1056400024B00AF0F3F8636848F20612C3F6156254
:105650009A6220460AF0EAF863680027DF62204673
:105660000AF0E4F804F63C3243F25031C3F6EE514E
:105670000AF10C031160C4F8E03A24236361272384
:10568000A3612B2323652D2363653023C4F88C305D
:105690003323C4F890303723C4F8C8303923C4F812
:1056A000CC303C23C4F804313F23C4F808314323F1
:1056B000C4F840314523C4F844314823C4F87C3150
:1056C0004B23C4F880314F23C4F8B8315123C4F8B8
:1056D000BC315423C4F8F4315723C4F8F8315B23A8
:1056E000C4F830325D23C4F834326023C4F86C321D
:1056F00040F2E733C4F8703242F21C13236241F2E5
:105700003013636242F21D13236343F678736363BD
:1057100041F22733A36343F67973636448F2057358
:10572000A36441F6FE03C4F81C90E36448F20673D8
:10573000A3654AF2A813E36540F6627323664AF252
:10574000A913E3664BF2C0232367384640F2616336
:1057500041F6C14743F22231C0F20107C0F2010114
:1057600063674BF2C123C4F88030C4F898704FF6D9
:10577000BB63C4F8AC1041F6C24240F69B0148F648
:105780002307C0F20102C4F88430C0F2010741F2DD
:105790007D43C4F8B0104CF24961C4F88830C4F8B5
:1057A000A8204FF6BC63C0F20101C4F8C07048F6EF
:1057B00024024FF4C757C4F89430C0F20102C4F871
:1057C000C470C4F8D41043F2233342F6D4014FF22C
:1057D000AD27C0F20103C0F20107C4F8D020C4F81D
:1057E000D8104FF2AE2243F2F121C4F8BC30C0F21F
:1057F0000102C0F20201C4F8E8704CF24A6341F2BF
:105800006147C0F20103C4F8EC70C4F8F820C4F892
:10581000FC1045F21F5740F61B4145F22052C4F8D8
:10582000E430C0F20207C0F20202C4F8001143F2F1
:10583000F2234AF23341C0F20203C0F20201C4F87B
:105840001071C4F8202141F2BC0740F6793240F6CD
:105850004C7CC4F80C31C4F81471C4F82411C4F899
:105860009C204FF2DE07C4F828C1C4F83C2141F661
:105870003672C0F20207C0F20302C4F83871C4F8ED
:105880004C2145F2737741F27C22C0F20307C4F841
:1058900050214AF2344349F24912C0F20203C0F2E5
:1058A0000302C4F8607141F27D27C4F83431C4F8B2
:1058B0006471C4F8742141F6377340F6ED024CF67A
:1058C000CB07C0F20303C0F20307C4F878214FF2FC
:1058D000DF0140F64742C0F20201C4F85C31C0F279
:1058E0000402C4F8887149F24A1341F20207C4F86D
:1058F0004811C0F20303C4F88C71C4F89C2145F22E
:10590000747141F2030244F68F67C0F20301C4F8D8
:105910008431C0F20407C4F8A02140F6484347F69A
:105920009032C4F87011C0F20403C0F20402C4F84B
:10593000B0714CF6CC0140F61967C0F20301C4F80F
:10594000AC31C4F8B471C4F8C42147F6913340F6C1
:105950008E124CF2F647C4F89811C0F20403C0F25C
:105960000407C4F8C82144F6906140F6D81268F3E1
:105970001F42C0F20401C4F8D431C4F8D87140F613
:10598000D91341F6860768F31F43C4F8C011C4F861
:10599000DC71C4F8EC214CF2F74140F6EB0245F221
:1059A000D92768F31F47C0F20401C4F8F021C4F8F6
:1059B000FC3149F26B4249F26C4368F31F4268F3D1
:1059C0001F43C4F8E811C4F8007245F2DA2140F62A
:1059D00081274DF6AD2CC4F8047268F31F4168F3BB
:1059E0001F4C4DF6AE27C4F81422C4F8243241F2FD
:1059F000121243F21D2368F31F47C0F20603C4F8D6
:105A00001012C4F818224DF6AE219D22C4F828C207
:105A100041F2694C68F31F41C0F20602C4F82CC27F
:105A2000C4F8387245F2173C47F20827C4F86432CC
:105A300041F2AA13C0F2060CC0F20607C4F84C12D9
:105A4000C4F860229C2143F21E22C4F8683245F259
:105A50001633C0F20601C0F20603C0F2060247F296
:105A6000A40EC4F89CC240F6790840F6FB2CC4F89A
:105A7000A07240F60217C4F83C12C4F85012C4F8E1
:105A80007832C4F88C32C3F67D7EC4F8A482C4F8A0
:105A900040C2C4F854C2C4F87422C4F88822C4F8BE
:105AA0007C72C4F89072234604F50261C3F8D002F8
:105AB000C3F8D4E2343399424FF00002F6D104F631
:105AC00028310020C4F220300860002304F6F82EAC
:105AD00004F52F61C4F8DC3AC4F8EC3A04F53160FF
:105AE00004F6F42304F60C37CEF800200A604FF0D9
:105AF0007E5102603A602046196009F097FE4BF231
:105B00002003C1F6FF731C6008F05AFF0123C4F2A2
:105B100002031B78DF0740F134854FF0A0520123C8
:105B200012782A70C4F202031B78DC0740F1258545
:105B30000122C1F2004249F2A42343F6C054C2F24A
:105B40000004C1F6FF7312781A7003F001FDA06C17
:105B5000036847F61221DB69984743F6656143F60F
:105B6000F9420327C0F20101C0F2010243F6C53039
:105B700084F8647061602260C0F2010043F65D3316
:105B800043F6E52741F69D6141F64962E060C0F2C7
:105B90000103C0F20107C0F20101C0F2010241F6A7
:105BA000ED506361A7612161E261C0F2010041F63D
:105BB000715341F6155741F6C54141F675422062D1
:105BC000C0F20103C0F20107C0F20101C0F20102FC
:105BD00041F62540A360A762E1622263C0F20100A2
:105BE00041F6D53341F6853741F6353141F6E522A8
:105BF000C0F20101C0F201026063C0F20103C0F211
:105C000001074FF20C00A363E76300234FF6FF7711
:105C100021646264C0F20E0084F84C3084F84E3087
:105C200084F84D30A365636584F8E93084F8663004
:105C300084F8653084F8673084F86830E765276653
:105C400006F094FA4DF21802C4F204024FF2141353
:105C5000C4F20F034FF4807111601A684FF20411FF
:105C6000C4F20F0142F0400240241A600A200C6086
:105C700010F05EFB4FF45842C4F200024FF4804330
:105C80001168C4F2060341F04051116019784FF4D5
:105C9000A042C4F2060241F002011970117848F2E4
:105CA0000403C4F2040341F0800111701A6842F049
:105CB00002021A601A6847F20801C4F2040122F0D5
:105CC00001021A600B6848F23002C4F2040243F485
:105CD00000030B60116843F2040E42F23807C4F26D
:105CE0000A0741F00E0142F2340442F23410C4F2C9
:105CF0000A0E42F2A0031160C4F20A0384224FF09C
:105D00004041C4F20A04C4F20A00CEF8002039600F
:105D10004FF44042012743F24101226007601A46D6
:105D200019601368002BFCDA4FF40053C4F20A0325
:105D300000221A600A2010F0FBFA4FF48A53C4F2D2
:105D40000A0319461A6842F002021A600B689807A3
:105D5000FCD443F22474C2F2010444F2A05044F291
:105D6000A4514BF2F412C1F6FF72C2F20000C2F26B
:105D700000012368226002F12C0407687363046049
:105D800042F6FC730868376602F18C0402F5A677C8
:105D9000C2F20103C6F8C00002F1CC0002F586721F
:105DA0000F60C6F88021C6F80041C6F8400103F133
:105DB0008001012243F8042F8B424FF00106F9D1F4
:105DC00042F248204FF480720021C2F2010013F029
:105DD000D3FD43F21C73C2F2010341F2900841F279
:105DE000A81C0024C4F20A08C4F20A0C1C7041F278
:105DF0004812032341F2541041F24C11C8F80060DC
:105E0000C4F20A02CCF80030C4F20A00C4F20A015B
:105E100043F20003C2F2010341F258174FF48A5EC5
:105E20001460C4F20A070360C4F20A0E0C6048F65C
:105E3000153C41F28411C4F20A01C0F2080C3C6026
:105E4000CEF800C0D1F800E048F200634EF4805E66
:105E5000C1F800E0C1F6FF7346F2F531C0F201016E
:105E60004EF2081E3F680068C3F8B411CEF2000E6F
:105E700004234FF00051C0F20033CEF8001013603D
:105E8000136843F012031360176843F6C063C2F24D
:105E900000034EF2214147F44027C0F200014EF2C8
:105EA00079101760C0F20000C3F868114DF6956EC6
:105EB0004DF611674EF2C5014DF60172C3F870013F
:105EC000C0F2000EC0F20007C0F20001C0F20002F2
:105ED0004DF60150C3F878E1C3F87C71C3F8741132
:105EE000C3F88421C0F200004DF6995E4DF6754767
:105EF0004DF61D414DF6C932C3F88801C0F2000EBF
:105F0000C0F20007C0F20001C0F200024DF6753089
:105F1000C3F86CE1C3F89071C3F89411C3F89821E9
:105F2000C0F200004EF2B12C4DF6213E4DF6CD27C9
:105F30004DF679214DF62522C3F89C01C0F2000CE4
:105F4000C0F2000EC0F20001C0F20002C0F2000771
:105F50004FF22400C3F864C1C0F20E00C3F8A0E100
:105F6000C3F8A471C3F8A811C3F8AC214BF23807E9
:105F700006F0FCF8C1F6FF774DF6991CC0F2000C54
:105F80004BF23402C7F800C0C1F6FF724DF6290C7F
:105F9000C0F2000C4BF24000C2F800C0C1F6FF7026
:105FA0004DF2F16CC0F2000C4BF24801C0F800C099
:105FB000C1F6FF714DF2D15CC0F2000C4BF24C0304
:105FC000C1F800C0C1F6FF734DF24D5CC0F2000C89
:105FD0004BF2440EC3F800C0C1F6FF7E4DF23D6C9B
:105FE000C0F2000C4BF29C17CEF800C0C1F6FF7750
:105FF00041F6211CC0F2010C4BF25002C7F800C060
:10600000C1F6FF7241F6150CC0F2010C4BF23C00D8
:10601000C2F800C0C1F6FF7041F6AD0CC0F2010C31
:106020004BF25401C0F800C0C1F6FF7141F2897C07
:10603000C0F2010C4BF25803C1F800C0C1F6FF7367
:1060400041F2317CC0F2010C4BF25C0EC3F800C08F
:10605000C1F6FF7E41F2DD6CC0F2010C4BF260072D
:10606000CEF800C0C1F6FF7741F2896EC0F2010E92
:106070004BF264024BF26800C7F800E0C1F6FF7211
:10608000C1F6FF7041F2356741F2E15EC0F2010EE8
:10609000C0F201074BF26C014BF27003C1F6FF71C5
:1060A000C1F6FF731760C0F800E041F28D5741F26E
:1060B00039524FF24400C0F20102C0F20107C0F2AF
:1060C0000E001A600F6006F051F84EF28813CEF2FF
:1060D00000031E6072B643F2282E43F22C23C2F254
:1060E0000103C2F2010E40F2002743F2B81021462C
:1060F000C1F6FF77C2F2010070221F60AEF80040C7
:1061000013F03AFC43F2B8102346C2F201005C09D6
:1061100003F01F0150F8242006FA01F101330A436D
:10612000802B40F82420F2D140F20022C1F6FF7209
:10613000002353800133802B02F58272F9D162B6BD
:1061400040F6E470C2F2010009F01EF94FF440720B
:1061500011460E2006F078F90E2006F067F810F0D0
:106160000C0F04D00C2200210E2006F06DF940F631
:10617000E474C2F201044FF6FF7243F63C41102072
:1061800006F062F9E288242122F0100220460AF08B
:106190009BFF44F24002222120460AF095FFE2884C
:1061A000242122F4807220460AF08EFF41F61F72ED
:1061B00041F61A212E2006F047F9204601224FF41D
:1061C00080710AF081FF20B1204670220A210AF076
:1061D0007BFF032202214FF4847006F035F901227F
:1061E00011464FF4927006F02FF9012211464FF438
:1061F000827006F029F94FF26000C0F20E0005F03F
:10620000B5FF43F2B41043F22A21C2F2010043F277
:10621000B612C2F20102C2F2010143F230234EF281
:106220000814C2F20103008809881080CEF200042D
:1062300001224FF27C001980C0F20E00226011F0A2
:106240003BFF00220A21802011F040FF4FF2940012
:10625000C0F20E0011F030FF00220A2140F6553046
:1062600011F034FF4FF2A800C0F20E0040F648567D
:1062700005F07CFFC2F201064BF280330027C1F625
:10628000FF734FF400684FF0000939461846424644
:10629000F784B78437863362C6F82C90A6F8288036
:1062A00040F67C5413F068FBC2F201044CF28033D8
:1062B000C1F6FF73394642461846E784A78427860D
:1062C0002362C4F82C90A4F8288013F055FB40F604
:1062D000B053C2F2010340F62852C2F2010239461D
:1062E000CFF6FF714FF0030E1F629F864FF4803789
:1062F000A3F832E05F6291613046B2EE0E0A09F017
:1063000017FA2046B2EE0E0A09F012FA40F6784269
:1063100040F6B043C2F20102C2F201034FF07857D7
:1063200043F233312878F7624FF40045E762956114
:106330009D61D161D9611162196212F0D9FB43F2FA
:106340002C73C2F201031A78002A48D172B64DF2BA
:10635000B0344FF4304643F24175C1F6FF74C4F2D5
:106360000306C2F2010505220123326004F8303C25
:1063700062B672B633681B060DD414F8303C002B9D
:10638000F1D062B62B78002BF3D111F0B3F872B6CE
:1063900033681B06F1D54BF21003C4F2030300224D
:1063A000186804F8302C62B613F034FB4FF2AC00DE
:1063B000C0F20E0005F0DAFE05F084FD12F0DAFA04
:1063C0004DF29442C1F6FF7240F6FC7312681192CE
:1063D000C2F20103119A1A6013B0BDE8F08F4BF2BC
:1063E00024000146C4F20B01C4F203000268120645
:1063F000FCD40A6812F08002F8D172B61B7843F21E
:106400002C71C2F20101002B00F0B1804BF2380474
:106410004BF23C034BF24000C4F20304C4F203000D
:10642000C4F203034BF2440725681B680468C4F2F6
:1064300003074BF24800C4F203004BF24C061D4424
:10644000C4F203063B6800682C441C4433682044B3
:1064500003444BF22C05C4F20305C3F34E034BF285
:1064600058044BF25C064BF2600043F40043C4F264
:106470000304C4F20306C4F203002B604BF264076A
:10648000256833680468C4F203074BF26800C4F25D
:1064900003004BF26C061D44C4F203063B6800681F
:1064A0002C441C443368204403444BF23005C4F2AE
:1064B0000305C3F34E034BF238044BF23C064BF298
:1064C000400043F40043C4F20B04C4F20B06C4F2D0
:1064D0000B002B604BF24407256833680468C4F254
:1064E0000B074BF24800C4F20B004BF24C061D4464
:1064F000C4F20B063B6800682C441C4433682044FB
:1065000003444BF22C05C4F20B05C3F34E034BF2CC
:1065100058044BF25C064BF2600043F40043C4F2B3
:106520000B04C4F20B06C4F20B002B604BF26407A1
:10653000256833680468C4F20B074BF26800C4F2A4
:106540000B004BF26C061D44C4F20B063B6800685E
:106550002C441C443368204403444BF23000C3F302
:106560004E03C4F20B0043F4004303600A7062B6AA
:10657000ECE60CF0CFF8FEF7B5BF0CF0CBF8FFF768
:10658000D7BA0CF0C7F8FFF7C8BA00BF2DE9F04F33
:106590004DF2A036C1F6FF76304642F20303C3F651
:1065A000000349F2A02241F2950189B040F8043B72
:1065B000C1F6FF72C0F2010113F0A4F949F2A02262
:1065C00041F29501C1F6FF72C0F2010106F10C0023
:1065D00013F098F949F2A02241F29501C1F6FF7239
:1065E000C0F2010106F1140013F08CF949F2A02267
:1065F00041F29501C1F6FF72C0F2010106F11C00E3
:1066000013F080F949F2A02241F29501C1F6FF7220
:10661000C0F2010106F1240013F074F949F2A0223E
:1066200041F29501C1F6FF72C0F2010106F12C00A2
:1066300013F068F949F2A02241F29501C1F6FF7208
:10664000C0F2010106F1340013F05CF949F2A02216
:1066500041F29501C1F6FF72C0F2010106F13C0062
:1066600013F050F949F2A02241F29501C1F6FF72F0
:10667000C0F2010106F1440013F044F949F2A022EE
:1066800041F29501C1F6FF72C0F2010106F14C0022
:1066900013F038F949F2A02241F29501C1F6FF72D8
:1066A000C0F2010106F1540013F02CF949F2A022C6
:1066B00041F29501C1F6FF72C0F2010106F15C00E2
:1066C00013F020F949F2A02241F29501C1F6FF72C0
:1066D000C0F2010106F1640013F014F949F2A0229E
:1066E00041F29501C1F6FF72C0F2010106F16C00A2
:1066F00013F008F949F2A02241F29501C1F6FF72A8
:10670000C0F2010106F1740013F0FCF849F2A02276
:1067100041F29501C1F6FF72C0F2010106F17C0061
:106720004FF2C0070024C0F20E0713F0EBF810255B
:106730000BF0F0FF0223272286F890304FF06048DC
:1067400086F8892003211A4686F88F50C6F884708F
:106750006FF0604506F1940086F8884086F88E4018
:1067600086F8914002F078FE1D221C21C6F8A88010
:10677000C6F8AC5006F1B40086F8B04002F06CFEEA
:10678000D6F8F430079334230799C6F8C88014224A
:10679000C4F2FE33C6F8D410C6F8D820C6F8CC50E0
:1067A00086F8D040C6F8DC4093F80052D6F8F430B2
:1067B000069340F64C03069986F8E0500420C4F294
:1067C000FE33C6F8E82086F8E100C6F8E410C6F803
:1067D000EC4093F80032D6F8F42005924FF01E0EEC
:1067E00086F8F1E0059D86F8F030224607F11003A7
:1067F000012106F1FC00C6F8F85012F095FA0122CA
:1068000007F11C03114606F5E07012F08DFA012223
:1068100007F12803114606F5217012F085FA0122CE
:1068200007F13003114606F5527012F07DFA01228D
:1068300007F13C03114606F20C4012F075FA0122F2
:1068400007F14403114606F59A6006F1840912F037
:106850006BFA07F14C032246012106F5BF6086F86A
:10686000E44586F8E54586F8E74586F8F44586F878
:10687000F545C6F8E89512F057FA49F2A421C1F699
:10688000FF7106F2BC6006F0F9FC07F158032246DE
:10689000012106F2E470C6F8D49786F8D04786F84E
:1068A000D14786F8D34786F8E04786F8E14712F0EB
:1068B0003BFA012207F16003114606F6A80012F028
:1068C00033FA012207F16803114606F66C1012F044
:1068D0002BFA012207F17403114606F5236012F02A
:1068E00023FA012207F17C03114606F6F42012F088
:1068F0001BFA012207F18C03114606F6B83012F09C
:1069000013FA012207F19803114606F67C4012F0B3
:106910000BFA012207F1A003114606F5546012F0AC
:1069200003FA012207F1A803114606F6046012F0EB
:10693000FBF907F1B8032246012106F62C704EF24E
:106940009845C6F81C9F86F8184F86F8194F86F8A8
:106950001B4F86F8284F86F8294F12F0E5F949F2C7
:10696000AC21C1F6FF75C1F6FF7106F57F6006F038
:1069700085FC07F1C003224605F120000121C5F87E
:1069800010902C736C73EC732C776C7712F0CCF93D
:1069900049F2AD2105F1E400C1F6FF7106F06EFC8D
:1069A00007F1C803224605F503700121C5F8FC91E3
:1069B00085F8F84185F8F94185F8FB4185F80842EA
:1069C00085F8094212F0B0F949F2AE2105F53470AC
:1069D000C1F6FF7106F052FC07F1D403224605F51B
:1069E0007E700121C5F8E89385F8E44385F8E54316
:1069F00085F8E74385F8F44385F8F54312F094F9F8
:106A000049F2AF2105F2BC40C1F6FF7106F036FC39
:106A100007F1DC03224605F2E4500121C5F8D495C4
:106A200085F8D04585F8D14585F8D34585F8E0450A
:106A300085F8E14512F078F949F2B02105F5D56005
:106A4000C1F6FF7106F044FC07F1E403224605F5A8
:106A5000FA600121C5F8C09785F8BC4785F8BD47A5
:106A600085F8BF4785F8CC4785F8CD4712F05CF92B
:106A700049F2B12105F69400C1F6FF7106F028FC39
:106A800007F1F003224605F6BC100121C5F8AC99C8
:106A900085F8A84985F8A94985F8AB4985F8B8492A
:106AA00085F8B94912F040F948F6310105F528603A
:106AB000C0F2000106F036FC07F1F803224605F6A5
:106AC000A8300121C5F8989B85F8944B85F8954B23
:106AD00085F8974B85F8A44B85F8A54B12F024F95F
:106AE00049F2B32105F66C40C1F6FF7106F0C6FB12
:106AF00007F58073224605F694500121C5F8849D60
:106B000085F8804D85F8814D85F8834D85F8904D49
:106B100085F8914D12F008F949F2B42105F6586054
:106B2000C1F6FF7106F0AAFB4FF2905A07F5887381
:106B300005F5786022460121C1F6FF7AC5F8709FFD
:106B400085F86C4F85F86D4F85F86F4F85F87C4F51
:106B500085F87D4F12F0E8F8012207F59073114691
:106B6000AAF1B40012F0E0F8012207F5987311467B
:106B70000AF1100012F0D8F8012207F59E731146B1
:106B80000AF1D40012F0D0F8012207F5A4731146DF
:106B90000AF5CC7012F0C8F8012207F5AC73114663
:106BA0000AF5177012F0C0F8012207F5B27311460A
:106BB0000AF5487012F0B8F8012207F5BA731146C9
:106BC0000AF5797012F0B0F8012207F5C273114688
:106BD0000AF5956012F0A8F8012207F5C87311466E
:106BE0000AF26C5012F0A0F8012207F5D07311469A
:106BF0000AF5C66012F098F8012207F5D87311461D
:106C00000AF2F46012F090F8012207F5DE731146E3
:106C10000AF5F76012F088F8012207F5E6731146CD
:106C20000AF67C0012F080F8012207F5EE73114697
:106C30000AF5146012F078F8012207F5F673114690
:106C40000AF6042012F070F8012207F5FE731146CF
:106C50000AF6C82012F068F8012207F503731146FE
:106C60000AF68C3012F060F8012207F5077311461E
:106C70000AF5456012F058F8012207F5097311462C
:106C80000AF6145012F050F807F50C732246012151
:106C90000AF63C60CAF82C9E8AF8284E8AF8294EDB
:106CA0008AF82B4E8AF8384E8AF8394E12F03CF8A2
:106CB00049F2B521C1F6FF710AF5706006F0DEFAFF
:106CC00040F2886841F2140341F2150241F21701C3
:106CD000C2F20008A8F1D0000AF803400AF8024006
:106CE00007F5107322460AF80140012148F8E09C9C
:106CF00008F8D44C08F8D34C12F016F849F2B62133
:106D0000A8F10C00C1F6FF7106F0B8FA07F514738C
:106D1000224608F58E700121C8F80C9188F80841C8
:106D200088F8094188F80B4188F8184188F819411A
:106D300011F0FAFF49F2B72108F5F070C1F6FF71C2
:106D400006F09CFA07F51773224608F542700121F8
:106D5000C8F8F89288F8F44288F8F54288F8F742C3
:106D600088F8044388F8054311F0DEFF48F21D114E
:106D700008F57370C0F2000106F0D4FA07F51A7333
:106D8000224608F2F4400121C8F8E49488F8E0446F
:106D900088F8E14488F8E34488F8F04488F8F1443E
:106DA00011F0C2FF48F2FD0108F5B760C0F2000122
:106DB00006F0B8FA07F51E73224608F5DC600121DB
:106DC000C8F8D09688F8CC4688F8CD4688F8CF46E3
:106DD00088F8DC4688F8DD4611F0A6FF48F2DD01B0
:106DE00008F2A470C0F2000106F09CFA07F52173C6
:106DF000224608F6CC000121C8F8BC9888F8B848AB
:106E000088F8B94888F8BB4888F8C84888F8C9485D
:106E100011F08AFF48F6E10108F51960C0F200019F
:106E200006F080FA07F52573224608F6B8200121FE
:106E3000C8F8A89A88F8A44A88F8A54A88F8A74A02
:106E400088F8B44A88F8B54A11F06EFF48F69D01FB
:106E500008F67C30C0F2000106F064FA07F52973E9
:106E6000224608F6A4400121C8F8949C88F8904C6A
:106E700088F8914C88F8934C88F8A04C88F8A14C7D
:106E800011F052FF48F6590108F66850C0F20001AF
:106E900006F048FA07F52C73224608F569600121CF
:106EA000C8F8809E88F87C4E88F87D4E88F87F4E22
:106EB00088F88C4E88F88D4E41F2807511F034FFC1
:106EC00049F2BE21C2F2000508F65470C1F6FF7106
:106ED00006F0D4F907F530732246A5F17C000121B4
:106EE00045F88C9C05F8904C05F88F4C05F88D4CB6
:106EF00005F8804C05F87F4C11F016FF49F2BF21D0
:106F000005F14800C1F6FF7106F0B8F907F53473D2
:106F1000224605F5B8700121C5F8609185F85C41FD
:106F200085F85D4185F85F4185F86C4185F86D41D4
:106F300011F0FAFE49F2C02105F50D70C1F6FF719E
:106F400006F09CF907F53873224605F557700121C4
:106F5000C5F84C9385F8484385F8494385F84B4379
:106F600085F8584385F8594311F0DEFE48F2ED717B
:106F700005F58460C0F2000106F0D4F907F53C7312
:106F8000224605F5A9600121C5F8389585F83445F4
:106F900085F8354585F8374585F8444585F84545F4
:106FA00011F0C2FE48F2A97105F20C60C0F20001B6
:106FB00006F0B8F907F54073224605F23470012156
:106FC000C5F8249785F8204785F8214785F8234799
:106FD00085F8304785F8314711F0A6FE49F2C32104
:106FE00005F5FF60C1F6FF7106F048F907F5447337
:106FF000224605F512600121C5F8109985F80C4963
:1070000085F80D4985F80F4985F81C4985F81D4913
:1070100011F08AFE49F2C42105F6E410C1F6FF71B1
:1070200006F02CF907F54873224605F60C300121CD
:10703000C5F8FC9A85F8F84A85F8F94A85F8FB4ABC
:1070400085F8084B85F8094B11F06EFE49F2C52111
:1070500005F53D60C1F6FF7106F010F907F54C73B8
:10706000224605F6F8400121C5F8E89C85F8E44C75
:1070700085F8E54C85F8E74C85F8F44C85F8F54C37
:1070800011F052FE49F2C62105F6BC50C1F6FF715F
:1070900006F0F4F807F55073224605F6E460012186
:1070A000C5F8D49E85F8D04E85F8D14E85F8D34EDC
:1070B00085F8E04E85F8E14E42F6780811F034FE8E
:1070C00049F2C721C2F2000805F6A870C1F6FF71A7
:1070D00006F0FEF807F5527322460121A8F12800B8
:1070E00048F8389C08F83C4C08F83B4C08F8394CF8
:1070F00008F82C4C08F82B4C11F016FE49F2C82168
:10710000C1F6FF7108F19C0006F0E2F807F555732F
:107110002246012108F5E270C8F8B49188F8B04120
:1071200088F8B14188F8B34188F8C04188F8C14176
:1071300011F0FAFD49F2A421C1F6FF7108F52270A1
:1071400006F09CF807F558732246012108F56C708B
:10715000C8F8A09388F89C4388F89D4388F89F431B
:1071600088F8AC4388F8AD4311F0DEFD012207F545
:107170005B73114608F2744011F0D6FD012207F549
:107180005F73114608F5A76011F0CEFD012207F5E7
:107190006373114608F2FC5011F0C6FD07F56773E2
:1071A0002246012108F22470C8F8149788F8104785
:1071B00088F8114788F8134788F8204788F821474E
:1071C00011F0B2FD49F2C921C1F6FF7108F5FD6069
:1071D00006F054F807F56A732246012108F511609C
:1071E000C8F8009988F8FC4888F8FD4888F8FF48F6
:1071F00088F80C4988F80D4911F096FD48F62D11D4
:10720000C0F2000108F6D41006F08CF807F56E7392
:107210002246012108F6FC20C8F8EC9A88F8E84AD2
:1072200088F8E94A88F8EB4A88F8F84A88F8F94A71
:1072300011F07AFD48F29501C0F2000108F53C60BA
:1072400006F070F807F572732246012108F6E8404F
:10725000C8F8D89C88F8D44C88F8D54C88F8D74C16
:1072600088F8E44C88F8E54C11F05EFD49F2CC2139
:10727000C1F6FF7108F6AC5006F000F843F6701541
:1072800007F576732246214608F6D460C2F200055F
:10729000C8F8C49E88F8C04E88F8C14E88F8C34E1E
:1072A00088F8D04E88F8D14E11F03EFD07F57A737C
:1072B0002146012208F6987011F036FD07F57C731F
:1072C00022460121A5F1380045F8489C05F84C4CB0
:1072D00005F84B4C05F8494C05F83C4C05F83B4C7F
:1072E00011F022FD49F2D021C1F6FF7105F18C00A9
:1072F00005F0C4FF07F580632246012105F5DA7029
:10730000C5F8A49185F8A04185F8A14185F8A3416D
:1073100085F8B04185F8B14111F006FD48F2510100
:10732000C0F2000105F51E7005F0FCFF95F8B434BD
:1073300085F8B544012249F2D42E43F0010362F3EB
:107340004703C1F6FF7E4FF6FF772146802205F204
:10735000B94085F8B64485F8B74485F8B84485F84F
:10736000394585F8B434C5F898E4C5F8AC74C5F867
:10737000B074C5F8909385F88C4385F88D4385F8F3
:107380008F4385F89C4385F89D4385F84C4485F8E8
:107390004D4485F89C4485F89D4485F89E44C5F885
:1073A000A444C5F8A84412F0E7FA49F2A02248F62E
:1073B0007111C1F6FF72C0F2010105F58A60C5F8CE
:1073C0005044C5F85444C5F85844C5F85C44C5F861
:1073D0006044C5F86444C5F86844C5F86C44C5F811
:1073E0007044C5F87444C5F87844C5F87C44C5F8C1
:1073F0008044C5F88444C5F88844C5F88C44C5F871
:107400009044C5F8944412F07DFA4FF2D443C0F290
:107410000E0305F6282005F6682105F6A822C5F812
:107420005035C5F8640505F6E8234020C5F8681511
:10743000C5F86C255021C5F8743505F5EE62D5F810
:10744000303CA5F87A0505F5FA6005F5E267A5F880
:107450007C15C5F8103705F5036105F50763C5F818
:10746000D027C5F8300C05F50F62D5F8340CC5F8F7
:107470007077C5F83008C5F87018C5F8B03805F54C
:107480001B61C5F8302905F50B6CD5F8382CC5F80B
:10749000341C05F5136705F5176005F51F63C5F87E
:1074A000F029C5F8B446C5F8B846C5F8BC46C5F8D5
:1074B000C046C5F8C446C5F8C846C5F8CC46C5F8A8
:1074C000D046C5F8F0C8C5F87079C5F8B009C5F858
:1074D000383CC5F8D446D5F83C2CC5F8D84605F557
:1074E000AA61C5F8DC46C5F8E046C5F8E446C5F82B
:1074F000E846C5F8EC46C5F8F046C5F8F446C5F8C8
:10750000F846C5F8FC46C5F80047A5F87E45A5F83D
:107510008045C5F85C45C5F86045C5F85845C5F8CF
:10752000544512B900F069BD1A465368002BFBD1CF
:10753000516044F2B058C2F2000800224FF2D44B1E
:107540001746C0F20E0B114640460BF11C0408F51D
:10755000A079C5F850B501F0CFFF3A46394608F199
:10756000A00085F8DC7CC5F8404CC5F8D87C85F8CF
:10757000DD7C01F0C1FF08F5AC724846012185F8B9
:107580007C7DC5F8E04CC5F8787D85F87D7D4FF4AD
:10759000004A01F0B1FF0BF1280408F5BE7247F66E
:1075A000FF73012108F5B270C5F8804DA5F89E3D26
:1075B0000193A5F8A0AD01F09FFF0BF12803C5F8DA
:1075C000A43D08F5C470019BA5F8C23DA5F8C4AD63
:1075D00040F2105405F002FF4AF6D810C2F201043E
:1075E000C2F2000005F0FAFE04F5F26204F5ED6067
:1075F000042101F081FF4FF4803A0BF1340504F5CA
:10760000F96204F5F4600421C4F86857C4F880A74F
:10761000C4F884A7C4F888A7C4F88CA701F06CFF4D
:1076200004F2F47204F5FB600121C4F8A057C4F819
:10763000B8A70BF14005C4F8BCA7C4F8C0A7C4F8AC
:10764000C4A701F059FF04F6140204F5FF600121FC
:10765000C4F8F0A7C4F8D85701F04EFF04F634027E
:1076600004F618000121C4F8F857C4F810A801F076
:1076700043FF04F5056204F638000221C4F81858E7
:10768000C4F830A804F50A6501F036FF0BF14C0A86
:1076900004F6840204F66C000221C4F838A801F054
:1076A0002BFF39463A462846C4F86CA801F024FF5F
:1076B0000BF160024FF0804304F6D800C4F8C838DC
:1076C000C4F8DC98C4F8D888C4F8A028C4F8B878FE
:1076D000C4F8BC78C4F8C078C4F8C478C4F8CC78CE
:1076E000A4F8D078A4F8D278A4F8D47884F8E07814
:1076F00084F8E178C4F8E47884F8E87805F03CFE92
:1077000049F2A02248F62141C1F6FF72C0F2000101
:1077100004F6D80012F0F6F808F5B27304F6EC009F
:10772000C4F8F03808F1A003C4F8EC3884F8F47811
:1077300084F8F578C4F8F87884F8FC7805F01CFE35
:1077400049F2A02248F62141C1F6FF72C0F20001C1
:1077500004F6EC0012F0D6F808F5C47304F51060D6
:10776000C4F80439C4F8008984F8087984F80979E0
:10777000C4F80C7984F8107905F0FEFD49F2A022D6
:1077800048F62141C1F6FF72C0F2000104F5106015
:1077900012F0B8F808F1A003C4F814394AF6D81367
:1077A000C2F2000304F61410C4F8183984F81C79E6
:1077B00084F81D79C4F8207984F8247905F0DCFD7B
:1077C00049F2A02248F62141C1F6FF72C0F2000141
:1077D00004F6141012F096F804F62810A0F1F00345
:1077E000C4F82C39C4F8288984F8307984F83179C0
:1077F000C4F8347984F8387905F0BEFD49F2A02246
:1078000048F62141C1F6FF72C0F2000104F62810CB
:1078100012F078F804F63C10A0F1D003C4F8403917
:1078200008F1A003C4F83C3984F8447984F8457918
:10783000C4F8487984F84C7905F09EFD49F2A022FD
:1078400048F62141C1F6FF72C0F2000104F63C1077
:1078500012F058F804F515604FF00109A0F58C738B
:10786000C4F85439C4F8505984F85879C4F85C798C
:1078700084F8607984F8599905F07EFD49F2A022D8
:1078800048F62141C1F6FF72C0F2000104F515600F
:1078900012F038F804F66410A0F5A673C4F868393D
:1078A000C4F8645984F86C7984F86D79C4F87079F7
:1078B00084F8747905F060FD49F2A02248F6214170
:1078C000C1F6FF72C0F2000104F6641012F01AF85B
:1078D00004F67810A0F5B073C4F87839A0F5867373
:1078E000C4F87C3984F8807984F88199C4F8847963
:1078F00084F8887905F040FD49F2A02248F621413C
:10790000C1F6FF72C0F2000104F6781011F0FAFF20
:1079100004F68C10A0F50973C4F89039C4F88C896A
:1079200084F8947984F89579C4F8987984F89C79E6
:1079300005F022FD49F2A02248F62141C1F6FF726E
:10794000C0F2000104F68C1011F0DCFF04F51A609F
:1079500008F1A003C4F8A039A0F50073C4F8A43955
:1079600084F8A87984F8A979C4F8AC7984F8B07956
:1079700005F002FD49F2A02248F62141C1F6FF724E
:10798000C0F2000104F51A6011F0BCFF04F6B41057
:10799000A0F5BE730225C4F8B439A0F51373C4F87A
:1079A000B83984F8BC79C4F8C07984F8C47984F80B
:1079B000BD5905F0E1FC49F2A02248F62141C1F68B
:1079C000FF72C0F2000104F6B41011F09BFF04F640
:1079D000C810A0F5AE73C4F8C839A0F50A73C4F88E
:1079E000CC3984F8D07984F8D159C4F8D47984F8A2
:1079F000D87905F0C1FC49F2A02248F62141C1F630
:107A0000FF72C0F2000104F6C81011F07BFF04F60B
:107A1000DC1008F5C473C4F8DC39A0F51D73C4F894
:107A2000E03984F8E47984F8E599C4F8E87984F8D1
:107A3000EC7905F0A1FC49F2A02248F62141C1F6FB
:107A4000FF72C0F2000104F6DC1011F05BFF4AF691
:107A5000D81304F51F60C2F20003C4F8F039A0F592
:107A60001473C4F8F43984F8F87984F8F999C4F8EF
:107A7000FC7984F8007A05F07FFC49F2A02248F6F0
:107A80002141C1F6FF72C0F2000104F51F6011F040
:107A900039FF04F60420A0F52773C4F8043AA0F5D2
:107AA0000B73C4F8083A84F80C7A84F80D7AC4F899
:107AB000107A84F8147A05F05FFC49F2A02248F6A7
:107AC0002141C1F6FF72C0F2000104F6042011F05A
:107AD00019FF04F61820A0F51E73C4F8183AA0F593
:107AE0000873C4F81C3A84F8207A84F8217AC4F820
:107AF000247A84F8287A05F03FFC49F2A02248F65F
:107B0000214104F62C2804F61820C1F6FF72C0F2B9
:107B1000000111F0F7FE294604F64422404601F028
:107B2000EBFC04F654200BF16C03A0F51F72C4F8B3
:107B30002C3AC4F8542AC4F8588AC4F84C7AC4F8C9
:107B4000507A84F85C7A84F85D7AC4F8607A84F8B4
:107B5000647A05F011FC49F2A02248F62141C1F6F1
:107B6000FF72C0F2000104F6542011F0CBFE04F6BF
:107B70006820A0F51C73C4F8683AC4F86C8A84F8CD
:107B8000719A84F8707AC4F8747A84F8787A05F077
:107B9000F3FB49F2A02248F6214104F66820C1F621
:107BA000FF72C0F2000111F0ADFE04F6942204F65B
:107BB0007C20294601F0A0FC0BF17803C4F87C3A44
:107BC00072B6B4F89C3A13EA090200F01B829A07D5
:107BD00040F1CA815F0740F11782180740F1168211
:107BE000D90640F116829A0640F116825F0640F1EE
:107BF00016821D0640F11682D80540F116829905BD
:107C000040F116825A0540F116821F0540F1168296
:107C1000DD0440F11682980440F11682590440F1C7
:107C2000A181DA0B08BF4FF00F0900F09D8162B609
:107C300000221023F26286F8303048F23C03C4F28E
:107C4000040348F2400219680020C4F2040241F41F
:107C50000041C4F8A00AC4F8A40A1960116841F0F0
:107C6000020111601A684FF4704142F00202C4F23E
:107C700002011A600B6883427EDB4FF28003C4F27C
:107C800002031B68834277DB4FF47142C4F20202A5
:107C90004FF0804313601368002BFCDB4FF2041598
:107CA000C4F202054FF26003C4F202034FF2FE0E6B
:107CB0004FF20400C5F800E0C4F202004FF0000EDD
:107CC000C3F800E04FF2080101230360C4F202018F
:107CD00018464FF20C07C4F20207C0F200700860A9
:107CE0004FF210024FF480303860C4F2020241F6C5
:107CF0001B7763F31F474FF214054FF2E001176043
:107D0000C4F20205C4F202014FF4F852C1F61F7228
:107D10004FF284072A60C4F20207C1F800E04FF274
:107D200088054FF28C01C4F20205C4F2020141F64B
:107D30001B7C3B6063F31F4CC4F200732B604FF25B
:107D4000900E08604FF294074BF208054BF20C00BE
:107D50004BF21801C4F2020EC4F20207C4F2040589
:107D6000C4F20400C4F204014FF4C063CEF800C0B2
:107D70003A602B6003600B604BF20402C4F2040211
:107D8000F36A94F8A87A4FF4C060106002229A80D7
:107D90009A6048F200414FF22202C4F20202C1F698
:107DA000FF7119601A6140F20112DA804FF47E42CD
:107DB00096F83000CFF6FF72DA604FF48072DA8204
:107DC00000F18040DA8306229A8300F50430002215
:107DD0004FF470459A829A61C4F202058D230270B5
:107DE00003704FF080732B600123C9F2000340F24F
:107DF00010502B60C2F20100002F40F0FC804EF2C8
:107E00004042CEF200024EF20813CEF20003D0251B
:107E1000157001221A60134680F8A82A96F83020BF
:107E200084F8A93A53119B0003F1604301EB8201EE
:107E3000012703F5614340F6695002F01F0207FA7B
:107E400002F2C0F2010048F21B0540F68C78C2F243
:107E50000108C1F84002C4F200051A6096F83030FB
:107E60002B7008F130000025A0F53573C4F8AC3A4A
:107E7000C4F8B08A84F8B45A84F8B55AC4F8B85A29
:107E800084F8BC5A05F078FA49F2A02248F621415C
:107E9000C1F6FF72C0F2000108F1300011F032FDAE
:107EA00008F14400A0F53273C4F8C03A84F8C97AE6
:107EB000C4F8C48A84F8C85AC4F8CC5A84F8D05A92
:107EC00005F05AFA49F2A02248F6214108F144008F
:107ED000C1F6FF72C0F2000111F014FD4FF25853C9
:107EE000C0F20E03C4F8D43A0A2384F8DC3A72B61E
:107EF0004EF218034EF60451CEF20001CEF200030A
:107F00001B68D6F8F4000A6862B6520102D5322B1B
:107F100088BFC019D6F8F4200492049FD6F8F42044
:107F20000392C3F52F3303F21F3346F61741039D27
:107F3000D6F8F4600296C1F2C1619B084FF47A72E0
:107F400002FB00F2A1FB031302EB9303029AC4F8B5
:107F5000E03AC4F8E47AC4F8E85AC4F8EC2A09B064
:107F6000BDE8F08F4FF00E09012202FA09F2134327
:107F7000A4F89C3A62B648F240035FFA89F1C4F271
:107F8000040386F83010186848F23C02C4F2040278
:107F900040F00200186010684FF40045C4F200057C
:107FA00040F00200106009F1007940F2824048F28E
:107FB0001A0748F21E022860C4F2000209F590690F
:107FC000C4F2000748F2180548F21F004FEA4913AF
:107FD000C4F20005C4F2000039701170002229704B
:107FE0000170F3625A601A609A60DA601A615A612D
:107FF0009A61DA6121E6134610E72B46C3F83C1C70
:10800000FFF797BA9146AFE7A946ADE74FF00309EE
:10801000AAE74FF00409A7E74FF00509A4E74FF0DE
:108020000609A1E74FF007099EE74FF008099BE713
:108030004FF0090998E74FF00A0995E74FF00B094F
:1080400092E74FF00C098FE74FF00D098CE700BF66
:108050004BF21C03C1F6FF731B786BB149F2E423AA
:10806000C1F6FF7346F25952C0F2730249F2E4209E
:108070001A60C1F6FF70704749F2E423C1F6FF733E
:1080800046F64E72C0F2200249F2E4201A60C1F6B0
:10809000FF70704749F2A823C1F6FF7393F82330AD
:1080A0006BB149F2E423C1F6FF7346F64F62C0F2AA
:1080B000200249F2E820C1F6FF705A60704749F289
:1080C000E423C1F6FF7346F24F62C0F2660249F242
:1080D000E820C1F6FF705A60704700BF49F2A8233C
:1080E000C1F6FF7349F2EC22C1F6FF72987C02F1EF
:1080F0000C0300280CBF10461846704749F2A8230D
:10810000C1F6FF735B7C032B9DBF4FF2CC72C0F2B4
:108110000E0252F823000020704700BF49F2A82346
:10812000C1F6FF731A7C022A07D84FF2CC73C0F253
:108130000E0303EB8203186970470020704700BFED
:1081400010B4036841681A780C78417A037A0C42BB
:1081500002EA03021AD0837A03F003030AB143F060
:10816000040343F008039A10082B82722AD8072BC5
:1081700022D2032B2ED011D9042B13D0062B14D1CD
:10818000C3685DF8044B023BC3607047837A03F019
:108190000303002AE7D043F00403E4E7012B0BD0EC
:1081A000022B02D1C368013BC3605DF8044B7047EA
:1081B0000D2BF7D00E2BF8D1C3685DF8044B0133BB
:1081C000C36070470C2B05D0F2D8092BD8D00B2BED
:1081D000E8D0EAE7C3685DF8044B0233C360704738
:1081E00041F20003C2F20103D3F8EC00A8E700BF9C
:1081F00041F20003C2F20103D3F8E800A0E700BF98
:1082000041F20003C2F20103D3F8E40098E700BF93
:1082100041F20003C2F20103D3F8E00090E700BF8F
:1082200041F20003C2F20103D3F8DC0088E700BF8B
:1082300041F20003C2F20103D3F8D80080E700BF87
:1082400041F20003C2F20103D3F8D40078E700BF83
:1082500041F20003C2F20103D3F8D00070E700BF7F
:1082600041F20003C2F20103D3F8CC0068E700BF7B
:1082700041F20003C2F20103D3F8C80060E700BF77
:1082800041F20003C2F20103D3F8C40058E700BF73
:1082900041F20003C2F20103D3F8C00050E700BF6F
:1082A00041F20003C2F20103D3F8BC0048E700BF6B
:1082B00041F20003C2F20103D3F8B80040E700BF67
:1082C00041F20003C2F20103D3F8B40038E700BF63
:1082D00041F20003C2F20103D3F8B00030E700BF5F
:1082E00041F20003C2F20103D3F8AC0028E700BF5B
:1082F00041F20003C2F20103D3F8A80020E700BF57
:1083000041F20003C2F20103D3F8A40018E700BF52
:1083100041F20003C2F20103D3F8A00010E700BF4E
:1083200041F20003C2F20103D3F89C0008E700BF4A
:1083300041F20003C2F20103D3F8980000E700BF46
:1083400041F20003C2F20103D3F89400F8E600BF43
:1083500041F20003C2F20103D3F89000F0E600BF3F
:1083600041F20003C2F20103D3F88C00E8E600BF3B
:1083700041F20003C2F20103D3F88800E0E600BF37
:1083800041F20003C2F20103D3F88400D8E600BF33
:1083900041F20003C2F20103D3F88000D0E600BF2F
:1083A00041F20003C2F20103D86FC9E641F20003B3
:1083B000C2F20103986FC3E641F20003C2F2010367
:1083C000586FBDE641F20003C2F20103186FB7E631
:1083D00041F20003C2F20103D86EB1E641F200039C
:1083E000C2F20103986EABE641F20003C2F2010350
:1083F000586EA5E641F20003C2F20103186E9FE633
:1084000041F20003C2F20103D86D99E641F2000384
:10841000C2F20103986D93E641F20003C2F2010338
:10842000586D8DE641F20003C2F20103186D87E634
:1084300041F20003C2F20103D86C81E641F200036D
:10844000C2F20103986C7BE641F20003C2F2010321
:10845000586C75E641F20003C2F20103186C6FE636
:1084600041F20003C2F20103D86B69E641F2000356
:10847000C2F20103986B63E641F20003C2F201030A
:10848000586B5DE641F20003C2F20103186B57E638
:1084900041F20003C2F20103D86A51E641F200033F
:1084A000C2F20103986A4BE641F20003C2F20103F3
:1084B000586A45E641F20003C2F20103186A3FE63A
:1084C00041F20003C2F20103D86939E641F2000328
:1084D000C2F20103986933E641F20003C2F20103DC
:1084E00058692DE641F20003C2F20103186927E63C
:1084F00041F20003C2F20103D86821E641F2000311
:10850000C2F2010398681BE641F20003C2F20103C4
:10851000586815E641F20003C2F2010318680FE63D
:10852000002070470020704730B443F2357343F2A7
:108530003674C2F20103C2F201041A782378D2B26F
:10854000DBB29A422AD001333F2B14D943F288611F
:1085500043F2C863C2F20101C2F20103087819684C
:108560000023C0B2237021B1D31A1A2B01DC0023DF
:108570000B7030BC704743F2886043F2C861C2F2AE
:108580000100C2F20101C05C0968DDB2C0B2257011
:108590000029EED09A4238BF4032E5E74FF0FF3075
:1085A000E7E700BF43F2357243F23673C2F20102CD
:1085B000C2F2010310781B78C0B2DBB2984238BF18
:1085C0004030C01A704700BF084611460FF092B8FD
:1085D000F8B54BF2C0164FF2F470C1F6FF762D21BC
:1085E000C0F20E000FF086F896F902000028BABF1C
:1085F00040422D2200220A2143F610550FF066FD5D
:10860000C2F2000503F05EFC4EF2BC20C1F6FF7022
:1086100003F034FC95F8AD3055F823E09EF80C30AB
:10862000D3B10027384602240EEB8702516891F837
:1086300050206AB1002351F823201471D07090703B
:10864000013391F85020DBB29A42F4D89EF80C30F6
:108650000137FFB29F42E7D34BF2EC11C1F6FF7135
:1086600096F902204B683370002A4BF2C013C1F612
:10867000FF731DDB4DF23443C1F6FF730824002065
:10868000A2424A609C6383F83C005863D4BF9200C6
:10869000202272B6DA6262B695F8AD3055F8234002
:1086A000206808F087FE2046BDE8F84002F0F4BEDE
:1086B0004DF23442C1F6FF7200240820906382F824
:1086C0003C4054639C704C6072B6D46262B695F8BC
:1086D000AD3055F82360306808F06CFE737B06EB14
:1086E00083035A6892F8513092F8500008E098429B
:1086F00082F851300CD052F8231091F8C11039B9DA
:10870000591C9842CBB2F2D8002382F85140F2E7CC
:10871000306808F04FFE304602F0BEFEBCE700BFF6
:108720004FF6240070B5C0F20E0003F01FFD4DF6A9
:108730007430C1F6FF7003F0A1FB49F2A422C1F628
:10874000FF724BF2EC11C1F6FF7112784E684A606D
:108750004BF2C0104DF23443C1F6FF736321C1F6F2
:10876000FF70002501248A42067083F83C505C6348
:10877000996316DC9AB1920072B6DA6262B643F679
:108780001053C2F2000393F8AD2053F82240206842
:1087900008F010FE2046BDE8704002F07DBE0422C5
:1087A000EAE74FF4C672E7E710B549F2A823C1F62D
:1087B000FF73B2EE047A9B7E07EE903AF8EE677A8A
:1087C00049F20434C7EE876AC1F6FF7416EE900AC8
:1087D00010F0C2FD0B464FF644010246C0F20E01F6
:1087E000204617F069FD204610BD00BF10B549F2C4
:1087F000A823C1F6FF73B2EE047A5B7E07EE903ACF
:10880000F8EE677A49F20C34C7EE876AC1F6FF7456
:1088100016EE900A10F0A0FD0B464FF650010246EE
:10882000C0F20E01204617F047FD204610BD00BFE4
:1088300010B549F2A823C1F6FF7349F21434C1F60A
:10884000FF744FF65C0193F90A202046C0F20E0136
:1088500017F032FD204610BD10B549F2A823C1F62D
:10886000FF73B2EE047A5B7D07EE903AF8EE677A1A
:1088700049F22034C7EE876AC1F6FF7416EE900AFB
:1088800010F06AFD0B464FF668010246C0F20E0179
:10889000204617F011FD204610BD00BF10B549F26B
:1088A000A823C1F6FF73B2EE047A1B7D07EE903A5F
:1088B000F8EE677A49F22834C7EE876AC1F6FF748A
:1088C00016EE900A10F048FD0B464FF6680102467E
:1088D000C0F20E01204617F0EFFC204610BD00BF8D
:1088E00008B549F2A823C1F6FF73DA7C72B14FF6DE
:1088F000800149F23030C0F20E01C1F6FF7017F06E
:10890000DBFC49F23030C1F6FF7008BD4FF6740150
:1089100049F23030C0F20E01C1F6FF7017F0CCFC06
:1089200049F23030C1F6FF7008BD00BF08B549F20A
:10893000A823C1F6FF7393F8222072B14FF6940179
:1089400049F23C30C0F20E01C1F6FF7017F0B4FCE2
:1089500049F23C30C1F6FF7008BD4FF68C03C0F2FF
:108960000E0393E8030049F2E423C1F6FF73986510
:1089700083F85C1049F23C30C1F6FF7008BD00BFBF
:1089800010B5044619B1012911D0002010BD55229F
:10899000202108F099FB0028F7D0E28842F0040279
:1089A000204692B22421BDE8104008F08DBB40F271
:1089B00073122A2108F088FB0028E6D088222021A3
:1089C000204608F081FB0028DFD0E288204622F014
:1089D00004022421BDE8104008F076BB38B500231E
:1089E000C4F2013307EE103A47F6EE43C3F6FF63D5
:1089F00007EE903AE0EE077A0546FCEEE77A17EECE
:108A0000902AF2B1802A03799ABFC2F1800444EA25
:108A10000424002433B9224628462221BDE83840E8
:108A200008F052BBC288002322F0100203712421F7
:108A300008F04AFB224628462221BDE8384008F0CB
:108A400043BB0123037147F67F72222108F03CFBF0
:108A5000EA8842F01002284692B22421BDE838404C
:108A600008F032BB10B50846144611460DF0C2FAA4
:108A7000204610BD48F23403C4F204031B685A05B3
:108A800078D543F21473C2F201032DE9F0471B6855
:108A90000BB101221A7043F2CC68C2F2010843F212
:108AA000CD6598F8004001343F2C88BF4FF0000A94
:108AB00043F2D0674FF4204694BF5FFA84FA5446DD
:108AC0008946C2F20105C2F20107C4F206062B78FC
:108AD000A3422AD1EFF31383002B39D1EFF3108394
:108AE000002B35D1EFF30582002A40D00F2A05D99B
:108AF0004EF2F033CEF2000313441B78EFF31182F1
:108B000012B1934228BF1346402B21D9B3F5807F81
:108B1000DDD143F24173C2F201031B78002BD6D1A1
:108B20000EF0E8FC2B78A342D4D043F210734FF43C
:108B30002042C2F20103C4F2060207F804900120A9
:108B4000BC21187088F800A0D1700120BDE8F08722
:108B500033791B06BBD52B7801333F2B86BF002210
:108B60001346DAB2FB5CDBB2F3712A70AFE74FF465
:108B70008073C3E7012070474FF42853C1F2755347
:108B800003EB5100B0FBF1F00DF03EBB70B50446B5
:108B900008460D4612F094F92368024629462046FD
:108BA0005B68BDE87040184710B5037C012B044694
:108BB0002CD972B6E36862B6002BB8BF0333626982
:108BC0009B1093420DDBA1698B4217DC237C012BA8
:108BD00020D972B6E06862B60028B8BF03308010B2
:108BE00010BD237F23B972B69200E26062B6EDE752
:108BF000A3699B0072B6E36062B6E7E7237F002BB0
:108C0000F1D172B68900E16062B6DFE772B6FFF7B4
:108C100097FACFE772B62046FFF792FADAE700BF7D
:108C2000037C10B50446002B31D04368427A5B7A4E
:108C30009A422CD872B60268D3683BB3984202D1EC
:108C400029E09C4202D0DB68002BFAD16368617A8C
:108C50001B6953F8210048B10BF004FD72B663683C
:108C6000627A1B69002143F822102268937A013B43
:108C7000937223689A7A02B91A726268937A013BF6
:108C8000937263689A7A22B10023237462B62046F5
:108C900010BD1A72F8E7C368D360D7E71D2810B576
:108CA0000A4600F0AF8321D92C2800F054813DD82A
:108CB000242800F0B48340F2A280282800F04283E8
:108CC00000F2CE80262800F0DB8140F2AD8241F236
:108CD0000003C2F2010348F22131C0F20001272053
:108CE000C3F89C2003F090FC012010BD0E2800F07A
:108CF000628338D8062800F06B8368D90A2800F010
:108D0000D98200F2FB80082800F06A8140F252828A
:108D100041F20003C2F2010348F2A941C0F200018E
:108D200009205A6203F070FC012010BD342800F0C5
:108D3000848334D8302800F0308300F2CC802E2891
:108D400000F0408140F2E58141F20003C2F20103EC
:108D500048F2A121C0F200012F20C3F8BC2003F08B
:108D600053FC012010BD152800F03F8360D919285D
:108D700000F0DE8100F29D80172800F0748140F23F
:108D8000A68241F20003C2F2010348F2F531C0F2BB
:108D9000000118201A6603F037FC012010BD3828A6
:108DA00000F0A38270D8362800F0278140F2598263
:108DB00041F20003C2F2010348F22121C0F2000196
:108DC0003720C3F8DC2003F01FFC012010BD02286F
:108DD00000F0E38140F26281042800F0378140F224
:108DE000928241F20003C2F2010348F2D941C0F27B
:108DF000000105205A6103F007FC012010BD202866
:108E000000F0218240F27281222800F0118140F2AC
:108E1000A78241F20003C2F2010348F26131C0F2BD
:108E200000012320C3F88C2003F0EEFB012010BDCD
:108E3000112800F0978140F24581132800F0EB8063
:108E400040F29D8141F20003C2F2010348F2254144
:108E5000C0F2000114201A6503F0D6FB012010BDFA
:108E60002A2800F0A18040F2C28141F20003C2F240
:108E7000010348F2E121C0F200012B20C3F8AC202D
:108E800003F0C2FB012010BD3A287FD0C0F04B8216
:108E90003B2840F0468241F20004C2F2010448F24D
:108EA000E111C0F20001C4F8EC2003F0ADFB012099
:108EB00010BD1B285DD040F2628241F20003C2F275
:108EC000010348F2C531C0F200011C201A6703F00B
:108ED0009BFB012010BD322822D040F2798141F263
:108EE0000003C2F2010348F26121C0F20001332005
:108EF000C3F8CC2003F088FB012010BD0C281DD046
:108F000040F2848141F20003C2F2010348F2794148
:108F1000C0F200010D205A6303F076FB012010BD62
:108F200041F20003C2F2010348F27121C0F20001D4
:108F3000C3F8C82003F068FB012010BD41F2000314
:108F4000C2F2010348F28541C0F200011A6303F046
:108F50005BFB012010BD41F20003C2F2010348F2A5
:108F6000D121C0F20001C3F8B02003F04DFB012075
:108F700010BD41F20003C2F2010348F2D131C0F248
:108F80000001DA6603F040FB012010BD41F200034E
:108F9000C2F2010348F2F111C0F20001C3F8E82067
:108FA00003F032FB012010BD41F20003C2F20103C5
:108FB00048F2F121C0F20001C3F8A82003F024FB1D
:108FC000012010BD41F20003C2F2010348F2B121B9
:108FD000C0F20001C3F8B82003F016FB012010BD59
:108FE00041F20003C2F2010348F2B541C0F20001B0
:108FF0001A6203F009FB012010BD41F20003C2F226
:10900000010348F23121C0F20001C3F8D82003F077
:10901000FBFA012010BD41F20003C2F2010348F245
:109020003141C0F20001DA6403F0EEFA012010BD14
:1090300041F20003C2F2010348F27131C0F20001B3
:10904000C3F8882003F0E0FA012010BD41F20003CC
:10905000C2F2010348F2E541C0F200011A6103F0D7
:10906000D3FA012010BD41F20003C2F2010348F21D
:109070000141C0F20001DA6503F0C6FA012010BD1B
:1090800041F20003C2F2010348F23131C0F20001A3
:10909000C3F8982003F0B8FA012010BD002800F0B2
:1090A000EF80012840F03D8141F20003C2F201034C
:1090B00048F20951C0F2000101205A6003F0A4FAFD
:1090C000012010BD0F2800F0E880102840F0298111
:1090D00041F20003C2F2010348F25541C0F200011F
:1090E00010201A6403F090FA012010BD1E282CD025
:1090F0001F2840F0168141F20003C2F2010348F23A
:10910000A131C0F200011F20DA6703F07DFA0120CF
:1091100010BD41F20003C2F2010348F2C121C0F2C6
:1091200000012D20C3F8B42003F06EFA012010BD19
:1091300041F20003C2F2010348F2E931C0F200013A
:109140005A6603F061FA012010BD41F20003C2F239
:10915000010348F2AD31C0F200019A6703F054FAFE
:10916000012010BD41F20003C2F2010348F249415F
:10917000C0F200015A6403F047FA012010BD41F229
:109180000003C2F2010348F23D41C0F20001122087
:109190009A6403F039FA012010BD41F20003C2F2D3
:1091A000010348F2FD41C0F200019A6003F02CFA7D
:1091B000012010BD41F20003C2F2010348F2C14197
:1091C000C0F200010720DA6103F01EFA012010BD91
:1091D00041F20003C2F2010348F28121C0F2000112
:1091E0003120C3F8C42003F00FFA012010BD41F272
:1091F0000003C2F2010348F20131C0F2000129204C
:10920000C3F8A42003F000FA012010BD41F20003CE
:10921000C2F2010348F29141C0F200010B20DA6270
:1092200003F0F2F9012010BD41F20003C2F2010384
:1092300048F24131C0F200012520C3F8942003F028
:10924000E3F9012010BD41F20003C2F2010348F22C
:109250009131C0F20001C3F8802003F0D5F901205C
:1092600010BD41F20003C2F2010348F24121C0F2F5
:1092700000013520C3F8D42003F0C6F9012010BD49
:1092800041F20003C2F2010348F21551C0F200019D
:109290001A6003F0B9F9012010BD41F20003C2F2D7
:1092A000010348F26141C0F20001DA6303F0ACF956
:1092B000012010BD41F20003C2F2010348F29D41BA
:1092C000C0F200019A6203F09FF9012010BD41F243
:1092D0000003C2F2010348F20D41C0F20001162062
:1092E0009A6503F091F9012010BD41F20003C2F22A
:1092F000010348F21121C0F20001C3F8E02003F09D
:1093000083F9012010BD41F20003C2F2010348F2CB
:10931000F141C0F200010320DA6003F075F9012089
:1093200010BD002010BD41F20003C2F2010348F25B
:109330000121C0F200013920C3F8E42003F064F9F0
:10934000012010BD41F20003C2F2010348F21131C5
:10935000C0F20001C3F8A02003F056F9012010BDAF
:1093600041F20003C2F2010348F28131C0F2000170
:109370002120C3F8842003F047F9012010BD41F2F9
:109380000003C2F2010348F2DD31C0F200011A20ED
:109390009A6603F039F9012010BD41F20003C2F2D0
:1093A000010348F29121C0F20001C3F8C02003F08C
:1093B0002BF9012010BD41F20003C2F2010348F273
:1093C0006D41C0F200019A6303F01EF9012010BD47
:1093D00041F20003C2F2010348F2CD41C0F20001A4
:1093E0009A6103F011F9012010BD41F20003C2F2AD
:1093F000010348F21941C0F200015A6503F004F973
:10940000012010BD41F20003C2F2010348F2B9315C
:10941000C0F200015A6703F0F7F8012010BD41F2D5
:109420000003C2F2010348F25131C0F20001C3F857
:10943000902003F0E9F8012010BD41F20003C2F2D0
:10944000010348F25121C0F20001C3F8D02003F01B
:10945000DBF8012010BD00BFF8B53F294FF2CC5317
:1094600004461546C0F20E030AD803EBC10253F8B6
:1094700031605268002740F2031086F88072106055
:109480003F2D0AD803EBC50253F835005268002778
:1094900040F2031680F88072166053F8316053F87A
:1094A000350006F50077276000F500770122676038
:1094B0004DF2C043002762F31F4322726272E760DD
:1094C000013BFDD196F8003290F8002203F0010331
:1094D000D20744BF43F00203DBB2A3720846214621
:1094E000FFF7DCFB214620742846FFF7D7FB237CDF
:1094F000184420742046F8BD10B44FF2F0740023D5
:10950000C0F20E044172026104600372C36041B193
:10951000194600E0026942F82310427A01339A4268
:10952000F8DC43F2B013C2F201031A680AB90CE086
:109530001A465369002BFBD150610023436183809D
:10954000C38083725DF8044B70471860F5E700BF75
:109550002DE9F04149F2A425C1F6FF7540F2A4407F
:109560009AB00B21C0F202000EF0C4F800220A21CA
:1095700028780EF0ABFD02F0A5FC0123C4F2020333
:109580002C781B78DE0740F19D830123C1F2004354
:109590001B789C422ED00123C4F202031B78D8070B
:1095A00040F169830123C1F200431B789C4221D022
:1095B0004EF20302C4F207021378802B00F070838E
:1095C0000022C4F20202137813F0700340F05183BA
:1095D0000123C1F2004301221C70C4F2020213787D
:1095E000D907FCD54EF20302C4F207021378012B0F
:1095F00000F044832F78013F07EB8707FF004FF00F
:109600000108BC1CC4F202082A370DF1FF360DE038
:1096100098F80030DB0740F1F58204F1A0530134E3
:109620001B78BC42DBB206F8013F08D0B4F5805F7E
:10963000EED301340023BC4206F8013FF6D14FF6C9
:109640009C04C0F20E040FCC0AAE37460FC70FCCF5
:109650000FC70FCC0FC794E80F004FF0FF3487E817
:109660000F0001A911F8013B83EA04021AA802F0D5
:109670000F0200EB8202B14252F8402C82EA14142D
:1096800084EA131303F00F0300EB830353F8403C09
:1096900083EA14146FEA0404E4D14FF6DC000E21CF
:1096A000C0F20E000EF026F800220A2128780EF0F3
:1096B0000DFD4FF6EC000821C0F20E000EF01AF876
:1096C0002B78013B03EB8303D800002210210230EA
:1096D0000EF0FCFC4FF6F8001421C0F20E000EF064
:1096E00009F8009F0022102138460EF0EFFC4FF6DB
:1096F00010100521C0F20E000DF0FCFF0022102119
:10970000204649F2A4260EF0E1FCA742C1F6FF76FE
:1097100000F07B824FF62010C0F20E0002F026FD12
:109720000123C4F2020334781B78D90740F19E82EA
:109730000123C1F200431B789C422ED00123C4F2C6
:1097400002031B78DA0740F1C0820123C1F2004313
:109750001B789C4221D04EF20302C4F20702137818
:10976000802B00F0C7820022C4F20202137813F0AB
:10977000700300D013700123C1F2004301221C705A
:10978000C4F202021378DB07FCD54EF20302C4F2E6
:1097900007021378012B00F09B8205F011F94FF6B8
:1097A00050100F21C0F20E000DF0A4FF49F2D0239B
:1097B000C1F6FF73002218780A210EF087FC02F030
:1097C00081FB4FF660100721C0F20E000DF092FFF2
:1097D00049F2A82400220A212878C1F6FF740EF06D
:1097E00075FC02F06FFB4FF668100C21C0F20E0002
:1097F0000DF080FF0022102120680EF067FC02F0BF
:1098000061FB4FF678100721C0F20E000DF072FFD9
:1098100000220A2120790EF059FC02F053FB4FF68A
:1098200080100921C0F20E000DF064FF00220A2111
:1098300060790EF04BFC02F045FB4FF68C100A21CC
:10984000C0F20E000DF056FF00220A21A0790EF0A2
:109850003DFC02F037FB4FF698100821C0F20E00D5
:109860000DF048FF00220A21E0790EF02FFC02F0F3
:1098700029FB4FF6A4100821C0F20E000DF03AFFAC
:1098800094F908000028B6BF2D22002240420A2188
:109890000EF01CFC02F016FB4FF6B0100B21C0F2CC
:1098A0000E000DF027FF94F909000028B6BF2D2205
:1098B000002240420A210EF009FC02F003FB4FF6A1
:1098C000BC100621C0F20E000DF014FF94F90A003E
:1098D0000028B6BF2D22002240420A210EF0F6FBDE
:1098E00002F0F0FA4FF6C4100821C0F20E000DF09D
:1098F00001FF00220A21E07A0EF0E8FB02F0E2FA12
:109900004FF6D0101021C0F20E000DF0F3FE002231
:109910000A21207B0EF0DAFB02F0D4FA4FF6E410B5
:109920001721C0F20E000DF0E5FE00220A21607B37
:109930000EF0CCFB02F0C6FA4FF6FC101321C0F279
:109940000E000DF0D7FE00220A21A07B0EF0BEFB18
:1099500002F0B8FA4FF610200A21C0F20E000DF006
:10996000C9FE00220A21E07B0EF0B0FB02F0AAFA49
:109970004FF61C201121C0F20E000DF0BBFE00229C
:109980000A21207C0EF0A2FB02F09CFA4FF6302058
:109990001421C0F20E000DF0ADFE00220A21607C01
:1099A0000EF094FB02F08EFA4FF648201221C0F21E
:1099B0000E000DF09FFE00220A21A07C0EF086FB17
:1099C00002F080FA4FF65C201621C0F20E000DF076
:1099D00091FE00220A21E07C0EF078FB02F072FA80
:1099E0004FF674201321C0F20E000DF083FE00220A
:1099F0000A21207D0EF06AFB02F064FA4FF68820FF
:109A00001221C0F20E000DF075FE00220A21607DC9
:109A10000EF05CFB02F056FA4FF69C201121C0F2CA
:109A20000E000DF067FE00220A21A07D0EF04EFB15
:109A300002F048FA4FF6B0201021C0F20E000DF0EF
:109A400059FE00220A21E07D0EF040FB02F03AFAB6
:109A50004FF6C4200E21C0F20E000DF04BFE002286
:109A60000A21207E0EF032FB02F02CFA4FF6D420B1
:109A70001221C0F20E000DF03DFE00220A21607E90
:109A80000EF024FB02F01EFA4FF6E8200E21C0F281
:109A90000E000DF02FFE00220A21A07E0EF016FB14
:109AA00002F010FA4FF6F8201221C0F20E000DF06D
:109AB00021FE00220A21E07E0EF008FB02F002FAED
:109AC0004FF60C300E21C0F20E000DF013FE0022F6
:109AD0000A21207F0EF0FAFA02F0F4F94FF61C305A
:109AE0001021C0F20E000DF005FE00220A21607F59
:109AF0000EF0ECFA02F0E6F94FF630301121C0F228
:109B00000E000DF0F7FD00220A21A07F0EF0DEFA14
:109B100002F0D8F94FF644300921C0F20E000DF0E2
:109B2000E9FD94F91F000028B6BF2D220022404213
:109B30000A210EF0CBFA02F0C5F94FF650300B2196
:109B4000C0F20E000DF0D6FD94F920000028B6BF3B
:109B50002D22002240420A210EF0B8FA02F0B2F99A
:109B60004FF65C300A21C0F20E000DF0C3FD00225A
:109B70000A2194F821000EF0A9FA02F0A3F94FF699
:109B800068300E21C0F20E000DF0B4FD00220A2153
:109B900094F822000EF09AFA02F094F94FF6783019
:109BA0001021C0F20E000DF0A5FD00220A2194F84C
:109BB00023000EF08BFA02F085F94FF68C3013215A
:109BC000C0F20E000DF096FD00220A2194F8240048
:109BD0000EF07CFA02F076F94FF6A0300A21C0F2BE
:109BE0000E000DF087FD94F925000028BABF404211
:109BF0002D2200220A210EF069FA1AB0BDE8F041C8
:109C000002F060B908F086FD07E53778013F07EB01
:109C10008707FF0049F2A7264FF00108BC1CC1F6D8
:109C2000FF762A37C4F202080CE098F80030D80713
:109C300019D504F1A05301341B78BC42DBB206F8FD
:109C4000013F08D0B4F5805FEFD301340023BC425C
:109C500006F8013FF6D14FF618100521C0F20E00AC
:109C60000DF048FD99E508F055FDE2E708F052FDDA
:109C70005EE51370ACE408F04DFD93E44EF2010391
:109C8000C4F20703602119701378802BFCD148F2CD
:109C90004403C4F204030022C0F206221A60A9E4BD
:109CA00048F244014EF20103C4F204010020C4F260
:109CB0000703C2F22820002608601E701378802B4C
:109CC000FCD07DE408F026FD5FE408F023FD3CE5D0
:109CD0004EF20103C4F20703602119701378802B40
:109CE000FCD148F24403C4F204030022C0F206226D
:109CF0001A6052E548F244014EF20103C4F2040135
:109D00000020C4F20703C2F22820002608601E705B
:109D10001378802BFCD026E54FF6AC3010B5C0F29E
:109D20000E0002F023FA41F6CC20C2F2000002F04D
:109D3000A5F84BF2EC11C1F6FF7149F2A8224BF2E3
:109D4000C010C1F6FF70C1F6FF724DF23443C1F688
:109D5000FF734C68C470127E4A60002063249C63C9
:109D600083F83C00586372B6A242A8BF2246920014
:109D7000DA6262B643F61053C2F2000393F8AD20E4
:109D800053F82240206807F015FB2046BDE810403C
:109D900001F082BB4FF6CC3010B5C0F20E0002F0DD
:109DA000E5F941F6E000C2F2000002F067F84BF27C
:109DB000EC11C1F6FF7149F2A8224BF2C010C1F6B6
:109DC000FF70C1F6FF724DF23443C1F6FF734C6869
:109DD000C470D27D4A60002063249C6383F83C00F9
:109DE000586372B6A242A8BF22469200DA6262B6F7
:109DF00043F61053C2F2000393F8AD2053F822400B
:109E0000206807F0D7FA2046BDE8104001F044BBB7
:109E10004FF6F03010B5C0F20E0002F0A7F941F293
:109E2000F460C2F2000002F029F84BF2EC11C1F626
:109E3000FF7149F2A8224BF2C010C1F6FF70C1F6C3
:109E4000FF724DF23443C1F6FF734C68C470927DCB
:109E50004A60002063249C6383F83C00586372B618
:109E6000A242A8BF22469200DA6262B643F61053BD
:109E7000C2F2000393F8AD2053F82240206807F0A7
:109E800099FA2046BDE8104001F006BB4FF6144099
:109E900010B5C0F20E0002F069F941F21C30C2F2B6
:109EA000000001F0EBFF4BF2EC11C1F6FF7149F23B
:109EB000A8224BF2C010C1F6FF70C1F6FF724DF23E
:109EC0003443C1F6FF734C68C470127D4A600020B1
:109ED00063249C6383F83C00586372B6A242A8BF17
:109EE00022469200DA6262B643F61053C2F20003D1
:109EF00093F8AD2053F82240206807F05BFA204623
:109F0000BDE8104001F0C8BA4FF6344010B5C0F2B9
:109F10000E0002F02BF941F23010C2F2000001F005
:109F2000ADFF4BF2EC11C1F6FF7149F2A8224BF2E2
:109F3000C010C1F6FF70C1F6FF724DF23443C1F696
:109F4000FF734C68C470D27C4A60002060249C631C
:109F500083F83C00586372B6A242A8BF2246920022
:109F6000DA6262B643F61053C2F2000393F8AD20F2
:109F700053F82240206807F01DFA2046BDE8104043
:109F800001F08ABA4FF6584010B5C0F20E0002F048
:109F9000EDF840F64470C2F2000001F06FFF4BF2A2
:109FA000EC11C1F6FF7149F2A8224BF2C010C1F6C4
:109FB000FF70C1F6FF724DF23443C1F6FF734C6877
:109FC000C470927C4A60002001249C6383F83C00AA
:109FD000586372B69200DA6262B643F61053C2F268
:109FE000000393F8AD2053F82240206807F0E2F90F
:109FF0002046BDE8104001F04FBA00BF4FF6784050
:10A0000010B5C0F20E0002F0B1F840F66C30C2F2AA
:10A01000000001F033FF4BF2EC11C1F6FF7149F281
:10A02000A8224BF2C010C1F6FF70C1F6FF724DF2CC
:10A030003443C1F6FF734C68C470127C4A60002040
:10A0400002249C6383F83C00586372B6A242A8BF06
:10A050002246A240DA6262B643F61053C2F200030F
:10A0600093F8AD2053F82240206807F0A3F920466A
:10A07000BDE8104001F010BA4FF6944010B5C0F2A0
:10A080000E0002F073F840F68010C2F2000001F0FA
:10A09000F5FE4BF2EC11C1F6FF7149F2A8224BF22A
:10A0A000C010C1F6FF70C1F6FF724DF23443C1F625
:10A0B000FF734C68C470D27B4A60002063249C63A9
:10A0C00083F83C00586372B6A242A8BF22469200B1
:10A0D000DA6262B643F61053C2F2000393F8AD2081
:10A0E00053F82240206807F065F92046BDE810408B
:10A0F00001F0D2B94FF6B04010B5C0F20E0002F038
:10A1000035F840F29470C2F2000001F0B7FE4BF255
:10A11000EC11C1F6FF7149F2A8224BF2C010C1F652
:10A12000FF70C1F6FF724DF23443C1F6FF734C6805
:10A13000C470927B4A60002063249C6383F83C00D7
:10A14000586372B6A242A8BF22469200DA6262B693
:10A1500043F61053C2F2000393F8AD2053F82240A7
:10A16000206807F027F92046BDE8104001F094B9B7
:10A170004FF6D44010B5C0F20E0001F0F7FF40F2E8
:10A18000A850C2F2000001F079FE4BF2EC11C1F6CA
:10A19000FF7149F2A8224BF2C010C1F6FF70C1F660
:10A1A000FF724DF23443C1F6FF734C68C470527BAA
:10A1B0004A60002063249C6383F83C00586372B6B5
:10A1C000A242A8BF22469200DA6262B643F610535A
:10A1D000C2F2000393F8AD2053F82240206807F044
:10A1E000E9F82046BDE8104001F056B94FF6FC40B2
:10A1F00010B5C0F20E0001F0B9FF4FF21C20C1F6FD
:10A20000FF7001F03BFE4BF2EC11C1F6FF7149F219
:10A21000A8224BF2C010C1F6FF70C1F6FF724DF2DA
:10A220003443C1F6FF734C688470D27A4A600020D0
:10A2300063249C6383F83C00586372B6A242A8BFB3
:10A2400022469200DA6262B643F61053C2F200036D
:10A2500093F8AD2053F82240206807F0ABF8204671
:10A26000BDE8104001F018B94FF6185070B5C0F2B3
:10A270000E0001F07BFF4EF64460C1F6FF7001F066
:10A28000FDFD49F2A823C1F6FF734BF2EC11C1F6B4
:10A29000FF7193F909304E684B604BF2C0104DF2DC
:10A2A0003442C1F6FF726FF01701C1F6FF7000254E
:10A2B00018248B428670B8BF0B46516382F83C501D
:10A2C000946372B6A342A8BF23469B00D36262B6D2
:10A2D00043F61053C2F2000393F8AD2053F8224026
:10A2E000206807F067F82046BDE8704001F0D4B858
:10A2F0004FF6345010B5C0F20E0001F037FF4EF6A5
:10A300006C20C1F6FF7001F0B9FD4BF2EC11C1F603
:10A31000FF7149F2A8224BF2C010C1F6FF70C1F6DE
:10A32000FF724DF23443C1F6FF734C688470D279EA
:10A330004A60002063249C6383F83C00586372B633
:10A34000A242A8BF22469200DA6262B643F61053D8
:10A35000C2F2000393F8AD2053F82240206807F0C2
:10A3600029F82046BDE8104001F096B84FF650504D
:10A3700010B5C0F20E0001F0F9FE4EF68000C1F6F5
:10A38000FF7001F07BFD4BF2EC11C1F6FF7149F259
:10A39000A8224BF2C010C1F6FF70C1F6FF724DF259
:10A3A0003443C1F6FF734C68847092794A60002090
:10A3B00063249C6383F83C00586372B6A242A8BF32
:10A3C00022469200DA6262B643F61053C2F20003EC
:10A3D00093F8AD2053F82240206806F0EBFF2046AA
:10A3E000BDE8104001F058B84FF66C5010B5C0F2FF
:10A3F0000E0001F0BBFE4EF29460C1F6FF7001F05A
:10A400003DFD4BF2EC11C1F6FF7149F2A8224BF26F
:10A41000C010C1F6FF70C1F6FF724DF23443C1F6B1
:10A42000FF734C68847052794A60002063249C63F7
:10A4300083F83C00586372B6A242A8BF224692003D
:10A44000DA6262B643F61053C2F2000393F8AD200D
:10A4500053F82240206806F0ADFF2046BDE81040CA
:10A4600001F01AB84FF6885010B51E21C0F20E0048
:10A470000DF040F901F026FD41F6A460C2F20000A3
:10A4800001F0FCFC4BF2EC11C1F6FF7149F2A8227D
:10A490004BF2C010C1F6FF70C1F6FF724DF23443AB
:10A4A000C1F6FF734C68C470927E4A600020C824D5
:10A4B0009C6383F83C00586372B6A242A8BF224650
:10A4C0009200DA6262B643F61053C2F2000393F8C8
:10A4D000AD2053F82240206806F06CFF2046BDE80E
:10A4E000104000F0D9BF00BF4FF6A85010B5222190
:10A4F000C0F20E000DF0FEF801F0E4FC41F6B840A9
:10A50000C2F2000001F0BAFC4BF2EC11C1F6FF718F
:10A5100049F2A8224BF2C010C1F6FF70C1F6FF72DB
:10A520004DF23443C1F6FF734C68C470527E4A60EA
:10A530000020C8249C6383F83C00586372B6A24292
:10A54000A8BF22469200DA6262B643F61053C2F206
:10A55000000393F8AD2053F82240206806F02AFF4C
:10A560002046BDE8104000F097BF00BF4FF6CC502A
:10A5700010B51C21C0F20E000DF0BCF801F0A2FCD9
:10A5800041F20850C2F2000001F078FC4BF2EC11ED
:10A59000C1F6FF7149F2A8224BF2C010C1F6FF705C
:10A5A000C1F6FF724DF23443C1F6FF734C68C470BC
:10A5B000527D4A60002063249C6383F83C0058630A
:10A5C00072B6A242A8BF22469200DA6262B643F691
:10A5D0001053C2F2000393F8AD2053F822402068D4
:10A5E00006F0E8FE2046BDE8104000F055BF00BF71
:10A5F0004FF6EC5010B51F21C0F20E000DF07AF8A6
:10A6000001F060FC40F65850C2F2000001F036FC48
:10A610004BF2EC11C1F6FF7149F2A8224BF2C010C7
:10A62000C1F6FF70C1F6FF724DF23443C1F6FF73FD
:10A630004C68C470527C4A60002003249C6383F8F9
:10A640003C00586372B6A242A8BF22469200DA626A
:10A6500062B643F61053C2F2000393F8AD2053F8EC
:10A660002240206806F0A6FE2046BDE8104000F01B
:10A6700013BF00BF4FF60C6010B52021C0F20E00D2
:10A680000DF038F84FF20840C1F6FF7001F0F6FB0C
:10A690004BF2EC11C1F6FF7149F2A8224BF2C01047
:10A6A000C1F6FF70C1F6FF724DF23443C1F6FF737D
:10A6B0004C688470127B4A60002063249C6383F89A
:10A6C0003C00586372B6A242A8BF22469200DA62EA
:10A6D00062B643F61053C2F2000393F8AD2053F86C
:10A6E0002240206806F066FE2046BDE8104000F0DB
:10A6F000D3BE00BF4FF6306070B51621C0F20E0019
:10A700000CF0F8FF01F0DEFB4FF23000C1F6FF70F5
:10A7100001F0B4FB49F2A823C1F6FF734BF2EC1130
:10A72000C1F6FF7193F90A304E684B604BF2C010CE
:10A730004DF23442C1F6FF726FF03101C1F6FF7085
:10A74000002532248B428670B8BF0B46516382F8D5
:10A750003C50946372B6A342A8BF23469B00D362C9
:10A7600062B643F61053C2F2000393F8AD2053F8DB
:10A770002240206806F01EFE2046BDE8704000F032
:10A780008BBE00BF4FF6486038B51821C0F20E00EE
:10A790000CF0B0FF01F096FB4EF65840C1F6FF708A
:10A7A00001F06CFB49F2A823C1F6FF734BF2EC11E8
:10A7B000C1F6FF714BF2C0104DF23442C1F6FF7288
:10A7C00093F908304D684B60C1F6FF700021632497
:10A7D00023EAE3738570946382F83C10516372B688
:10A7E000A342A8BF23469B00D36262B643F6105330
:10A7F000C2F2000393F8AD2053F82240206806F01F
:10A80000D9FD2046BDE8384000F046BE4FF66460F2
:10A8100010B51721C0F20E000CF06CFF01F052FBD6
:10A820004EF2A840C1F6FF7001F028FB4BF2EC118C
:10A83000C1F6FF7149F2A8224BF2C010C1F6FF70B9
:10A84000C1F6FF724DF23443C1F6FF734C68847059
:10A8500012794A60002063249C6383F83C005863AB
:10A8600072B6A242A8BF22469200DA6262B643F6EE
:10A870001053C2F2000393F8AD2053F82240206831
:10A8800006F098FD2046BDE8104000F005BE00BF70
:10A89000F8B54BF2C0164FF67C60C1F6FF76292161
:10A8A000C0F20E000CF026FF96F903000028BABF94
:10A8B00040422D2200220A2143F610550DF006FCDD
:10A8C000C2F2000501F0FEFA40F2BC30C2F2000014
:10A8D00001F0D4FA95F8AD3055F823E09EF80C302D
:10A8E000D3B10027384602240EEB8702516891F855
:10A8F00050206AB1002351F823201471D070907059
:10A90000013391F85020DBB29A42F4D89EF80C3013
:10A910000137FFB29F42E7D34BF2EC11C1F6FF7152
:10A9200096F903204B683370002A4BF2C013C1F62E
:10A93000FF731DDB4DF23443C1F6FF731324002077
:10A94000A2424A609C6383F83C005863D4BF9200E3
:10A950004C2272B6DA6262B695F8AD3055F82340F3
:10A96000206806F027FD2046BDE8F84000F094BDC1
:10A970004DF23442C1F6FF7200241320906382F836
:10A980003C405463DC704C6072B6D46262B695F899
:10A99000AD3055F82360306806F00CFD737B06EB94
:10A9A00083035A6892F8513092F8500008E09842B8
:10A9B00082F851300CD052F8231091F8C11039B9F7
:10A9C000591C9842CBB2F2D8002382F85140F2E7EA
:10A9D000306806F0EFFC304600F05EFDBCE700BFDB
:10A9E0004FF6A86070B5C0F20E0001F0BFFB43F255
:10A9F0003C70C2F2000001F041FA49F2A822C1F60F
:10AA0000FF724BF2EC11C1F6FF7192F824204E68F0
:10AA10004A604BF2C0104DF23443C1F6FF73282157
:10AA2000C1F6FF70002501248A42467183F83C502C
:10AA30005C63996316DC9AB1920072B6DA6262B610
:10AA400043F61053C2F2000393F8AD2053F82240AE
:10AA5000206806F0AFFC2046BDE8704000F01CBD49
:10AA60000422EAE7A022E8E74FF6C46010B5C0F27E
:10AA70000E0001F07BFB43F26430C2F2000001F0F3
:10AA8000FDF94BF2EC11C1F6FF7149F2A8224BF22D
:10AA9000C010C1F6FF70C1F6FF724DF23443C1F62B
:10AAA000FF734C68447192F822204A600020102401
:10AAB0009C6383F83C00586372B6A242A8BF22464A
:10AAC0009200DA6262B643F61053C2F2000393F8C2
:10AAD000AD2053F82240206806F06CFC2046BDE80B
:10AAE000104000F0D9BC00BF4FF6E46010B5C0F2D2
:10AAF0000E0001F03BFB43F27810C2F2000001F0BF
:10AB0000BDF94BF2EC11C1F6FF7149F2A8224BF2EC
:10AB1000C010C1F6FF70C1F6FF724DF23443C1F6AA
:10AB2000FF734C68447192F821204A60002063242E
:10AB30009C6383F83C00586372B6A242A8BF2246C9
:10AB40009200DA6262B643F61053C2F2000393F841
:10AB5000AD2053F82240206806F02CFC2046BDE8CA
:10AB6000104000F099BC00BF4FF6007070B5C0F205
:10AB70000E0001F0FBFA42F61840C2F2000001F0AC
:10AB80007DF949F2A422C1F6FF724BF2EC11C1F635
:10AB9000FF7112784E684A604BF2C0104DF2344398
:10ABA000C1F6FF736321C1F6FF70002501248A42BC
:10ABB000067083F83C505C63996316DC9AB192008E
:10ABC00072B6DA6262B643F61053C2F2000393F82B
:10ABD000AD2053F82240206806F0ECFB2046BDE88B
:10ABE000704000F059BC0422EAE74FF4C672E7E770
:10ABF0004FF6207070B5C0F20E0001F0B7FA42F6C1
:10AC00002C20C2F2000001F039F949F2A823C1F664
:10AC1000FF734BF2EC11C1F6FF7193F920304E68CF
:10AC20004B604BF2C0104DF23442C1F6FF726FF030
:10AC30003101C1F6FF70002532248B42C670B8BFC7
:10AC40000B46516382F83C50946372B6A342A8BF8E
:10AC500023469B00D36262B643F61053C2F2000350
:10AC600093F8AD2053F82240206806F0A3FB20465D
:10AC7000BDE8704000F010BC4FF63C7010B5C0F25B
:10AC80000E0001F073FA42F26840C2F2000001F0D7
:10AC9000F5F84BF2EC11C1F6FF7149F2A8224BF224
:10ACA000C010C1F6FF70C1F6FF724DF23443C1F619
:10ACB000FF734C68C470527F4A60002063249C6319
:10ACC00083F83C00586372B6A242A8BF22469200A5
:10ACD000DA6262B643F61053C2F2000393F8AD2075
:10ACE00053F82240206806F065FB2046BDE810407E
:10ACF00000F0D2BB4FF65C7010B5C0F20E0001F050
:10AD000035FA42F29000C2F2000001F0B7F84BF2BF
:10AD1000EC11C1F6FF7149F2A8224BF2C010C1F646
:10AD2000FF70C1F6FF724DF23443C1F6FF734C68F9
:10AD3000C470D27E4A60002064249C6383F83C0087
:10AD4000586372B6A242A8BF22469200DA6262B687
:10AD500043F61053C2F2000393F8AD2053F822409B
:10AD6000206806F027FB2046BDE8104000F094BBA9
:10AD70004FF6807010B51621C0F20E000CF0BAFC30
:10AD800001F0A0F843F62810C2F2000001F076F8B6
:10AD900043F61053C2F200034BF2EC1193F8AD00EE
:10ADA000C1F6FF714BF2C012C1F6FF7253F820409A
:10ADB0004B681370206806F0FDFA2046BDE810408D
:10ADC00000F06ABB4FF6987010B52021C0F20E005B
:10ADD0000CF090FC01F076F843F25050C2F2000003
:10ADE00001F04CF84BF2EC11C1F6FF7149F2A822C8
:10ADF0004BF2C010C1F6FF70C1F6FF724DF2344342
:10AE0000C1F6FF734C68447192F823204A60002019
:10AE100001249C6383F83C00586372B69200DA62A6
:10AE200062B643F61053C2F2000393F8AD2053F814
:10AE30002240206806F0BEFA2046BDE8104000F02F
:10AE40002BBB00BF4FF6BC7010B52021C0F20E0026
:10AE50000CF050FC01F036F843F60050C2F200004E
:10AE600001F00CF84BF21C02C1F6FF724BF2EC1130
:10AE7000C1F6FF714DF23443C1F6FF7312784A6098
:10AE800001200021986383F83C10596372B6920048
:10AE9000DA6262B643F61053C2F2000393F8AD20B3
:10AEA00053F82240206806F085FA2046BDE810409D
:10AEB00000F0F2BA4FF6E07070B51921C0F20E0042
:10AEC0000CF018FC00F0FEFF42F64000C2F2000059
:10AED00000F0D4FF49F2A823C1F6FF734BF2EC1146
:10AEE000C1F6FF7193F91F304E684B604BF2C010F2
:10AEF0004DF23442C1F6FF726FF03101C1F6FF70BE
:10AF0000002532248B42C670B8BF0B46516382F8CD
:10AF10003C50946372B6A342A8BF23469B00D36201
:10AF200062B643F61053C2F2000393F8AD2053F813
:10AF30002240206806F03EFA2046BDE8704000F04E
:10AF4000ABBA00BF4FF6FC7010B52121C0F20E0065
:10AF50000CF0D0FB00F0B6FF42F25460C2F20000E9
:10AF600000F08CFF4BF2EC11C1F6FF7149F2A82200
:10AF70004BF2C010C1F6FF70C1F6FF724DF23443C0
:10AF8000C1F6FF734C68C470927F4A60002063244E
:10AF90009C6383F83C00586372B6A242A8BF224665
:10AFA0009200DA6262B643F61053C2F2000393F8DD
:10AFB000AD2053F82240206806F0FCF92046BDE899
:10AFC000104000F069BA00BF40F2200010B51E2109
:10AFD000C0F20F000CF08EFB00F074FF42F27C20F8
:10AFE000C2F2000000F04AFF4BF2EC11C1F6FF7113
:10AFF00049F2A8224BF2C010C1F6FF70C1F6FF72F1
:10B000004DF23443C1F6FF734C68C470127F4A603E
:10B01000002063249C6383F83C00586372B6A2420C
:10B02000A8BF22469200DA6262B643F61053C2F21B
:10B03000000393F8AD2053F82240206806F0BAF9D7
:10B040002046BDE8104000F027BA00BFF8B54BF22B
:10B05000C01640F24000C1F6FF762921C0F20F0071
:10B060000CF048FB96F905000028BABF40422D229B
:10B0700000220A2143F610550DF028F8C2F200050F
:10B0800000F020FF42F68C70C2F2000000F0F6FEE5
:10B0900095F8AD3055F823E09EF80C30D3B1002779
:10B0A000384602240EEB8702516891F850206AB1AD
:10B0B000002351F823201471D0709070013391F85F
:10B0C0005020DBB29A42F4D89EF80C300137FFB220
:10B0D0009F42E7D34BF2EC11C1F6FF7196F90520C0
:10B0E0004B683370002A4BF2C013C1F6FF731DDBAF
:10B0F0004DF23443C1F6FF7303240020A2424A609C
:10B100009C6383F83C005863D4BF92000C2272B653
:10B11000DA6262B695F8AD3055F82340206806F043
:10B1200049F92046BDE8F84000F0B6B94DF2344286
:10B13000C1F6FF7200240320906382F83C40546300
:10B140005C714C6072B6D46262B695F8AD3055F859
:10B150002360306806F02EF9737B06EB83035A6890
:10B1600092F8513092F8500008E0984282F851303D
:10B170000CD052F8231091F8C11039B9591C9842DB
:10B18000CBB2F2D8002382F85140F2E7306806F0E3
:10B1900011F9304600F080F9BCE700BFF8B504466D
:10B1A0004DF25440C1F6FF70FDF7FEFC4BF2C017A4
:10B1B000C1F6FF77385540F2BC30C2F2000000F013
:10B1C0005DFE43F61053C2F2000393F8AD2053F82E
:10B1D0002260337BCBB100252846022406EB850292
:10B1E000516891F8502062B1002351F82320147166
:10B1F000D0709070013391F85020DBB29A42F4D8AD
:10B20000337B0135EDB29D42E8D34BF2EC114DF2A8
:10B210003442C1F6FF7297F90330C1F6FF71002086
:10B2200013244B60946323EAE37382F83C00506379
:10B2300072B6A342A8BF23469B00D36262B6F8BD94
:10B24000F8B504464DF25440C1F6FF70FDF7ACFC72
:10B250004BF2C017C1F6FF7738554EF2BC20C1F64D
:10B26000FF7000F00BFE43F61053C2F2000393F898
:10B27000AD2053F82260337BCBB100252846022451
:10B2800006EB8502516891F8502062B1002351F815
:10B2900023201471D0709070013391F85020DBB2EC
:10B2A0009A42F4D8337B0135EDB29D42E8D34BF29C
:10B2B000EC114DF23442C1F6FF7297F90230C1F63B
:10B2C000FF71002008244B60946323EAE37382F843
:10B2D0003C00506372B6A342A8BF23469B00D362D2
:10B2E00062B6F8BDF8B504464DF25440C1F6FF70A1
:10B2F000FDF75AFC4BF2C017C1F6FF7738554DF6F3
:10B300008810C1F6FF7000F0B9FD43F61053C2F289
:10B31000000393F8AD2053F82260337BCBB10025B6
:10B320002846022406EB8502516891F8502062B14C
:10B33000002351F823201471D0709070013391F8DC
:10B340005020DBB29A42F4D8337B0135EDB29D42F6
:10B35000E8D34BF2EC114DF23442C1F6FF7297F98B
:10B360000030C1F6FF71002005244B60946323EA8E
:10B37000E37382F83C00506372B6A342A8BF234631
:10B380009B00D36262B6F8BD70B54DF25444C1F66D
:10B39000FF7406462046FDF707FC4BF2C015C1F6C8
:10B3A000FF75A85542F68C70C2F2000000F066FDF1
:10B3B00000F0F4FE4BF2EC12A4F1200095F90530F8
:10B3C000C1F6FF72002103245360846323EAE37310
:10B3D00080F83C10416372B6A342A8BF23469B008D
:10B3E000C36262B670BD00BF2DE9F041091A0026A4
:10B3F00043F610544FB2B046C2F2000487EAE77237
:10B40000F3B2A2EBE772934244DA94F8AD3054F809
:10B410002350002F28681DDA05F0CCFF6B7B05EB6D
:10B4200083035B6893F8501093F85100421C8842E4
:10B43000D2B204D2914283F8512002D122E083F8A3
:10B44000518093F8512053F8222092F8C120002A0D
:10B45000EAD017E005F0AEFF6B7B05EB83035B687A
:10B4600093F851104A1ED2B221B993F8502083F8B4
:10B47000512007E083F8512053F8222092F8C12090
:10B48000002AEDD0286805F095FF284600F004F862
:10B490000136B3E7BDE8F0812DE9F04F49F2783588
:10B4A0009DB0C1F6FF752B7802AF04469BB12A46CA
:10B4B000002302F8043B0F21006800F0FDFB05F1BA
:10B4C0000C020E21206800F0F7FB05F114020D219B
:10B4D000206800F0F1FB637BD4F8009004EB830458
:10B4E0006368BB6393F85220002A40F0AE8393F860
:10B4F0005030FB611846BA6B92F851203A63824291
:10B5000080F0918300247C61B861BA69944280F232
:10B51000F18240F26C02C0F20F023A610022FA633B
:10B520007A6949F63C064CF6CD41C1F6FF76CCF679
:10B53000CC410132B246B960FA604FF0010B97F886
:10B540003C207869FA6211468218D2B2BA62FA696E
:10B550009A4203D2BB6B53F8243019703B69BD6B20
:10B560000FCB55F8248007F1440498F8005098F860
:10B5700001E084E80F0099F8093099F8052086F871
:10B580005EB09D4284BF03F1FF35EDB207F1680361
:10B5900003EB8505520055F8243C86F85DB00EEBB0
:10B5A000030464F07F04E4B2B6F85E3086F83B2012
:10B5B0002501EDB204F0F0043BB199F80D30022200
:10B5C00023438AF83C308AF85D2001200CF094FC7B
:10B5D00099F8053086F85EB0B6F85E2086F85DB062
:10B5E0005B0086F83B304AB199F80D3043F0040314
:10B5F000234302228AF83C308AF85D2001200CF0B7
:10B600007BFC3C23013BFDD199F8053086F85EB008
:10B61000B6F85E2086F85DB05B0086F83B303AB144
:10B6200099F80D301C4302238AF83C408AF85D30BB
:10B6300001200CF061FC40F6B833013BFDD199F8D4
:10B64000053086F85EB0B6F85E2086F85DB05B0027
:10B6500086F83B303AB199F80D3002222B438AF834
:10B660003C308AF85D2001200CF046FC99F805304A
:10B6700086F85EB0B6F85E2086F85DB05B0086F8AE
:10B680003B304AB199F80D3043F004032B430222BA
:10B690008AF83C308AF85D2001200CF02DFC3C2318
:10B6A000013BFDD199F8053086F85EB0B6F85E2012
:10B6B00086F85DB05B0086F83B303AB199F80D3002
:10B6C0001D4302238AF83C508AF85D3001200CF0BB
:10B6D00013FC40F6B833013BFDD141F2613308F170
:10B6E000BC02C0F2010308F1BB0508F1A804C7F8C9
:10B6F00034803B6290467E6215F8012F412A00F0AB
:10B7000056815AD8202A00F0828176D8092A00F082
:10B710002A8100F2B480012A00F0A081082A14D105
:10B72000236893F90020002AC0F2538240F0A682D9
:10B73000302387F8653001222121D9F8003007F144
:10B74000440001445B684846984704344445D3D1DB
:10B750003B6BBA6AD7F834807E6A93421BD198F863
:10B760000420022A00F0AF81032A00F09581012A0B
:10B77000D9F8003000F082811A6888F804B041F2EC
:10B780006133C0F201039A4240F06A8201220F2124
:10B79000484605F097FDFB6AFA681344DCB2FB6B80
:10B7A0000133FB63BB699C4280F2A481BA6B92F8BF
:10B7B00051303B6392F85030C1E6D92A53D032D988
:10B7C000F02A00F03A8149D9FB2A00F0A780FC2A30
:10B7D00000F0A480FA2AB8D12368002BB5D098478E
:10B7E000D9F800303A6A1B689342014640F0A680BF
:10B7F0000122484605F066FDA7E73C2A00F0958047
:10B800006BD8212A00F0A780322A9ED123681868BD
:10B810000DF0A2FD7B6B5B79009302460B46484618
:10B8200007F03AF891E7D02A00F08B8066D8462AD4
:10B830007BD0C92A89D12368002B86D0984707F18D
:10B84000680100280CBF3023312301F8033DD9F8EB
:10B85000003001225B684846984776E7E82A70D0B6
:10B86000E92A7FF472AF2368002B3FF46EAF98474C
:10B87000002301460A22484606F0CEFF65E7102A5B
:10B8800079D0112A7FF461AF23681A88002A3FF427
:10B890004FAFBE68A6FB0213DB0803EB8301A2EBEC
:10B8A0004102303287F86520002B00F0D68121213B
:10B8B000A6FB0302D20802EB82000139A3EB40038E
:10B8C000C9B207F168000844303300F8243C13463D
:10B8D000002AEDD1C1F122022FE73D2A63D03E2A92
:10B8E0007FF433AF266830460FF0EAFAD9F800301B
:10B8F000024631465B684846984726E7D12AB2D0CF
:10B90000D82A7FF422AF2368002B3FF41EAF98475C
:10B9100000280146C0F284810023ABE72368002B96
:10B920003FF413AF98470646DEE72268D9F80030A7
:10B9300011781B683A6A93423FF45AAF48469847D9
:10B9400003E72368002B3FF400AF9847011EE3DABA
:10B9500049422D238EE722680023116848460A22B7
:10B9600006F05AFFF1E622680023117848460A22C1
:10B9700006F052FFE9E62368B3F90020002AC0F27E
:10B98000F3803FF4D5AEBB68A3FB0213DB0803EBE7
:10B990008301A2EB4102303287F86520002B00F0D2
:10B9A0005C810026F0E023681E6830469CE7226830
:10B9B0003A6010460FF084FA38643B6C386CC7F874
:10B9C00004D0073323F00703ADEB030D002802A9D1
:10B9D0003A680BDD0020034603F1010E3E6CD35C98
:10B9E0000B545FFA8EF3B3421846F5DB3B6C3960BB
:10B9F0000022CA5408460FF063FAD9F800303968BB
:10BA00005B68024648469847D7F804D09DE623680D
:10BA10001B68002B72DB3FF48BAEBA68A2FB0321DC
:10BA2000C90801EB8102A3EB4203303387F865308C
:10BA3000002900F01281002670E02368002B3FF4FB
:10BA400084AE984710EE100A0DF086FC02260246DE
:10BA50000B460096484606F01FFF76E623681B78E3
:10BA600007F16801002B0CBF3023312301F8033D9F
:10BA7000D9F8003048465B68984766E641F2613184
:10BA80001B68C0F201018B4248464FF00F0140F0A5
:10BA9000F38005F017FC7EE698F8022098F8031072
:10BAA000484605F063FCD9F8002041F26133126882
:10BAB000C0F201039A4240F0DB8001220D2148468A
:10BAC00005F000FC67E698F8011098F800200139AD
:10BAD000C9B2484605F04AFCD9F8002041F261336A
:10BAE0001268C0F201039A4240F0BE8001220E218A
:10BAF0004846CEE76C37BD46BDE8F08FB9685B427B
:10BB0000A1FB0301C90801EB8100A3EB4003303323
:10BB100087F86530002900F0C6802D262120D7F84F
:10BB200008C000E01846ACFB0132D20802EB820EDE
:10BB3000431EA1EB4E01DBB207F1680E9E4430318B
:10BB40000EF8241C1146002AECD1002E00F0A9802A
:10BB50000238C0B20146C0F1220207F1680318445E
:10BB60002D2300F8243CE8E5BB685242A3FB0213F6
:10BB7000DB0803EB8301A2EB4102303287F865203A
:10BB8000002B00F08A802D262120D7F808C000E085
:10BB90001046ACFB0321C90801EB810E421EA3EB4A
:10BBA0004E03D2B207F1680E964430330EF8243CAF
:10BBB0000B460029ECD1002E79D0831EDBB219464A
:10BBC000C3F1220207F1680003442D2003F8240C7E
:10BBD000B3E5BB685242A3FB0213DB0803EB83010E
:10BBE000A2EB4102303287F86520002B55D02D267C
:10BBF0002120D7F808C000E01046ACFB0321C9089B
:10BC000001EB810E421EA3EB4E03D2B207F1680E88
:10BC1000964430330EF8243C0B460029ECD1CAE799
:10BC200041422D2326E60132121AD2B201461044B7
:10BC300098427A61B86114467FF767AC5A1AD2B25B
:10BC40007A6114468A18BA615FE493F850309A42D8
:10BC500028BF1A46FA6110464DE4012221216CE505
:10BC60000F214846904796E50E214846904792E5B9
:10BC70000D21484690478EE598478CE5BB68A3FBAD
:10BC80000213DB0803EB8301A2EB4102303287F899
:10BC90006520002BE1D00026AAE720210B460222D6
:10BCA00090E7194616E611461046022255E711465E
:10BCB000C2F1220241E500BF2DE9F04F01F007017A
:10BCC000C900914683B041F040010022054649F683
:10BCD0003C0B05F0F7FA41F2613A09F10703C1F6AE
:10BCE000FF7B09F1FF370193C0F2010A0124A3E0B1
:10BCF00068798BF85E40BBF85E308BF85D4001F0F0
:10BD0000F009400009018BF83B00CEB249F0010870
:10BD10005BB1697B49F63C03C1F6FF73022048EA38
:10BD2000010183F83C1083F85D0001200CF0E4F879
:10BD300069798BF85E40BBF85E008BF85D40490086
:10BD40008BF83B1048B1697B41F0050149EA0102DB
:10BD500002218BF83C208BF85D1001200CF0CCF810
:10BD60003C22013AFDD16A798BF85E40BBF85E1047
:10BD70008BF85D4052008BF83B2039B16A7B022181
:10BD800048EA02088BF83C808BF85D1001200CF02B
:10BD9000B3F840F6B832013AFDD16A798BF85E40CB
:10BDA000BBF85E108BF85D4052008BF83B2041B130
:10BDB0006A7B42F00102324302218BF83C208BF86F
:10BDC0005D1001200CF098F86A798BF85E40BBF8A2
:10BDD0005E108BF85D4052008BF83B2041B16A7BCE
:10BDE00042F00502324302218BF83C208BF85D10B3
:10BDF00001200CF081F83C22013AFDD16A798BF8E0
:10BE00005E40BBF85E108BF85D4052008BF83B2023
:10BE100041B1697B41F001010E4302228BF83C6085
:10BE20008BF85D2001200CF067F840F6B832013A3B
:10BE3000FDD1019BBB420BD02A6817F8011F126885
:10BE400052453FF455AF28469047019BBB42F3D182
:10BE500003B0BDE8F08F00BF10B543F61053C2F237
:10BE6000000393F8AD2053F82240206805F0A2FAB1
:10BE70002046BDE81040FFF70FBB00BF38B543F6C2
:10BE80001055C2F2000595F8AC1069B12C688442D7
:10BE90000CD02A46002303E052F8044F844206D017
:10BEA0000133DBB28B42F7D1002038BD002385F887
:10BEB000AD30206805F07EFA2046FFF7EDFA01204C
:10BEC00038BD00BF00B540F27C03C0F20F0383B061
:10BED0001B88ADF80430022101A80BF00BFC03B065
:10BEE0005DF804FB72B641F20813C2F201039A78BE
:10BEF000012A23D01CD3022A07D0032A24D140F2DE
:10BF000078020421C1F6FF7204E040F27002C1F62B
:10BF1000FF7205219970018812F0080F14BFC82321
:10BF20008823083043EA01435060136062B67047CB
:10BF300040F270020321C1F6FF72EBE740F2780293
:10BF40000221C1F6FF72E5E71A6922B11A6B50604F
:10BF5000186362B670471861FAE700BF72B641F223
:10BF60000813C2F20103DA78012A23D01CD3022A73
:10BF700007D0032A24D140F298020421C1F6FF72AF
:10BF800004E040F29002C1F6FF720521D9700188E9
:10BF900012F0080F14BFC8238823083043EA014376
:10BFA0005060136062B6704740F290020321C1F600
:10BFB000FF72EBE740F298020221C1F6FF72E5E75B
:10BFC0005A6922B15A6B5060586362B67047586123
:10BFD000FAE700BF72B641F20813C2F201031B690F
:10BFE00033B100205B680130002BFBD162B6704793
:10BFF0001846FBE799B3012938B540D04378044689
:10C0000000781B0643EA004040F470408D1E40F06B
:10C0100004000BF057FC022D04F1020315D905347E
:10C0200014F8023C14F8032C14F8010C1B0443EA26
:10C03000022343F0040343EA0060033D0BF042FC9B
:10C04000022D234604F10304EAD8022D22D0012D4B
:10C050000BD04FF20570BDE838400BF033BC4FF207
:10C060000600C0F2F7000BF02DBC1878000240F477
:10C07000770040F00600BDE838400BF023BC0378A1
:10C080004FF207001B04CFF200701843BDE83840A0
:10C090000BF018BC5A781878130443EA002040F0DB
:10C0A000774040F00700BDE838400BF00BBC00BF04
:10C0B00099B3012938B540D04378044600781B066F
:10C0C00043EA004040F470408D1E40F004000BF045
:10C0D000A7FF022D04F1020315D9053414F8023C20
:10C0E00014F8032C14F8010C1B0443EA022343F058
:10C0F000040343EA0060033D0BF092FF022D234648
:10C1000004F10304EAD8022D22D0012D0BD04FF206
:10C110000570BDE838400BF083BF4FF20600C0F257
:10C12000F7000BF07DBF1878000240F4770040F074
:10C130000600BDE838400BF073BF03784FF20700EC
:10C140001B04CFF200701843BDE838400BF068BF05
:10C150005A781878130443EA002040F0774040F002
:10C160000700BDE838400BF05BBF00BF10B50446C8
:10C170000EF0A6FE014620460BF0BCFA0446FFF77F
:10C18000A1FE204410BD00BF10B500220A210BF013
:10C190009DFF0446FFF796FE204410BD70B443F6A1
:10C1A0001053C2F2000393F8AD2053F82260337BA2
:10C1B000CBB100252846022406EB8502516891F890
:10C1C000502062B1002351F823201471D070907078
:10C1D000013391F85020DBB29A42F4D8337B013519
:10C1E000EDB29D42E8D3012070BC7047002810B525
:10C1F000BABF40422D2200220A210BF067FF0446FD
:10C20000FFF760FE204410BD43F61053C2F2000356
:10C2100093F8AC202A2A06D8511C43F8220083F850
:10C22000AC10012070470020704700BFF0B540F609
:10C23000E47549F63C04C1F6FF74C2F2010501221F
:10C240002B7A84F85E20B4F85E1084F85D20934069
:10C2500089B084F83B3039B1020A032384F83D00E9
:10C2600084F83C2084F85D3000200BF045FE10B1CE
:10C27000002009B0F0BD23692E7A84F8380012221C
:10C2800084F83900DA702269937849F63C0503F0A6
:10C29000200303F0FF07C1F6FF75002B00F0A78015
:10C2A000B42393704DF29442C1F6FF722169136872
:10C2B0000793079D06E013680693069B5B1B042B00
:10C2C00000F29080CB7803F0200303F0FF00002BF6
:10C2D000F1D0730043F00103DBB20B7113680593D7
:10C2E000059D216905E013680493049B5B1B052BE6
:10C2F00078D8CB7803F0020303F0FF00002BF2D0D4
:10C300000223CB702169C87849F63C0310F0110F65
:10C31000C1F6FF7340F08180A020887019690B7905
:10C3200013680393039D05E013680293029B5B1B54
:10C33000052B67D8CB7803F0020303F0FF00002B36
:10C34000F2D00223CB702069C178C9B249F63C0310
:10C35000CE06C1F6FF738BD48D0689D5A8218170D6
:10C3600019690879156801951876019805E0136830
:10C370000093009B1B1A052B52D8CB7803F00203C5
:10C3800003F0FF05002BF2D00225CD702169CB7898
:10C39000DBB249F63C02D806C1F6FF7248D49B06D0
:10C3A0007FF566AFB0238B7013691979517600BFA2
:10C3B00000BF00BF8021997092F8383082F8395060
:10C3C000012B26D8D1180133087ED9B202294FEAB1
:10C3D000002382F838101CD0507E82F83850184361
:10C3E00009B0F0BD8870236980229A7040E70BF095
:10C3F000FFFA00283FF43CAF2B6985F85F70B0224C
:10C400009A704FE78870236980229A7084F8390007
:10C410002EE74FF0FF3009B0F0BD80238B7027E787
:10C420008D70226980210123917084F839301FE7D3
:10C4300010204FF49673C870013BFDD112699378B8
:10C4400003F0F703937013E770B50D4614460646E4
:10C45000FFF7ECFE20EA040040EA050440F6E47031
:10C4600031462246C2F2010004F02EFE002814BF1D
:10C470002046002070BD00BFF3EE047A80EE277ADC
:10C480002DE9704F054614460E4604F00104640180
:10C490002DED048B17EE100A82B0B0EE609AF0EE2C
:10C4A000418A0CF059FF9FED508A41EC110B9FED32
:10C4B0004C0B11F03DFEC9EE087A5BEC10ABF1EECF
:10C4C000677A17EE900A0CF047FF9FED450B41ECA1
:10C4D000110B11F02DFEC8EE887A59EC108BF1EE9D
:10C4E000677A17EE900A0CF037FF9FED3D0B41EC99
:10C4F000110B11F01DFE45F61C234FF02042C3F630
:10C50000E473504659468DED000B0CF0C9FF002333
:10C51000C4F2E00300220CF0C3FF0DF0D3F9C2B265
:10C5200040F6E4704FF49371C2F2010004F0CCFDC8
:10C53000002142464B460020C3F6F0710CF0ACFDE2
:10C540000023C4F2201300220CF0AAFF0DF0BAF968
:10C55000C2B240F6E4704FF49471C2F2010004F0EC
:10C56000B3FD9DED000B002153EC102B0020C3F612
:10C57000F0710CF091FD0023C4F2601300220CF066
:10C580008FFF0DF09FF9C2B240F6E4704FF4957141
:10C59000C2F2010004F098FD4FF49270FFF746FEDE
:10C5A000022D06F0030144EA012128BF022520F4F0
:10C5B0004C5020F0200041EA0534044340F6E4707A
:10C5C0002246C2F201004FF4927104F07DFD00B1E9
:10C5D000A0B202B0BDEC048BBDE8708FAFF3008059
:10C5E000000000000000244000555749002810B505
:10C5F000BABF40422D2200220A210BF067FD0446FB
:10C60000FFF760FC204410BDF0B44FF2CC54C0F2F0
:10C610000E0404EBC0035A68136813F4E06301D1FD
:10C620003F2856D948F20063C1F6FF7349F27127DB
:10C63000C1F6FF7749F24126C1F6FF76C3F82C71A7
:10C6400002F1404749F2112549F2E11449F2B110D3
:10C65000C3F83061A7F59226C1F6FF75C1F6FF74E5
:10C66000C1F6FF707C2EC3F83451C3F83841C3F8CB
:10C670003C0129D9A7F594237C2B10D9A7F5962343
:10C680007C2B33D9A7F598237C2B2AD9A7F59A2799
:10C690007C2F17D849F29434C1F6FF7403E049F2B5
:10C6A0007044C1F6FF7472B6136823F4702343F02C
:10C6B0008570C2F3840540F48030136044F825107F
:10C6C000106062B6F0BC704749F2D044C1F6FF7406
:10C6D000E9E754F830404FF4807084F880321060FD
:10C6E000A0E749F20044C1F6FF74DCE749F2404498
:10C6F000C1F6FF74D7E700BF013BDBB20F2B1BD89D
:10C700002DE9F04145B2002D01DBBDE8F081E028C4
:10C7100013D9F728F9D900F10803DAB201239340BD
:10C7200013F0DD0FF1D0014643F60860C2F20000BD
:10C73000BDE8F04103F094BA704743F6C058C2F226
:10C7400000081646D8F848E0DEF8002048F67527BD
:10C750001268C0F200072B43BA42044601F07F057D
:10C76000D8B222D109F0CEFCD8F8480003681B6883
:10C77000BB4217D1284609F0C5FC04F0EF00C028E1
:10C78000C3D0D8F8482013681B68BB4206F07F006E
:10C7900003D1BDE8F04109F0B5BC0146BDE8F04168
:10C7A0001046184729469847E7E7014670469047E4
:10C7B000DAE700BF72B642F20003C2F20103586822
:10C7C00050B101885A8C10B4521A44685C605A8483
:10C7D00062B65DF8044B704762B6704772B642F2BB
:10C7E0000003C2F20103186950B101881A8D10B418
:10C7F000521A44681C611A8562B65DF8044B704792
:10C8000062B67047C368BBB110B401E0DB688BB19E
:10C810001A7A002AFAD15A68587A126952F82040D6
:10C82000002CF3D142F820100A7801320A70DB683C
:10C83000002BEDD15DF8044B704700BFF0B44FF40E
:10C840004044C4F202044FF000462368FE2743F43C
:10C85000806323602246E6622346676335464C1CAC
:10C8600001F20127D16A0029FCDA196814F8016C79
:10C8700041F480611960DD625E63D16A0029FCDAEF
:10C88000196814F8026B41F48061A7421960DD62F7
:10C890005E63E7D14FF44041C4F20201CA6A4FF42B
:10C8A0004043002AC4F20203F8DA1A684FF0004548
:10C8B00042F48062FF241A601946DD625C63CA6A32
:10C8C0004FF44043002AC4F20203F8DA1A684FF02A
:10C8D000004542F48062FF241A601946DD625C6301
:10C8E000CA6A4FF44043002AC4F20203F8DA1A6815
:10C8F0004FF0004542F48062FF241A601946DD6261
:10C900005C63CA6A4FF44043002AC4F20203F8DAB7
:10C910009B6BDBB203F01F024370A2F10500B0FA7B
:10C9200080F04009F0BC70472DE9F04F8468066A3A
:10C9300083B0002C55D0002301340193F368591CB7
:10C940008846A3B3A045274638BF022442F2000A16
:10C9500049F2485B38BF27468C428146C2F2010A41
:10C96000C1F6FF7B4FF0000521D896F82030F06922
:10C97000102BDBF8003022D000EBD410984222D1EB
:10C9800004F07F030AEB83031B6B23F0704393B126
:10C9900001342746F3680135AB4208D9A04538BFBA
:10C9A000022403F1010138BF27468C42DDD9002063
:10C9B00003B0BDE8F08FBC4217D00134EAE700EBCA
:10C9C0001420984208D0002104F016FD0028EED073
:10C9D00096F82030102BD3D1E3B20AEB43031B8E21
:10C9E000D5E7012334680193A8E7012FDFD9F36865
:10C9F00001339F42DBD86FF070423946304604F075
:10CA000013FD0028D3D0D9F8081059B10129CED987
:10CA1000F36801339942CAD83A46304604F004FD1F
:10CA20000028C4D0019BC9F808700BB17B1C33608F
:10CA3000D9F81C305BB999F80530C9F81C7063F05F
:10CA40007F03012089F8053003B0BDE8F08F012095
:10CA500003B0BDE8F08F00BF38B50269D478E4B206
:10CA6000E106054628D51023D370630623D504F0CC
:10CA7000040404F0FF03002C62D042F20003C2F26F
:10CA80000103696E002283F8302285F85D200029B9
:10CA90006ED0884795F85D30002B69D02B69D02285
:10CAA0009A702B6995F83B201A712B69012285F841
:10CAB0005C200222DA7038BD04F0400303F0FF006E
:10CAC000002BD4D19379DBB203F06001602956D0FA
:10CAD000937803F0100303F0FF01B3B114F00104E5
:10CAE0003FD195F85C3095F85D10994253D9591CA7
:10CAF0002B4485F85C1093F83B3013712B69D022DE
:10CB00009A702B690222DA70D5E785F86010937964
:10CB100043F0200393712B6995F839101A791F2976
:10CB2000D2B2C6D842F20000C2F2010090F8300240
:10CB30000028BED06818013185F839100276B8E7B0
:10CB40002A6985F83930C02393702B6942F20002BC
:10CB5000C2F201021979012182F830120222DA7040
:10CB6000A9E7C02393702B691A790222DA70A2E731
:10CB70000122002385F85D2085F83B308EE703F025
:10CB8000DF039371AB6E23B185F8380095F8390057
:10CB900098472A699CE71471B0E700BF2DE9F04F70
:10CBA00044F2A454C2F200042268002A66D013683A
:10CBB0002360002B00F09A8042F20005C2F20105CA
:10CBC0008B46B5F8466219682160002E52D148F2B2
:10CBD00080141360C8F2000442F2402CC2F2010C2F
:10CBE0002CF47F614FF4207921F00F014FF0010EFA
:10CBF000C0F20809C2F804E001F5805AC2F80890B2
:10CC0000C2F80CC001F5005901F5405C01F5804106
:10CC1000C2F810A0C2F81490C2F818C0D161C3F8CD
:10CC200004E0D5F84412D5F8408205689D629C6006
:10CC300099634FF0000C4FF48059C3F834804FF4DF
:10CC4000005A4FF440554FF480440068C3F80CC0BC
:10CC5000C3F83CC0C3F81090C3F82CB0C3F814A0BC
:10CC60001E639D611146DC61C3F800E0BDE8F04F32
:10CC700008F0E6BD29B911601A6023600020BDE804
:10CC8000F08F95F940820F6827604FEA064C6FEAF3
:10CC900008044CF0004C4FEAD878E40F2BF47F6E78
:10CCA0004CF0800C2EF00F0E4CEA082C4FF00109CE
:10CCB0002402C1F804900EF58058C1F808C00EF5A2
:10CCC00000590EF5405C44F080240EF5804EC1F80A
:10CCD0000CB044F08004C1F81080C1F81490C1F881
:10CCE00018C0C1F81CE011600B6075E7136022608A
:10CCF000C4E700BF2DE9F04F44F2A054C2F2000493
:10CD000089B0D4F800A00594BAF1000F74D026467B
:10CD100044F2A454C2F20004274607943D68DAF8AE
:10CD20000040346006952E46002D00F0748288463F
:10CD30001D460392336802918146019060220021D2
:10CD4000402450463B600CF017FE2246002130463E
:10CD50000CF012FE43460122EDB2032B3260414635
:10CD6000B460CAF810608AF83550CAF83090CAF832
:10CD700014208AF8348000F0A280039B4BB1019B01
:10CD80005A680AB96FE21A46936B002BFBD1C2F8BE
:10CD900038A0029B002B33D1019B9AF837001D7DF0
:10CDA000039F9AF83630012D8CBF00210121C9065E
:10CDB0004FF48042019E747D44F0704444EA07249D
:10CDC000129F44EA07442143114341EA0532CAF85D
:10CDD0000420B27DF17D120442EAC15242F0804249
:10CDE000134343EA0023CAF80830029B33F00203DE
:10CDF00010D0029B032B1FD0504609B0BDE8F08F26
:10CE0000019B9AF837001D7D039F9AF83630002267
:10CE10001146CFE741F25812C4F20A021368002B00
:10CE200000F00B821A68CAF8002050464AF002024D
:10CE30001A6009B0BDE8F08FBAF84200BAF84010A5
:10CE40001F28D9D843F20005C2F201054AF00206B4
:10CE500055F82020D4074FEA800729D402F00604B1
:10CE6000022C22F01F0308D1E1E19A4517D01A687D
:10CE7000D20708D41B6823F01F03B3F84020914267
:10CE8000F3D99A450BD01A6832F01F0205D1C9E1D7
:10CE9000126832F01F0200F0C5819245F8D10844B3
:10CEA0001F28A9D855F82020D4074FEA8007D5D5E8
:10CEB00008441F28CAF80020EE51F3D99CE70199D5
:10CEC0001298097D42F6AB23C0F2010303FB00F385
:10CED00002294FEA134300F00881AAF84020002DF0
:10CEE00040F0C48184334FEA5318022700224FF0E8
:10CEF000FF3342F2000C99469646C2F2010CCDF87F
:10CF000010A0934651E0824580F08980A04238BF4E
:10CF10002046984228BF18460CEB050338BFF1465F
:10CF200093F8491293F84D32414438BF4FF0000B4B
:10CF30008A453B446DD3544566D29A45514638BF25
:10CF40001946884298BF01460CEB0500424490F810
:10CF50004E0284BFF1464FF0010B944238444DD34A
:10CF60009C4246D98442224638BF024665449142DB
:10CF700098BF0A46464495F84F1284BFF1464FF0D9
:10CF8000020BB342394430D3834229D98B4238BF94
:10CF90000B469A4288BFF1460EF1010E94BF13462C
:10CFA0004FF0030BBEF1200F3ED04FEACE050CEB45
:10CFB000050494F8480294F84A2294F84B6294F8D5
:10CFC0004C4200EB0801D01981423C4406EB070AB1
:10CFD00099D9514523D9A14238BF2146084698E73F
:10CFE0008842034638BF0B46D3E7B042F8D23346F7
:10CFF000CCE783421A4638BF0246B7E79342F8D2DD
:10D00000824238BF0246B1E79C42214638BF1946EA
:10D0100097E78C42F8D2994238BF194691E75445B8
:10D02000204638BF504674E7BB2BDDF810A05E46A3
:10D030004CD85FFA88F8FFB201231FFA89F4B9F1DE
:10D040001F0F8AF84A808AF84B70AAF848B0AAF8ED
:10D050004430AAF8464098BF584622D800EBC9038E
:10D060000CEB0305991C95F848226144424485F86D
:10D07000482291F84852DA1C62443D4481F84852F3
:10D0800092F8481204336344394482F8481293F802
:10D09000482209F101093A44B9F1200F83F84822E6
:10D0A000DCD101231C20B340B040DBB2C0B2AAF8EF
:10D0B00042408AF836308AF83700039A002A7FF413
:10D0C0005EAE019917460D7D114673E6079A0698E4
:10D0D0001368059C0360236810600020CAF80030C4
:10D0E000C4F800A009B0BDE8F08F42F24720C2F2B8
:10D0F00001005733AAF840205B0900F58074002135
:10D1000010F8012F1A44914238BF11468442F7D1DA
:10D11000BB29DBD842F2000CC2F2010C0CF51274F0
:10D12000614201F00301B1F5807FDBB24FF00100F5
:10D130004FF0000228BF4FF480718AF84A30AAF8F5
:10D140004400AAF84620002900F095809CF8482267
:10D1500081421A448CF8482200F08D809CF84922C4
:10D1600002291A448CF8492200F085809CF84A2252
:10D170001A448CF84A220322002663F3070663F35D
:10D180000F26C1F1FC0563F31746AD080C4463F3A9
:10D190001F66013506F07F39C1F5807B4FEA850EA9
:10D1A000A4F10408002758F8041F01F07F307140F3
:10D1B000484401F0803101374140AF4244F8041B3C
:10D1C000F1D3DE4572441DD0944442F200009CF835
:10D1D000481219448CF84812511CB1F5807FC2F2F4
:10D1E00001000FD00144023291F84842B2F5807F2D
:10D1F0001C4481F8484205D0024492F848120B447E
:10D2000082F848320020FF238AF83630AAF842001C
:10D210008AF8370051E7059BCAF800402846C3F852
:10D2200000A0EAE51A68CAF800201E6037E6B3F8E5
:10D230004040A1427FF619AE3AE6DAF804104FF406
:10D240008A534AF00200C4F20A0341F40041CAF8CA
:10D250000410CAF80000C2F800A01A6842F02002C8
:10D2600050461A60C9E5C3F804A092E566335F0929
:10D270004FF002083AE60A467EE700BFF8B50446DA
:10D28000002301250570457005718370C37080F817
:10D29000C130C0F8A830C0F8AC30C0F8B030C0F829
:10D2A000B430C0F8B8300E46C4F8BC30194684F823
:10D2B000C030A02208300CF05FFB02220923A571C8
:10D2C0006271C4F8A86084F8BC302046F8BD00BF85
:10D2D000F8B504460023012505704570057183707B
:10D2E000C37080F8C130C0F8A830C0F8AC30C0F8C6
:10D2F000B030C0F8B430C0F8B8300E46C4F8BC3016
:10D30000194684F8C030A02208300CF035FB022208
:10D310000823A5716271C4F8A86084F8BC30204667
:10D32000F8BD00BFF8B5044600230125057045701F
:10D3300005718370C37080F8C130C0F8A830C0F8A0
:10D34000AC30C0F8B030C0F8B430C0F8B8300E46D9
:10D35000C4F8BC30194684F8C030A02208300CF064
:10D360000BFB0222FB23A5716271C4F8A86084F84C
:10D37000BC302046F8BD00BF4368427A5B7A9A42CF
:10D380001FD830B472B60468E3682BB3DA6832B1E0
:10D3900019688C4216D01346DA68002AF8D1D86092
:10D3A0000023C360A37A0133A3720268416801239A
:10D3B00013728A7A1A448A7242681372037462B6CC
:10D3C00030BC70475D6841688D42E4D1198903899A
:10D3D0009942F4D01346DFE7E060E1E7F8B500F1E9
:10D3E000180204460121FCF787F8204640F2880322
:10D3F000C0F20F0340F81C3B40F6B80200210CF0CD
:10D40000BBFA04F6D40040F6481200210CF0B4FA3E
:10D4100004F5905040F6FA1200211C300CF0ACFAE2
:10D4200004F5E05040F69822002116300CF0A4FAE2
:10D4300004F51A5040F61C3200212E300CF09CFAF4
:10D4400004F5475040F6A63200210A300CF094FA59
:10D4500004F5755040F62A42002130300CF08CFA69
:10D4600004F5934040F6A24200211A300CF084FAF1
:10D4700045F23E6745F23C63002545F2406645F2C1
:10D48000426245F24460E55245F24661E55345F299
:10D49000486345F24A67A553A55245F24C662552AA
:10D4A00045F24E6245F250606552E55245F25261D6
:10D4B000E55345F2546345F25667A553A55245F22C
:10D4C0005866255245F25A6245F25C606552E55253
:10D4D00045F25E61E55345F2606341F69917A55345
:10D4E000A55246F26766275246F6843204F5AC40F0
:10D4F00066526230E25229464FF48B620CF03CFADD
:10D5000004F5B540294640F272323A300CF034FA54
:10D5100004F5BC40294640F2AA222C300CF02CFA2B
:10D5200004F5C14029464FF4E17256300CF024FA5C
:10D5300046F2982046F29A2146F29C2246F29E2319
:10D54000255265522046A552E552F8BD38B505462C
:10D5500040F28C000C46C0F20F000D210AF0CAF810
:10D5600049F2A823C1F6FF7393F823305BB304F5A7
:10D570000051C1F3C6122B4601F07F01E020FFF7F6
:10D58000BBF804F30D0440F29C0004F50054C0F213
:10D590000F00013D0AF090FD2D02200400F4FE0072
:10D5A00005F47065054345F46040640440F00E00E6
:10D5B00004F0FE4420430AF033FD40F2AC00C0F218
:10D5C0000F000AF079FDBDE83840FEF77BBC00BFD4
:10D5D00038B5054640F2C4000C46C0F20F000D21DC
:10D5E0000AF088F849F2A823C1F6FF7393F82330B4
:10D5F000FBB121462B460022D020FFF77DF840F2F8
:10D600009C00C0F20F0024040AF056FD04F4FE044E
:10D61000681E44F45044000244F00D0400F47060AD
:10D6200020430AF0FDFC40F2AC00C0F20F000AF00B
:10D6300043FDBDE83840FEF745BC00BF70B549F278
:10D64000A825C1F6FF750C4695F82230064623B191
:10D65000984202D00BF062F9C0B149F2A423C1F69E
:10D66000FF731C70FBF774FF43F61053C2F2000304
:10D670004DF6203293F8AD1053F82130597B03EB6F
:10D680008103C1F6FF725B6893422DD040F2D40053
:10D69000C0F20F000D210AF02DF895F82330FBB1F0
:10D6A000214633460022C020FFF726F840F29C00B6
:10D6B000C0F20F0024040AF0FFFC04F4FE04701E04
:10D6C00044F44044000244F00C0400F47060204331
:10D6D0000AF0A6FC40F2AC00C0F20F000AF0ECFC2D
:10D6E000BDE87040FEF7EEBBFEF7B6FBCEE700BF2D
:10D6F000F8B549F2A826C1F6FF760C4696F8223016
:10D7000015460746B3B3984234D00BF007F988BBEF
:10D7100040F2E400C0F20F000D2109F0EBFF96F893
:10D7200023301BB32A4621463B46B020FEF7E4FFD8
:10D730002D0640F29C00C0F20F0005F0FE450AF0F5
:10D74000BBFC45F430452404781E45F00B0504F479
:10D75000FE0400022C4300F4706020430AF060FCD9
:10D7600040F2AC00C0F20F000AF0A6FCBDE8F840A1
:10D77000FEF7A8BB5C2CCBD00CD80A2C29D05B2C94
:10D7800047D105EB850000EB8000C0F347100AF09D
:10D79000F1FEBDE75D2C33D05E2C3AD107EE905AF6
:10D7A0000023C4F2FE2306EE903AB8EE676A002327
:10D7B000C6EE267A07EE103A4BF22003C1F6FF734D
:10D7C00077EE877A18684368C3ED0A7A02F02EF87C
:10D7D0009EE707EE905A0023C4F2FE2306EE903A2D
:10D7E000B8EE676A0023C6EE267A07EE103A77EEA7
:10D7F000877AFDEEE77A17EE903A86F8253087E7CC
:10D8000005EB850000EB8000C0F347100AF07AFDBD
:10D810007EE74BF22003C1F6FF732A4618680368BF
:10D8200021465B68984773E72DE9F04F49F2A82637
:10D83000C1F6FF7687B096F82230029104920390E9
:10D84000D3B3984238D00BF069F8A8BB40F2F4008B
:10D85000C0F20F00122109F04DFF96F8233033B3C8
:10D86000039E049D029C33462A4621468020FEF7F3
:10D8700043FF40F29C00C0F20F000AF01DFC2B0693
:10D8800003F0FE4343F400432204701E02F4FE0240
:10D8900043F008030002134300F4706018430AF0D9
:10D8A000BFFB40F2AC00C0F20F000AF005FC07B06D
:10D8B000BDE8F04FFEF706BB4BF22003C1F6FF7345
:10D8C00096F909A0D3F800B0029B9BF81020DBF872
:10D8D00004809A44002AB9D005965C46002580272A
:10D8E000464604E00135AA4204F134040FDDD4F8C1
:10D8F000EC329A45F6D1DBF8EC3A53B1C4F8EC724D
:10D900009BF810200135AA4204F13404EFDC059E97
:10D910009CE7DBF80C0080F000400BF01DFDCDE92A
:10D92000000150460BF006FD47F6E1234FF0804220
:10D93000C3F684730BF0B4FD00230022C4F2180375
:10D940000BF0ACFB736807EE103AF1EE047A67EE69
:10D95000277A804617EE900A89460BF0FDFC0246B6
:10D960000B46404649460BF097FB41EC100B10F07C
:10D970005BFBDDE9000153EC102B0BF091FD41EC5A
:10D98000100B10F051FB51EC100B0BF039FDC4F8EB
:10D99000D4029BF81020A5E7F8B549F2A825C1F6F6
:10D9A000FF750E4695F822301446074623B198427B
:10D9B00002D00AF0B3FF18B12146304602F0DAF97E
:10D9C00040F20810C0F20F00112109F093FE95F803
:10D9D00023301BB3224631463B469020FEF78CFE97
:10D9E000240640F29C00C0F20F0004F0FE440AF04E
:10D9F00063FB44F410443604781E44F0090406F432
:10DA0000FE060002344300F4706020430AF008FB75
:10DA100040F2AC00C0F20F000AF04EFBBDE8F84047
:10DA2000FEF750BA40F21C1008B5C0F20F001B21DF
:10DA300009F060FE49F2A823C1F6FF7393F8233082
:10DA4000B3B143F60860FF21C2F2000002F008F90A
:10DA500040F29C00C0F20F000AF02EFB4FF60F7050
:10DA600009F030FF40F23810C0F20F000AF024FB3A
:10DA7000BDE80840FEF726BA40F2481008B5C0F2EB
:10DA80000F001D2109F036FE49F2A823C1F6FF73ED
:10DA900093F82330B3B143F60860FE21C2F20000D0
:10DAA00002F0DEF840F29C00C0F20F000AF004FB26
:10DAB0004FF60F6009F006FF40F23810C0F20F0079
:10DAC0000AF0FAFABDE80840FEF7FCB940F2681027
:10DAD00008B5C0F20F00142109F00CFE49F2A8238A
:10DAE000C1F6FF7393F82330B3B143F60860FC210D
:10DAF000C2F2000002F0B4F840F29C00C0F20F0045
:10DB00000AF0DAFA4FF60F4009F0DCFE40F2381066
:10DB1000C0F20F000AF0D0FABDE80840FEF7D2B913
:10DB200040F2801008B5C0F20F00182109F0E2FDA4
:10DB300049F2A823C1F6FF7393F82330B3B143F63B
:10DB40000860FB21C2F2000002F08AF840F29C005B
:10DB5000C0F20F000AF0B0FA4FF60F3009F0B2FE33
:10DB600040F23810C0F20F000AF0A6FABDE80840F3
:10DB7000FEF7A8B940F29C1008B5C0F20F001521BD
:10DB800009F0B8FD49F2A823C1F6FF7393F82330DA
:10DB9000B3B143F60860FA21C2F2000002F060F867
:10DBA00040F29C00C0F20F000AF086FA4FF60F20F8
:10DBB00009F088FE40F23810C0F20F000AF07CFA3B
:10DBC000BDE80840FEF77EB940F2B41008B5C0F2D7
:10DBD0000F00152109F08EFD49F2A823C1F6FF734D
:10DBE00093F82330B3B143F60860F821C2F2000085
:10DBF00002F036F840F29C00C0F20F000AF05CFA26
:10DC00004FF60F0009F05EFE40F23810C0F20F0030
:10DC10000AF052FABDE80840FEF754B940F2CC10C1
:10DC200008B5C0F20F001B2109F064FD49F2A823DA
:10DC3000C1F6FF7393F82330C3B143F6C053C2F269
:10DC40000003F621986C0368DB6C984740F29C0057
:10DC5000C0F20F000AF030FA4FF20F6009F032FE06
:10DC600040F23810C0F20F000AF026FABDE8084072
:10DC7000FEF728B938B5044640F2E810C0F20F00AC
:10DC80001A2109F037FD49F2A823C1F6FF7393F872
:10DC900023301BB9BDE83840FEF714B943F6C05530
:10DCA000C2F2000548F67523A86C02681268C0F23B
:10DCB00000039A4221D1F32008F024FAA86C0368EB
:10DCC00004F07F01DB6C984740F29C00C0F20F002B
:10DCD0000AF0F2F9200400F4FE0040F4734040F032
:10DCE000020009F0EFFD40F23810C0F20F000AF018
:10DCF000E3F9BDE83840FEF7E5B8F3219047DDE7EA
:10DD000070B5044640F20420C0F20F00242109F04F
:10DD1000F1FC49F2A823C1F6FF7393F823301BB935
:10DD2000BDE87040FEF7CEB843F6C056C2F200061A
:10DD300048F67525B06C03681B68C0F20005AB425D
:10DD400024D1F12008F0DEF9B06C03681B68AB4207
:10DD50001FD1204608F0D6F940F29C00C0F20F0017
:10DD60000AF0AAF904F00F044FF202102404C0F2E2
:10DD70001000204309F0A6FD40F23810C0F20F0059
:10DD80000AF09AF9BDE87040FEF79CB8F121984777
:10DD9000DAE721469847DFE770B5064640F22C20C7
:10DDA0000C46C0F20F001721154609F0A3FC49F2FA
:10DDB000A823C1F6FF7393F823301BB9BDE8704068
:10DDC000FEF780B8A02033462A462146FEF794FC91
:10DDD00040F24420C0F20F000AF06EF94EB140F25A
:10DDE0003810C0F20F000AF067F9BDE87040FEF786
:10DDF00069B8681E0002240404F4FE0400F4706094
:10DE0000204340F4504040F00D0009F05BFDE6E790
:10DE100038B5054640F250200C46C0F20F001221E2
:10DE200009F068FC49F2A823C1F6FF7393F8233088
:10DE30005BB304F50051C1F3C6122B4601F07F011C
:10DE4000E020FEF759FC04F30D0440F29C0004F5B9
:10DE50000054C0F20F00013D0AF02EF92D022004FB
:10DE600000F4FE0005F47065054345F46040640469
:10DE700040F00E0004F0FE44204309F023FD40F280
:10DE80003810C0F20F000AF017F9BDE83840FEF76D
:10DE900019B800BF38B5054640F264200C46C0F200
:10DEA0000F00122109F026FC49F2A823C1F6FF73E6
:10DEB00093F82330FBB121462B460022D020FEF7F9
:10DEC0001BFC40F29C00C0F20F0024040AF0F4F89E
:10DED00004F4FE04681E44F45044000244F00D04AF
:10DEE00000F47060204309F0EDFC40F23810C0F2FD
:10DEF0000F000AF0E1F8BDE83840FDF7E3BF00BFCE
:10DF00002DE9F04F87B0059040F278200491C0F2DF
:10DF10000F00152109F0EEFB49F2A823C1F6FF73AB
:10DF200093F8233023B907B0BDE8F04FFDF7CABF1F
:10DF300043F6C05BC2F2000BF021DBF84800036837
:10DF4000DB6C9847049B002B00F0B8801A4648F21F
:10DF50003403C4F20403DBF848000093059B056812
:10DF600048F6752A4FF420461F461344C0F2000AB3
:10DF7000C4F2060699462B6817F8011B534540F07A
:10DF80009580009B1B685C0560D543F21473C2F258
:10DF900001031B680BB10120187043F2CC63C2F27D
:10DFA000010343F2CD651C7801343F2C88BF00206B
:10DFB00043F2D06894BFE0B20446C2F20105C2F257
:10DFC00001082A78A24233D1EFF31382002A57D1F5
:10DFD000EFF31082002A53D1EFF3058EBEF1000F4C
:10DFE00061D0BEF10F0F05D94EF2F032CEF2000231
:10DFF00072441278EFF3118EBEF1000F02D0724519
:10E0000028BF7246402A3BD9B2F5807FD9D143F26E
:10E010004172C2F201021278002AD2D10393029116
:10E02000019009F067FA2A7801A8A2420BC8CBD068
:10E0300043F21075C2F2010508F804100124BC2156
:10E040002C701870F170DBF848000568B94592D162
:10E05000EB6CF721984740F29C00C0F20F000AF0E9
:10E060002BF804990598FDF7C5FF40F23810C0F26F
:10E070000F000AF021F807B0BDE8F04FFDF722BF0E
:10E08000327912069DD52A7801323F2A86BF4FF099
:10E09000000E72465FFA82FE18F80220D2B2F271C8
:10E0A00085F800E08DE74FF48072A3E79847DBF82E
:10E0B0004800B94505687FF45EAFC9E7DBF8480062
:10E0C0000568C5E770B549F2A825C1F6FF750C468D
:10E0D00095F82230064623B1984202D00AF01EFC81
:10E0E000C0B149F2A423C1F6FF731C70FBF730FAEC
:10E0F00043F61053C2F200034DF6203293F8AD10F0
:10E1000053F82130597B03EB8103C1F6FF725B6842
:10E1100093422DD040F29020C0F20F00122109F05E
:10E12000E9FA95F82330FBB1214633460022C0209E
:10E13000FEF7E2FA40F29C00C0F20F00240409F05E
:10E14000BBFF04F4FE04701E44F44044000244F09B
:10E150000C0400F47060204309F0B4FB40F2381066
:10E16000C0F20F0009F0A8FFBDE87040FDF7AABE9D
:10E17000FDF772FECEE700BFF8B549F2A826C1F65A
:10E18000FF760C4696F8223015460746B3B3984200
:10E1900034D00AF0C3FB88BB40F2A420C0F20F00C9
:10E1A000122109F0A7FA96F823301BB32A4621461C
:10E1B0003B46B020FEF7A0FA2D0640F29C00C0F2CC
:10E1C0000F0005F0FE4509F077FF45F430452404C3
:10E1D000781E45F00B0504F4FE0400022C4300F405
:10E1E0007060204309F06EFB40F23810C0F20F005F
:10E1F00009F062FFBDE8F840FDF764BE5C2CCBD0AF
:10E200000CD80A2C29D05B2C47D105EB850000EBFC
:10E210008000C0F347100AF0ADF9BDE75D2C33D0A4
:10E220005E2C3AD107EE905A0023C4F2FE2306EE8C
:10E23000903AB8EE676A0023C6EE267A07EE103AE7
:10E240004BF22003C1F6FF7377EE877A18684368B4
:10E25000C3ED0A7A01F0EAFA9EE707EE905A00232E
:10E26000C4F2FE2306EE903AB8EE676A0023C6EECB
:10E27000267A07EE103A77EE877AFDEEE77A17EE08
:10E28000903A86F8253087E705EB850000EB8000A3
:10E29000C0F347100AF036F87EE74BF22003C1F6D0
:10E2A000FF732A461868036821465B68984773E73E
:10E2B0002DE9F04F49F2A826C1F6FF7687B096F80F
:10E2C0002230029104920390D3B3984238D00AF0DE
:10E2D00025FBA8BB40F2B820C0F20F00172109F0BF
:10E2E00009FA96F8233033B3039E049D029C33460B
:10E2F0002A4621468020FEF7FFF940F29C00C0F23A
:10E300000F0009F0D9FE2B0603F0FE4343F400434F
:10E310002204701E02F4FE0243F0080300021343BD
:10E3200000F47060184309F0CDFA40F23810C0F2E2
:10E330000F0009F0C1FE07B0BDE8F04FFDF7C2BD08
:10E340004BF22003C1F6FF7396F909A0D3F800B091
:10E35000029B9BF81020DBF804809A44002AB9D075
:10E3600005965C4600258027464604E00135AA4212
:10E3700004F134040FDDD4F8EC329A45F6D1DBF821
:10E38000EC3A53B1C4F8EC729BF810200135AA4264
:10E3900004F13404EFDC059E9CE7DBF80C0080F010
:10E3A00000400AF0D9FFCDE9000150460AF0C2FF53
:10E3B00047F6E1234FF08042C3F684730BF070F808
:10E3C00000230022C4F218030AF068FE736807EE07
:10E3D000103AF1EE047A67EE277A804617EE900A3B
:10E3E00089460AF0B9FF02460B46404649460AF004
:10E3F00053FE41EC100B0FF017FEDDE9000153EC6A
:10E40000102B0BF04DF841EC100B0FF00DFE51EC02
:10E41000100B0AF0F5FFC4F8D4029BF81020A5E712
:10E42000F8B549F2A825C1F6FF750E4695F82230D9
:10E430001446074623B1984202D00AF06FFA18B189
:10E440002146304601F096FC40F2D020C0F20F0089
:10E45000162109F04FF995F823301BB322463146B7
:10E460003B469020FEF748F9240640F29C00C0F29B
:10E470000F0004F0FE4409F01FFE44F4104436047B
:10E48000781E44F0090406F4FE060002344300F44A
:10E490007060204309F016FA40F23810C0F20F0005
:10E4A00009F00AFEBDE8F840FDF70CBD70B5064660
:10E4B00049F2A82540F2E8202DED028B0E21C0F292
:10E4C0000F00C1F6FF7509F015F900220A21304648
:10E4D00009F0FCFDFDF7F6FC95F91F3007EE106A18
:10E4E00007EE903A0023C4F2482306EE103AF8EE05
:10E4F000E77AB8EE477A002377EE867A37EE067A27
:10E50000C4F2C82306EE903A77EEA77A37EE077A80
:10E51000C7EEA68A40F6E473C2F201035B7AC7EE47
:10E52000267AB7EE008A78EEC88A37EEC88A002BC2
:10E5300062D10023C4F2402307EE103A47F6EE43BF
:10E54000C3F6FF6307EE903A0023E8EE877ACCF239
:10E550003C2306EE903AF4EEE67AF1EE10FA47D458
:10E56000F4EEC77AF1EE10FAC8BF5F245FDD4FF416
:10E570008B70FDF75BFE20F07F0240F6E4702243D3
:10E58000C2F201004FF48B7102F09EFD0023C4F231
:10E59000402307EE103A47F6EE43C3F6FF6307EE5B
:10E5A000903A0023E8EE077ACCF23C2306EE903A4C
:10E5B000F4EEE67AF1EE10FA1CD4F4EEC77AF1EE3E
:10E5C00010FAC8BF5F2426DD4FF48F70FDF72EFED2
:10E5D00020F07F0240F6E4702243C2F201004FF4C3
:10E5E0008F7102F071FDBDEC028B85F8206070BD6B
:10E5F0000024BCE70024E7E74FF48470FDF716FE23
:10E6000000F00300022894D0032202214FF484700A
:10E61000FDF71AFF8DE70023C4F23C2307EE103A02
:10E6200077EE877AFCEEE77A17EE904ACCE7002384
:10E63000C4F23C2307EE103A77EE877AFCEEE77AD5
:10E6400017EE904A93E700BF70B5064649F2A82539
:10E6500040F2F8202DED028B0C21C0F20F00C1F624
:10E66000FF7509F047F800220A21304609F02EFD17
:10E67000FDF728FC95F9203007EE106A07EE903A76
:10E680000023C4F2482306EE103AF8EEE77AB8EE1B
:10E69000477A002377EE867A37EE067AC4F2C823EB
:10E6A00006EE903A77EEA77A37EE077A87EEA68ADB
:10E6B00040F6E473C2F201035B7AC7EE267AF7EE06
:10E6C000008A38EE688A77EEE88A002B61D1002351
:10E6D000C4F2402307EE103A47F6EE43C3F6FF6359
:10E6E00007EE903A0023E8EE877ACCF23C2306EE60
:10E6F000903AF4EEE67AF1EE10FA46D4F4EEC77AE8
:10E70000F1EE10FAC8BF5F245EDD4FF48B70FDF7A9
:10E710008DFD20F07F0240F6E4702243C2F201003A
:10E720004FF48B7102F0D0FC0023C4F2402307EEBB
:10E73000103A47F6EE43C3F6FF6307EE903A002324
:10E74000E8EE077ACCF23C2306EE903AF4EEE67A55
:10E75000F1EE10FA1BD4F4EEC77AF1EE10FAC8BF4E
:10E760005F2425DD4FF48F70FDF760FD20F07F0200
:10E7700040F6E4702243C2F201004FF48F7102F0C0
:10E78000A3FCBDEC028BEE7770BD0024BDE7002436
:10E79000E8E74FF48470FDF749FD00F0030002281C
:10E7A00095D0032202214FF48470FDF74DFE8EE7D1
:10E7B0000023C4F23C2307EE103A77EE877AFCEE92
:10E7C000E77A17EE904ACDE70023C4F23C2307EE28
:10E7D000103A77EE877AFCEEE77A17EE904A94E7E4
:10E7E000F0B5074649F2A82640F2083083B0C1F6DA
:10E7F000FF761421C0F20F0008F07CFF00220A21EE
:10E80000384609F063FCFDF75DFB737F06EE107A76
:10E8100007EE903A0023C4F2C62305EE903AF8EED4
:10E82000464AF8EE677A002387EEA56A4FF48370B4
:10E83000C4EEA57A07EE103A0023C4F27C2305EE5D
:10E84000103A47F6EE43C3F6FF6336EE076A37EE3B
:10E85000877A07EE903AE6EE057AFCEEE77ACDEDA0
:10E86000017A9DF804303F2B9CBFC3F13F031D028A
:10E870004FF00003C4F2FE2306EE903A47F6EE4353
:10E88000C3F6FF6307EE903AE7EE267A88BF0025CD
:10E89000FCEEE77ACDED017A9DF804307F2B94BF32
:10E8A000C3F17F040024FDF7C1FC20F47D5245EA4A
:10E8B000040322F03F0240F6E4701A434FF48371E0
:10E8C000C2F2010002F000FCB77703B0F0BD00BF58
:10E8D000F0B5074640F2203083B01221C0F20F009D
:10E8E00008F008FF00220A21384609F0EFFBFDF787
:10E8F000E9FA0023C4F2C62305EE103A002307EE1E
:10E90000103A07EE907A0023C4F27C2349F2A8263D
:10E9100004EE903AC1F6FF76F8EE677A47F6EE43DA
:10E92000C3F6FF6387EE856A4FF4837006EE903A74
:10E93000B37F05EE903AF8EE655A36EE076AC5EEFB
:10E94000857AE6EE246A37EE877AFCEEE67ACDED3C
:10E95000017A9DF804303F2B9CBFC3F13F031D0299
:10E960004FF00003C4F2FE2306EE903A47F6EE4362
:10E97000C3F6FF6307EE903AE7EE267A88BF0025DC
:10E98000FCEEE77ACDED017A9DF804307F2B94BF41
:10E99000C3F17F040024FDF749FC20F47D5245EAD1
:10E9A000040322F03F0240F6E4701A434FF48371EF
:10E9B000C2F2010002F088FB777703B0F0BD00BF20
:10E9C0002DE9F04149F2A8242DED048BC1F6FF7426
:10E9D00000232779C4F2C62340F2043008EE903AAF
:10E9E000C0F20200002308EE103A09F065FB384639
:10E9F000FDF7CAFB07EE907AB8EE677A4BF2200576
:10EA0000C7EE287AC1F6FF7528684368B2EE049A0B
:10EA100077EE887AC3ED007A00F008FF66792771F7
:10EA200040F21030C0F2020009F046FB3046FDF71C
:10EA3000ABFB07EE906AB8EE677A2868C7EE287AD3
:10EA4000436877EE887AC3ED017A00F0EFFEA7798C
:10EA5000667140F22030C0F2020009F02DFB38460A
:10EA6000FDF792FB07EE907AB8EE677A2868C7EE5A
:10EA7000287A436877EE887AC3ED027A00F0D6FEF2
:10EA8000E679A77140F23030C0F2020009F014FBC1
:10EA90003046FDF779FB07EE906AB8EE677A286892
:10EAA000C7EE287A436837EE888A83ED038A00F040
:10EAB000BDFE94F90870E67140F23C30C0F20200ED
:10EAC00009F0FAFA002FB5BF2D220022784238460D
:10EAD0000A2109F0FBFAFDF7F5F907EE907A002319
:10EAE000C4F2C623B8EEE76A06EE903AC6EE267A7E
:10EAF0000023286807EE103A436877EE877AC3ED63
:10EB0000077A00F093FE94F90A60277240F25830B9
:10EB1000C0F2020009F0D0FA002EB4BF2D2200226C
:10EB20004FF00A013046B8BF704209F0CFFAFDF746
:10EB3000C9F907EE906A0023C4F24823F8EEE77A99
:10EB400007EE103A0023C4F2C82306EE903A37EEDF
:10EB5000877A0023C7EE267A286808EE103A002349
:10EB6000C4F2C62308EE903A77EE887A4368C3ED84
:10EB7000097A00F05BFE94F80B80A67240F26430D4
:10EB8000C0F2020009F098FA4046FDF7FDFA07EEE0
:10EB9000908AB8EE677A2868C7EE287A436877EEDD
:10EBA000887AC3ED0A7A00F041FE277B84F80B8057
:10EBB00040F27030C0F2020009F07EFA3846FDF7EC
:10EBC000E3FA07EE907AB8EE677A2868C7EE287AFB
:10EBD000436877EE887AC3ED067A00F027FE667BFD
:10EBE000277340F28430C0F2020009F065FA304623
:10EBF000FDF7CAFA07EE906AB8EE677A2868C7EEA2
:10EC0000287A436877EE887AC3ED057A00F00EFE25
:10EC1000A77B667340F29C30C0F2020009F04CFA08
:10EC20003846FDF7B1FA07EE907AB8EE677A2868B1
:10EC3000C7EE287A436877EE887AC3ED047A00F04D
:10EC4000F5FDE67BA77340F2B030C0F2020009F098
:10EC500033FA3046FDF798FA07EE906AB8EE677A15
:10EC60002868C7EE287A436877EE887AC3ED0B7A76
:10EC700000F0DCFD207CE67309F00EFE607C09F0FC
:10EC8000C7FDA07C09F080FDE77C40F2C030C0F2F7
:10EC9000020009F011FA3846FDF776FA637DA27C8E
:10ECA000617C207C01EE103A237D00EE903A07EE65
:10ECB000907AB8EE411AF8EE600AB8EE670A81EE73
:10ECC000091AC0EE890AFDF7D7FB267DE77440F2EA
:10ECD000D430C0F2020009F0EFF93046FDF754FAE3
:10ECE000637DA27C617C207C07EE906A01EE103A85
:10ECF000E37CF8EE670A00EE103AB8EE411AC0EE77
:10ED0000890A81EE091AB8EE400AFDF7B5FB677D66
:10ED1000267540F2E830C0F2020009F0CDF938461D
:10ED2000FDF732FA237DA27C617C207C07EE907A8D
:10ED300000EE903AE37CB8EE671A00EE103AF8EE77
:10ED4000600A81EE091AC0EE890AB8EE400AFDF7A2
:10ED500093FBA67D677540F2F830C0F2020009F01F
:10ED6000ABF93046FDF710FA07EE906AF8EE676AE5
:10ED7000B7EE007AC6EEA87A77EE887AF4EEC77A14
:10ED8000F1EE10FA40F3308144F23872C2F2000220
:10ED900045F2606147F6705353524AF6D812C2F2F8
:10EDA000000245F26061E07D5352A67509F060FCF7
:10EDB000207E09F0DFFB677E40F21040C0F20200C7
:10EDC00009F07AF93846FDF7DFF907EE907AF8EEA8
:10EDD000676AB2EE047AC6EE877AF5EEC07AF1EE93
:10EDE00010FA00F1FA8045F2A653C4F2AC6307EEC4
:10EDF000103AF4EEC77AF1EE10FA00F3E78042F22F
:10EE00004B43C4F2BE7307EE103A67EE877A0022D6
:10EE1000FCEEE77A40F6B05617EE903AC7F6FE726F
:10EE2000C2F201069342C6ED077A03D90023C7F662
:10EE3000FE73F361A07E677609F030FBE77E40F257
:10EE40002840C0F2020009F037F93846FDF79CF976
:10EE500007EE907A0023C4F2C82306EE903AB8EE8B
:10EE6000676A0023C6EE267A07EE103A77EE877AB5
:10EE7000F4EEC77AF1EE10FA00F1EF80B7EE007A07
:10EE8000F4EEC77AF1EE10FA40F3E9804FF48033E4
:10EE90007362207FE77609F035FA607FFFF718FD8F
:10EEA000A07FFFF79DFCE07FFFF7CEFB94F82000EA
:10EEB000FFF7FCFA94F8216040F24040C0F20200F3
:10EEC00009F0FAF83046FDF75FF907EE906A002383
:10EED000C4F2C623F8EE675A06EE103A85EE867A3B
:10EEE000002394F8227084F8216040F25040C0F270
:10EEF000020007EE903A45F2EC13C3F6386306EED3
:10EF0000903A77EE277A2B6867EEA67A03F63C33C1
:10EF1000C3ED007A09F0D0F83846FDF735F994F8DA
:10EF2000236084F8227040F26440C0F2020009F0CD
:10EF3000C3F83046FDF728F994F8247084F823606C
:10EF400040F27840C0F2020009F0B6F83846FDF70A
:10EF50001BF9282F28683ED8002F14BF3B460123F9
:10EF600047F2A40503740026C3F67D75034684F8B2
:10EF7000247000F50261C3F8D062C3F8D452343370
:10EF80008B424FF00002F6D1BDEC048B00F6283125
:10EF90000024C4F220340C60002300F6F82700F5AA
:10EFA0002F6600F5316500F60C3400F6F421C0F848
:10EFB000DC3AC0F8EC3A4FF07E533A6032602A6097
:10EFC00022600B60BDE8F04100F030BC40F6B05666
:10EFD000C2F201062AE72823C2E740F6B056C2F281
:10EFE00001060023F36125E7F4EEC87AF1EE10FA8A
:10EFF0003FD445F62943C4F20F6307EE103A27EEDB
:10F00000877ABDEEC77A17EE103A03F5B34319338A
:10F010001BB244F23872B7EE007AC2F2000245F237
:10F020006061F4EEC77AF1EE10FA535224DCF5EE8B
:10F03000C07AF1EE10FA19D445F62943C4F20F63F1
:10F0400007EE103A67EE877AFDEEE77A17EE903A10
:10F0500003F5B34319331BB29FE6002318E7B0EE64
:10F06000677ABEEEC87A17EE103A11E745F69913A3
:10F0700093E645F69913CCE747F670538DE600BF4B
:10F080002DE9F04F2DED048B844685B00CF6F82366
:10F0900000F6083400F6243500F60C3900F5316826
:10F0A00093ED001A94ED000AD5ED004A99ED003A6F
:10F0B000D8ED003ADCF8DCEA9FED9E5ADFED9E9A2F
:10F0C0000CF6F42300F604301C460CF52F6BD0ED43
:10F0D000000A02930CF6FC200CF5306393ED008AD5
:10F0E000DBED002A94ED004AD0ED008A02F1FE0328
:10F0F0000239A2F1020A0193F6EE001AB7EE002AD5
:10F10000BFEE009ABEF1000F9FED8C6A40F30481C0
:10F11000DCF8E06AF0EE465A0CF53C70002550F839
:10F12000307C50F8343C50F82C2C50F8284C3B44A0
:10F1300002EB234201359BB2A2422DB240F82C2CA7
:10F1400040F8303C04DD50F8244C121B40F82C2CC5
:10F1500006EB420436F91220B4F9027010ED087A79
:10F1600050ED076ABF1A03FB07F302EB234307EED8
:10F17000903AF8EEE77A67EE266A67EE877A40ED16
:10F18000086A67EE857AF5EEC07AF1EE10FA0EDDC8
:10F1900024EEA77AE7EEC77AB0EE677AF1EE667AE8
:10F1A000B4EEE77AF1EE10FA58BFF0EE477A50ED80
:10F1B000036A10ED027A7545E7EEA65A00F13400B5
:10F1C000A7EE876AABDB36EE637A75EEC37AE7EEBD
:10F1D000003A029BA7EE803AE1EE042A36EE637A0B
:10F1E000A2EEC14AA7EE206A75EEC37A26EE087A2F
:10F1F000E7EEA05AA4EE076A65EEA87A26EE216A29
:10F20000E4EE275AB4EEC26AF1EE10FA89ED003A44
:10F2100065EEA15AC8ED003ACBED002A83ED004A15
:10F220006CDD47F6FF73F4EEC25AF1EE10FA57DDCB
:10F2300047F6FF722AF8022F21F8023F019B9A45F8
:10F240007FF460AFDFED3E7AB0EEC33AB4EEE73A5A
:10F25000DFED3B7AF1EE10FAF0EEE33A48BF00231F
:10F26000F4EEE73A48BFC9F80030F1EE10FA44BFB7
:10F270000023C8F80030BEF1000F2CDD00239FED05
:10F28000317A1E46342706E0DCF8DCEA013636B275
:10F29000764533461FDA07FB03C3D3EDB47A0EF18C
:10F2A000FF3EF4EEC77A07FB0EC4F1EE10FA04F548
:10F2B0002F7403F52F75E7D50FCCCCF8DCEA0FC51A
:10F2C0000FCC0FC50FCC0FC5013636B223682B60AB
:10F2D00076453346DFDB05B0BDEC048BBDE8F08F2F
:10F2E000F4EEC95AF1EE10FA19D465EEA95AFDEE02
:10F2F000E57ACDED037ABDF90C209BE7B4EEC96A3F
:10F30000F1EE10FA10D426EE296AFDEEC67ACDEDA4
:10F31000037ABDF90C3086E7F0EE465A53E748F21F
:10F320000102CFF6FF7285E748F20103CFF6FF73C3
:10F3300079E700BF0000003800FEFF460000000033
:10F34000FFE6DB2E17B7D138B5EEC00AF1EE10FAA2
:10F350000BD4F7EE007AB4EEE70AF1EE10FA09DD0D
:10F36000B6EE000A80ED0B0A70479FED060A80EDAD
:10F370000B0A7047F6EE007A20EE270A80ED0B0AA2
:10F38000704700BF0000000049F63C03C1F6FF7360
:10F39000012270B559690271002283F8382083F880
:10F3A000392083F85C2083F85D2083F85E2083F8A1
:10F3B0005F200D6804462E6848685A6630439A6696
:10F3C00028601869827093F861200D680A444FF232
:10F3D000CC50167A527BC0F20E0000EBC606120229
:10F3E000766802F4E06242F06402326093F86220D0
:10F3F0000A44967CD27D00EBC6001202406802F4FB
:10F40000E06242F06402026028684A68104205D057
:10F410001A692C2151701A69042191711A692021ED
:10F4200051711B6980229A70052006F081FF44F219
:10F4300060023021204601F047FE0546002859D0E1
:10F440006C222621204601F03FFE4FF4F97228215C
:10F45000204601F039FE40F622722C21204601F0B0
:10F4600033FE44F246423C21204601F02DFE40F29C
:10F4700037122421204601F027FE44F2FF023021FA
:10F48000204601F021FE73220221204601F01CFEDD
:10F490004FF4C87006F04CFF41F61D522E21204655
:10F4A00001F012FE04221146204601F00DFE4FF439
:10F4B00098720621204601F007FE10220A212046FC
:10F4C00001F002FE00220E21204601F0FDFD43F670
:10F4D0003C421021204601F0F7FD47F67F722221C1
:10F4E000204601F0F1FD36222421204601F0ECFDFA
:10F4F00001236372284670BD437AFBB1036970B47F
:10F500000646186800221A60B8B1B6F91E40B6F96E
:10F510002010031D00F5827533F9022B9442A8BF19
:10F5200014469142B8BF11469D42F5D80123F48399
:10F530003184337770BC05F095B870BC704700BF5C
:10F5400041689FED157AD1ED056ADFED147AE6EE9C
:10F55000877A45F2A65242F24B43C4F22C72C3F2B0
:10F56000BE7310B58260C360044617EE900A09F0BE
:10F57000F3FE41EC100B0EF057FD51EC100B09F0AF
:10F580003FFFDFED077A07EE100A67EE277A04F6F1
:10F59000F824C4ED007A10BD3D0AC7403D0A27C0DB
:10F5A00025551539036A002B00F0BB802DE9F04F7B
:10F5B0002DED048B0446ADF5057D002105F0D2F854
:10F5C000637A012B804640F2B08023695A68019229
:10F5D00000275F601346002800F0A480002A00F096
:10F5E0009380181D04A9802209F048FCD4ED0B8AF1
:10F5F000A38CD4F82090B7EE008A38EE688A0DF11B
:10F60000100A08F1040B84AEB6EE009A218DBAEC14
:10F61000017A994288BF5900B4F9303098BFA78465
:10F6200007EE903ABBF90030F8EEE77A06EE903A32
:10F6300067EEA87AF8EEE66A98BF0021E6EE887ACF
:10F6400003A827EE097AFDEEE77A17EE903A29F83B
:10F650000130258D07EE905AB8EEE70A27EE000A32
:10F660000EF062FCE38C9DED036A06EE903AA38CEB
:10F67000F8EEE66A07EE903AB8EEE77A76EE867A2A
:10F68000B7EE006A77EE677AFDEEE77ACDED007AA5
:10F69000BDF90030002BBCBF5B191BB2013DAB4272
:10F6A0001DBF591C09B249000021638639F90120A8
:10F6B00039F9133007EE902A06EE903AB8EEE77A61
:10F6C00076EE407AF8EEE66A67EE277AE0EE267A82
:10F6D000F5EEC07AF1EE10FAACBF77EE897A77EEEC
:10F6E000C97AB245FDEEE77A17EE903A2BF8023B65
:10F6F000A38C03F101039BB2A38487D1019804F08A
:10F70000B1FFB8F1000F06D020464146FDF77AF868
:10F71000404604F0A7FF0DF5057DBDEC048BBDE868
:10F72000F08F7047002AE9D1F5E70028ECD1F2E725
:10F730009FED3C7ADFED3C7A80EE070A38B505464E
:10F7400060EE277A17EE900A09F006FE41EC100BE6
:10F750000EF012FB51EC100B0AF0B4F82B8D06EEF4
:10F76000903AF8EEE66AB6EE087A26EE877AF6EE7A
:10F77000007AB5EEC07AF1EE10FAACBF77EE277AD8
:10F7800077EE677A84B2FDEEE77A17EE903AA342FD
:10F7900044DBF5EE007A66EEA77AB6EE007AF5EE77
:10F7A000C07AF1EE10FAACBF77EE877A77EEC77ABF
:10F7B000FDEEE77A17EE903AA3421BDAEC8407EEEF
:10F7C000904A9FED196A9FED177AF8EEE77AC7EE37
:10F7D000866A66EE877A17EE900A09F0BDFD41EC65
:10F7E000100B0EF0C9FA51EC100B09F009FE00EEF7
:10F7F000100A38BDF6EE007A66EEA76A66EEA77AC2
:10F8000017EE900A09F0A8FD41EC100B0EF0B4FAC7
:10F8100051EC100B0AF056F8E884D0E717EE100A06
:10F82000F0E700BF00007A44A6552C4770B5456844
:10F83000D0ED035A95ED024A95ED036A9FED697A82
:10F840009FED695AF2EE084AF9EE087AE4EE247A5E
:10F8500000F6043300F60836F1EE006A2DED028B57
:10F8600066EE266ABFEE008AF0EE484AE6EE264AC9
:10F870000446FDEEE77AF6EE008A17EE902AC0F80D
:10F88000E82AC3ED004AD5ED037AF4EEE87AF1EE0A
:10F8900010FAD4BFF0EE457AF0EE477AC6ED007A62
:10F8A00065EEE77A17EE900A09F056FD41EC100B71
:10F8B0000EF0BAFB51EC100B09F0A2FD07EE100A96
:10F8C000F7EE007A77EEC77AB0EE007AC6ED007AEE
:10F8D000D5ED047AA7EE878A04F6FC2204F530639E
:10F8E00082ED008A83ED008A95ED047AB4EEE87A21
:10F8F000F1EE10FA03D5F1EE487AC3ED007ADFEDB0
:10F900003B6A95ED056A9FED3A7AD4ED037A9FED57
:10F91000398AA6EE267A04F6F82627EE888A17EEAC
:10F92000100A09F019FD41EC100B0EF07DFB51ECB3
:10F93000100B09F065FD07EE900A27EE888AF7EEB6
:10F94000007A86ED008A95ED067A77EE277A04F63E
:10F95000343377EE877AF5EE006AC3ED007A95EDE1
:10F96000067AB4EEE67AF1EE10FA09D5B0EE086A3E
:10F97000F6EE086AE7EE466A77EEE67AC3ED007ABD
:10F9800095ED077A9FED1C6ADFED1C7ADFED1C6AAE
:10F9900027EE067A04F6E42383ED007A95ED097AE2
:10F9A000B6EE006A37EE467A04F6183383ED007A35
:10F9B00095ED0A7A67EE277A04F5326367EE877A67
:10F9C00004F61C310022C1ED007ABDEC028B1A60F6
:10F9D000D5ED0B7A67EEA67A04F62434C4ED007AEE
:10F9E00070BD00BF00C05A4600409C453D0AC7405C
:10F9F0003D0A27C0560EC9408FC2F53C2DB29D3D31
:10FA00006666E63F2DE9F84378292DED028B054621
:10FA1000476800F0968018D97B295DD076D97E2979
:10FA200053D07F294CD149F2A823C1F6FF7393F834
:10FA30002430282B00F2C780002B08BF01232B7431
:10FA4000BDEC028B0120BDE8F883072900F0AE80F1
:10FA50002AD8012934D107EE902ADFED7F6A9FED85
:10FA60007F7AF8EE677A00F6383367EEA67AF4EE1E
:10FA7000C77AF1EE10FAC3ED007A21DD00F6FC231F
:10FA800000F53065C3ED007AC5ED007AD7ED046A64
:10FA9000B6EE007AF4EEC76AF1EE10FA10D5F1EE88
:10FAA000677AC5ED007A0BE0402901D0422907D1E1
:10FAB00002F04004E4B2C5F8EC4A002C00F0868065
:10FAC000BDEC028B0120BDE8F88301230374BDEC7B
:10FAD000028B0120BDE8F8830021034600F5026295
:10FAE000C3F8D01234339A42FAD105F628320021F5
:10FAF000C4F22031002311602846C5F8DC3AFFF734
:10FB000095FEBDEC028B0120BDE8F8837929D7D1A1
:10FB100000F6F82700F52F6600F5316400F60C3189
:10FB200000F6F42500234FF07E523B6033602360E3
:10FB30000B602A60FFF77AFEBDEC028B0120BDE866
:10FB4000F88347F2A4000024C3F67D702B4605F528
:10FB50000261C3F8D042C3F8D402343399424FF063
:10FB60000002F6D105F628310024C4F220340C60DE
:10FB7000002305F6F82005F6F42105F52F6705F5B5
:10FB8000316605F60C34C5F8DC3AC5F8EC3A4FF0AE
:10FB90007E5302603A602846326022600B60FFF7B5
:10FBA00045FEBDEC028B0120BDE8F88302EB82022A
:10FBB00002EB8200C0F3471008F09AFFBDEC028B05
:10FBC0000120BDE8F88328232B7439E72A7C002A1A
:10FBD0003FF476AF2E46B1EE048A04E0A24206F16D
:10FBE00034067FF76DAFD6F8EC32802B04F10104B8
:10FBF000F4D1D5F8EC3A002BF0D1E86880F0004061
:10FC000009F0AAFBD7ED017A67EE887A804617EEF5
:10FC1000900A894609F0A0FB0B4641F6B8610246FE
:10FC2000C4F21D014FF0A04009F036FA41EC100B70
:10FC30000EF0FAF9404653EC102B494609F030FC1F
:10FC400041EC100B0EF0F0F951EC100B09F0D8FB61
:10FC5000C6F8D4022A7CC1E72497FF3BCDCC4C3DAB
:10FC60000068026848F675231268C0F200039A42E1
:10FC70007FD148F23403C4F204031B685A0565D5EA
:10FC800043F21473C2F201032DE9F0471B68884662
:10FC90000BB101221A7043F2CC69C2F2010943F29E
:10FCA000CD6599F8004001343F2C88BF4FF0000A21
:10FCB00043F2D0674FF4204694BF5FFA84FA54466B
:10FCC000C2F20105C2F20107C4F206062B78A34274
:10FCD0002AD1EFF31383002B39D1EFF31083002BDC
:10FCE00035D1EFF30582002A40D00F2A05D94EF214
:10FCF000F033CEF2000313441B78EFF3118212B1FC
:10FD0000934228BF1346402B21D9B3F5807FDDD124
:10FD100043F24173C2F201031B78002BD6D107F0E6
:10FD2000E9FB2B78A342D4D043F210734FF4204266
:10FD3000C2F20103C4F2060207F804800120BC21CC
:10FD4000187089F800A0D170BDE8F087704733794A
:10FD50001B06BBD52B7801333F2B86BF00221346F1
:10FD6000DAB2FB5CDBB2F3712A70AFE74FF4807359
:10FD7000C3E710472DE9F04F4BF220022DED028B27
:10FD800049F2A823C1F6FF72C1F6FF73166893F912
:10FD90000970D6F804A083B007440C46002900F08F
:10FDA000CF81D6F8DC5A317C8D4280F298813423A1
:10FDB00003FB05630022691CC6F8DC1AC3F8DC22C9
:10FDC000C3F8D822A7F13C094EF64F4309FB09F2CC
:10FDD000C4F6C46383FB0231D317C3EBA10303EB67
:10FDE000430103EB8103D31A07EE903AF8EEE77A6A
:10FDF000B1EE0A7A06F61C3106F6183377EEC77AAA
:10FE0000D3ED006A91ED007A3C2FE7EE276A09DD19
:10FE100007EE102A06F53263D3ED007AB8EEC77A02
:10FE2000E7EE876AD6F8E83AB2691A44974240F397
:10FE3000FD81726D1A44974240F32B82D6F89020D0
:10FE40001A44974240F32282D6F8CC201A449742B3
:10FE500040F30182D6F808211A44974240F3F88112
:10FE6000D6F844211A44974240F3EF81D6F8802116
:10FE70001A44974240F3E681D6F8BC211A449742CF
:10FE800040F3DD81D6F8F8211A44974240F3D4813B
:10FE9000D6F834221A44974240F3CB81D6F8702228
:10FEA00013449F42CCBF4FF021084FF01E084FEA89
:10FEB000880B0BEB080306EB8303D6ED037A5B6933
:10FEC0009FEDE68A9FEDE66AFB1A07EE103AB8EE60
:10FED000C77A27EE888A77EE267A67EE867A17EE5B
:10FEE000900A09F039FA41EC100B0EF09DF834231A
:10FEF00003FB056351EC100B009309F081FA07EE48
:10FF0000900A27EE888A009BBEEEC88A0022302C19
:10FF1000C3F8C02283EDAF8A07DD502CD4BF08F1AF
:10FF2000010808F102084FEA880BD84406EB88085C
:10FF30004FF0340E06F63432D8F82030D2ED008A75
:10FF4000D8F81C00D8F824100EFB0568013BC8F84F
:10FF5000C832C8F8C402C8F8CC1218EE900A09F0EA
:10FF6000FBF907EE904A9FEDBF7AF8EEE77ACDE90C
:10FF7000000167EE877AB0EE088A17EE900A09F062
:10FF8000EBF99DED001B41EC100B0EF0D1F8F0EEFB
:10FF9000007A51EC100BA8EEA78A09F031FA07EEAF
:10FFA000900A28EE278A3C2F88EDB48A00F31F813F
:10FFB000DAED046A9FEDAC7ADFEDAC5ADFEDAC7A96
:10FFC0009FEDAC6A96ED038A06F6283393ED005A4E
:10FFD00066EEA66A403CA6EE857A06F62C3306F657
:10FFE0003C3106EE904A05EE107AD3ED004AF8EE69
:10FFF000E66AB8EEC55AA4EEA67A342303FB05637D
:020000021000EC
:10000000E5EE257AC3F8EC7206F6E422B4EEE77A60
:10001000F1EE10FA58BFF0EE477AF4EEC67AF1EE40
:1000200010FAD4BF67EEA77ADFED937A68EE277AED
:100030000B2FC3EDB87A6CDD6C2F40F32F81D1ED1F
:10004000007A92ED007A9FED8D6A27EE877AF0EEC6
:10005000675AE7EE065A4EF685394FF0A858F0EE8B
:10006000006AB0EE657AC4F20109B0EE476A97EE15
:10007000A66A83EDBA7A83EDB96ADAED007A77EE93
:10008000A77A17EE900A09F067F902460B46404638
:10009000494609F001F841EC100B0DF0C5FFF1EEF7
:1000A000487A53EC102B17EE900ACDE9002309F0A3
:1000B00053F9DDE9002309F0F3F941EC100B0DF0E1
:1000C000B3FF342351EC100B03FB056609F098F9DC
:1000D000C6F8D40203B0BDEC028BBDE8F08F002956
:1000E00000F0DA800025DFED667A2B46324692ED8D
:1000F000B47AB4EEE77AF1EE10FA48BF1D4603F188
:10010000010348BFF0EE477A994202F13402EED182
:1001100058E6D1ED007A92ED007A9FED5A6A27EE0B
:10012000877AF0EE675AE7EE065A47F6E1294FF074
:100130002058F0EE006AB0EE657AC3F6D47994E701
:10014000327C002AC6D035464FF0800B04E00134E3
:10015000A24205F13405BDDDD5F8EC329F42F6D15F
:10016000D6F8EC3A1BB1C5F8ECB2327CEFE7F06898
:1001700080F0004009F0F0F8CDE90001384609F0C0
:10018000D9F847F6E1234FF08042C3F6847309F0B3
:1001900087F900230022C4F2180308F07FFF9AEDCC
:1001A000017AF1EE047A67EE277A804617EE900A1C
:1001B000894609F0D1F802460B464046494608F008
:1001C0006BFF41EC100B0DF02FFFDDE9000153EC4C
:1001D000102B09F065F941EC100B0DF025FF51ECE7
:1001E000100B09F00DF9C5F8D402327CAFE7C7F166
:1001F0003C0307EE903A9FED247AF8EEE77A67EE3B
:10020000877A17EE900A09F0A7F841EC100B0DF071
:100210000BFF51EC100B09F0F3F8D8EDB47A07EEB0
:10022000100A67EE877AC8EDB47AC1E64FF000088D
:100230003DE64FF01B083AE64FF0180837E64FF05E
:10024000150834E64FF0120831E64FF00F082EE69D
:100250004FF00C082BE64FF0090828E60000FA469C
:1002600020986C3D2497FF3B00004842CDCCCC3E0B
:1002700000005C420000524300442C470000404212
:100280000000C642000040C20AD7233C4FF00608D7
:100290000DE64FF003080AE60D4693E591ED007A6E
:1002A000D2ED006A07EE909A67EE266AF8EEE77ADA
:1002B000F0EE475AE6EEA75A2B2FB0EE006AF0EEAA
:1002C000656AD7EE066AC3EDBA5AC3EDB96A06DCB1
:1002D00047F6E1294FF02058C3F6D479CDE63846E9
:1002E00009F028F84BF651034FF06042C3F69E73B5
:1002F00009F0D6F800230022C3F6F07308F0CCFE14
:1003000080468946B9E600BF0020704770B449F2C4
:100310002463C1F6FF7348F21F02996BC4F2000216
:1003200008791070586B48F21C02C4F2000204797C
:100330001470097911701A6B002A4FD05968C96876
:100340008A4247D80168CC8B240402F1FF3069D47B
:10035000C0F30E00C883C88B80B2C882996B09684D
:10036000C88B000456D4C2F30E00C883C88B002487
:1003700080B212F1FF32C88218BF01221C63596B90
:10038000086849F224610568C1F6FF7101F12C0487
:10039000A54237D00968CC6814F0804F046805681E
:1003A00015BF248824780235013544F000440560E7
:1003B0004C63996B48F21B03C4F20003097919706E
:1003C00049F22461C1F6FF7112B14A6B12791A70B9
:1003D00070BC7047521A1A630122D0E71968D86BB3
:1003E0000A630024CFF60F74CC62CC68066824F050
:1003F0008044CC603468032583F82D501146234691
:1004000070BC1847086891F82C10C46841F000418E
:100410004163CEE7CC8BC2F3080004F47E44204352
:10042000C883A3E7CC8BC0F3080004F47E442043C8
:10043000C88390E7437A002B42D00369196870B5EE
:10044000002504461D6099B172B640F6B072C2F242
:10045000010243F288031068C2F2010300282BD086
:100460005E681EB3166059601D8062B604F0FAF82B
:10047000637A012B19D92369596800245C60A1B102
:1004800072B640F6B472C2F2010243F288031068F9
:10049000C2F20103A8B1DD685DB11560D9601C81AD
:1004A00062B6BDE8704004F0DDB870BD596062B658
:1004B000DEE7D96062B670BD1160188062B6D7E71A
:1004C00070471160188162B670BD00BF90F89D3012
:1004D00090F89C20DBB2934214D001331F2B84BFD1
:1004E00000210B4610B598BFD9B2063350F823400F
:1004F00080F89D102146FCF785F92046BDE81040A4
:1005000004F0B0B8704700BF2DE9F04F436AC469EA
:10051000866985B02BB906EBC414846105B0BDE8CB
:10052000F08F0546076A04F0C7F80290002800F033
:10053000E680F219B5F932300192029A042B02F1E9
:10054000040E00F0EE8054DD062B00F07A81C0F23C
:100550006381072B00F00881082B73D1AA6ACDF8BC
:100560000CE04FEA520C130C6FEA0C021146029A8F
:10057000D5F82480C3F57F4B4FF0FF39901D7646A8
:1005800002F5837A0BF1FF0B019AB9FBFBFB8E4658
:10059000B9FBF3F921E0CCEB02073F0C4FF6FF71FA
:1005A0000BFB07F7C7F6FF7102EB0C03C91B1B0C13
:1005B000091409FB03F308FB01F103F1004396451D
:1005C0004FEA21414FEA234370D931800230504530
:1005D000224406F1020600F04281130C09FB03F3EA
:1005E0001B0C08FB03F362454FEA1343D3D233805D
:1005F000ECE7012B00F088805DDD022B43D0032B5C
:1006000020D16F6A019802F5827C7646C30BC3F550
:100610007F43C113FF3307FB03F34FEA907807FBD7
:1006200001F11A0C091408F1FF33012B94BF134692
:100630000B4626F8023B66452044E7D1019B03EBBD
:10064000C41301932C6A019AB5F93430141BAC61C0
:1006500073B1029A02F5827101E0B5F93430BEF946
:100660000020134403F30F032EF8023B7145F4D826
:10067000029C28462146FCF7C5F8204605B0BDE897
:10068000F04F03F0EFBF686A20F34F0002F5827667
:10069000019A07B27346404237EA220128BF014659
:1006A00023F8021BB3422244F6D1C7E708FB03F349
:1006B0001B1433808AE7002BC4D140F23436D5F8BE
:1006C00024C00199C0F20F0602F5827770460B0E26
:1006D0005A1C36F9138036F91220C1F30F29C9F5D7
:1006E000803308FB03F309FB023353FB0CF320F8C0
:1006F000023BB8422144EAD1A0E703F0B3FFAB6963
:1007000003EBC413AB6109E702F582706E6A019ACC
:10071000734636FB12F123F8021B83422244F8D1C0
:100720008CE7EE6A002EE8D0D5F824C0019902F5D6
:10073000827770460A0E531CB3F5807F14BF5B00AE
:100740000023C1F30F28F35E36F9122008FB03F3F0
:10075000C8F5803808FB023353FB0CF320F8023B4A
:10076000B8422144E6D169E743F28803C2F20103AB
:1007700003931E69029B019940F65F384FF21D3AC0
:100780004FF2EC4BC8F24E38C0F2010ACFF6FF7BB5
:1007900003F5827C7746002201E0674532D0B5F947
:1007A000303027F8023B6118F7D3686A18B326B3D4
:1007B00086FB082388FB069233444FEAE6793244ED
:1007C000C9EB2343C9EB22420AFB13660BFB02F27F
:1007D00044F2A71303FB0626002E02DA06F10046B8
:1007E000013EB6FBF0F300FB13639BB20122A3EBC7
:1007F00060032B86D1E70346F9E74CF64266C1F663
:100800000C76EEE7019B03EBC4130193002A3FF43F
:1008100019AF039B1E6115E7686A20F34F0002F5CC
:100820008276D5F828C0019A07B2734640426245E5
:1008300034BF3946014623F8021BB3422244F6D1A5
:10084000FCE6686A02F58276019AC043734630FB83
:1008500012F123F8021BB3422244F8D1EEE6019BC9
:10086000DDF80CE003EBC4130193EBE62DE9F04F48
:100870009BB0044603F020FF637A1690002800F036
:100880006282002B00F0698223691A681792114670
:1008900000221A60002900F0608240F23853C0F252
:1008A0000F03199345F24C6945F24E6734F909304C
:1008B000059345F25065E35F099345F25266635F25
:1008C000189345F25661A35F089345F25862635E40
:1008D000079345F25A6AA35E069334F90A300493EB
:1008E00004F5AC431A4604F5C5491E46CDF84490BC
:1008F00002F13C093E320B9206F140020C9206F1E5
:1009000042020D9206F144020E9206F146020F9247
:1009100006F14802119B109232464A3203921A465F
:10092000183211921A461A3245F25460129245F268
:100930005E681A4645F25C6C45F2606E1C321E33EE
:1009400034F900B0139234F9088034F90CC034F94A
:100950000EE0CDF808901493179B189D9A1C0192F5
:10096000169A03F5817302321593019B0A924FF098
:10097000000A584633F9022F019302EB021202EBF0
:100980000222520022F34F42029B05991E8804EB7B
:10099000460701FB0CF9B7F91C3003FB089929F352
:1009A000CF390FFA89F1059112B201FB0EF929F343
:1009B000CF39914409F30F090136A7F81C90029929
:1009C000B6B240F25B47BE4294BF0E80A1F800A0D1
:1009D0000B99099F0E8804EB460907FB0CFBB9F93C
:1009E000D4783B4407FB08BB2BF3CF3B0FFA8BF7C4
:1009F000099707FB0EF727F3CF37174407F30F07C5
:100A00000136A9F8D4780B99B6B240F2A347BE429A
:100A100094BF0E80A1F800A00C990E8804EB460745
:100A200007F590571C37B7F9009005FB0CF54B44C0
:100A300009FB085525F3CF352DB205FB0EF929F337
:100A4000CF39914409F30F090136A7F80090B6B2E7
:100A500040F2FC47BE4294BF0E80A1F800A00D9961
:100A60000E88089904EB460707F5E0571637B7F9E3
:100A7000009001FB0CFB4B4409FB08BB2BF3CF3B65
:100A80000FFA8BF9CDF8209009FB0EF929F3CF3935
:100A9000914409F30F090136A7F800900D99B6B2F9
:100AA00040F24B57BE4294BF0E80A1F800A00E99B1
:100AB0000E8804EB460707F51A572E37B7F9009052
:100AC00000FB0CF04B4409FB080020F3CF3000B2D0
:100AD00000FB0EF929F3CF39914409F30F090136D0
:100AE000A7F80090B6B240F28D57BE4294BF0E8078
:100AF000A1F800A00F990E88079904EB460707F5A7
:100B000047570A37B7F9009001FB0CFB4B4409FB30
:100B100008BB2BF3CF3B0FFA8BF9CDF81C9009FBE8
:100B20000EF929F3CF39914409F30F090136A7F8DB
:100B300000900F99B6B240F2D257BE4294BF0E80D9
:100B4000A1F800A010990E88069904EB460707F556
:100B500075573037B7F9009001FB0CFB4B4409FB8C
:100B600008BB2BF3CF3B0FFA8BF9CDF8189009FB9C
:100B70000EF929F3CF39914409F30F090136A7F88B
:100B800000901099B6B240F21467BE4294BF0E8036
:100B9000A1F800A003990E88049904EB460707F515
:100BA00093471A37B7F9009001FB0CF14B4409FB4E
:100BB000081121F3CF3109B2049101FB0EF929F399
:100BC000CF394A4402F30F020136B6B2B6F5CA6F06
:100BD0003A808ABF039A0399A2F800A047F6E1225F
:100BE00098BF0E8002FB03F323F34F4311990E8845
:100BF00004EB460707F5AC470FFA83F9B7F9622013
:100C000003EB6203A7F86230C9EB020222F34F0242
:100C10000136B6B2B6F50B7F34BF0E80A1F800A046
:100C200012990E8804EB460707F5B5470FFA82F9CB
:100C3000B7F93A3002EB63027A87C9EB030323F377
:100C40004F030136B6B2B6F5DC7F94BF0E80A1F833
:100C500000A013990E8804EB460707F5BC470FFA6E
:100C600083F9B7F92C2003EB6203BB85C9EB0202C1
:100C700022F34F020136B6B2B6F5AA7F94BF0E80BA
:100C8000A1F800A014990E8804EB460707F5C147A8
:100C90000FFA82F9B7F9563002EB6302A7F8562033
:100CA000C9EB030323F34F030136B6B21BB2E02EA8
:100CB000C3EB031394BF0E80A1F800A05B0003F305
:100CC0000F030A9A22F8023F019B0A92159A934257
:100CD0007FF450AE0599002213461E4661F30F02C1
:100CE000069965F30F03354661F30F05099961F322
:100CF0001F42089961F31F43079960F30F0661F3E0
:100D00001F46049945F2546E45F2586C45F2506006
:100D100045F24C6761F31F45E251235044F80E60E1
:100D2000204644F80C50169C2146FBF76BFD2046EC
:100D300003F098FC1798199A90420BD01BB0BDE8AD
:100D4000F04F03F08FBC2BB12369169A18681A6014
:100D50000028F3D11BB0BDE8F08F40F23853C0F249
:100D60000F03199317939DE54DF2CC33C1F6FF7332
:100D70002DE9F04719681B79096848F21F0248F20B
:100D80000050C1F6FF70C4F200028142137031D2EC
:100D900040F6B973C2F201031B7873BB40F6B0781A
:100DA000C2F2010840F6B47743F28804C2F20104AB
:100DB000C2F20107D8F80090D7F800A0258826894C
:100DC000B9F1000F3CD0BAF1000F31D00AF10402A2
:100DD00009F1040102EB460201EB450107F0D2FFE5
:100DE000403640357F2D19D825807F2E0CD826819E
:100DF000BDE8F087A0F58070D0E74EF20823CEF270
:100E0000000301221A60C9E700255046258103F03E
:100E100029FCE3683B60E560BDE8F08700254846B3
:100E2000258003F01FFC6368C8F800306560DCE7CC
:100E300009F1040101EB450107F0C3FF4035D1E79B
:100E4000BAF1000F07D00AF1040101EB460107F0E7
:100E5000D8FF4036C6E74FF48072514608F08CFD4B
:100E6000C0E700BF70B58469054614B3B4F5803F90
:100E700027D0002103F076FC064608B3011D00F5DB
:100E800082700B6834FB03F234FB13F302F30F029E
:100E900003F30F03C2EA034341F8043B8842F0D84E
:100EA00028463146FBF7AEFC3046BDE8704003F003
:100EB000D9BB437A23B1036918681C600028F4D1B8
:100EC00070BD437A002BFBD003691C6800221A60B6
:100ED000002CF5D02146FBF795FC2046BDE870407C
:100EE00003F0C0BB2DE9F0470024804600F118074D
:100EF00025462646002D56D098F80930A34227D91A
:100F0000D8F8103053F8240043F8246000B3D7F821
:100F100000C0BCF5803F05F1040E00F1040905F5A1
:100F2000827125D059F8042B3CFB02F33CFB12FAEA
:100F300003F30F020AF30F03C2EA0343DEF80020B3
:100F400093FA12F34EF8043B7145EBD803F08AFB99
:100F50000134042C07F10407CCD1002D41D04046C8
:100F60002946FBF74FFC2846BDE8F04703F07ABB63
:100F700005F10C0E00F10C0C5EF8083C5CF8082C36
:100F800093FA12F34EF8083C5CF8042C5EF8043C2B
:100F900093FA12F371454EF8043C0CF1080C0EF173
:100FA000080EE9D8D2E72146404603F0DBFB0546B0
:100FB0000028CDD03868B0F5803FC9D0291D05F58F
:100FC000827E0B6830FB03F230FB13F302F30F0257
:100FD00003F30F03C2EA034341F8043B8E45F0D804
:100FE000B6E7BDE8F08700BF41F23003C4F20B035F
:100FF00041F224021968C4F20B0241F08001196029
:1010000011461368DB07FCD40B689B07F9D441F247
:101010000C03C4F20B0310B441F230041860C4F2A4
:101020000B044FF0807200E0D2B121680123C0F2BE
:101030000E030B4041F23001013AC4F20B01002BC8
:10104000F2D06AB1012B0BD10B6813F0800F0B6843
:1010500013D043F0011303200B605DF8044B70477D
:1010600041F23002C4F20B020120136843F47023F2
:10107000034313605DF8044B704713F480300B6832
:1010800004D043F001130B600520F3E743F00103A4
:101090000B60EFE703790F2B14D848F21A02C4F261
:1010A000000210B4137072B640F6AC73C2F20103C2
:1010B000047919880122A24021EA02021A8062B64C
:1010C0005DF8044B704700BF38B549F63C03C1F6E4
:1010D000FF730124242908BFC280007A83F85E4090
:1010E000B3F85E5083F85D40A04083F83B0065B1E3
:1010F0000D0A140A052083F83D1083F83C5083F84C
:101100003F2083F83E4083F85D00012006F0F4FEA6
:10111000B0FA80F0400938BDB0F85E306BB190F89D
:101120005D30202B07D8C218013380F85D300120D4
:1011300082F83B107047012303710020704700BF05
:10114000704700BF90F8383090F839209A4286BF37
:101150001B18187E4FF0FF30704700BF90F83830F2
:1011600090F839209A4205D95A1C034480F8382057
:10117000187E70474FF0FF30704700BF90F839205D
:1011800090F83800101A704749F24C50C1F6FF70C1
:10119000FBF762BC49F2B850C1F6FF70FBF75CBCCC
:1011A00049F63C00C1F6FF70FBF756BC38B5054662
:1011B000B0F85E0090B195F85D301446C3F121029D
:1011C00094420CD805F13B001844224609F0B4F8CB
:1011D00095F85D30234485F85D30204638BD012008
:1011E00014462871EEE700BF037B012B024601D9AC
:1011F0000020704700EB830001334160012013732E
:10120000704700BF70B549F63C04C1F6FF74012277
:10121000437984F85E200646B4F85E0084F85D20C9
:1012200093400D4684F83B3040B1737B43F0040398
:101230000B43022284F83C3084F85D20012006F044
:101240005BFE3C23013BFDD10123727984F85E30C3
:10125000B4F85E1084F85D309A4049F63C0384F897
:101260003B20C1F6FF7341B1717B25F004050D43AE
:10127000022283F83C5083F85D20012006F03CFEFA
:1012800040F6B833013BFDD170BD00BF30B449F624
:101290003C03C1F6FF730124427983F85E40B3F842
:1012A0005E5083F85D40A24083F83B2035B1407B1F
:1012B0000222014383F83C1083F85D20012030BCFA
:1012C00006F01ABE2DE9F04149F63C04C1F6FF7460
:1012D00006460120737984F85E00B4F85EE084F875
:1012E0005D004FEA0118834021F00F01174684F892
:1012F0003B305FFA88F842EA0105BEF1000F06D0E4
:10130000737B02222B4384F83C3084F85D2001205B
:1013100006F0F2FD29463046FFF774FF012371798C
:1013200084F85E30B4F85E2084F85D30994049F668
:101330003C0348EA070784F83B10C1F6FF7332B15B
:10134000727B02213A4383F83C2083F85D10012030
:1013500006F0D2FD39463046BDE8F04152E700BF05
:1013600008B50122FFF7AEFF012008BDF0B540F23D
:101370003C63C0F20F03144606460F460FCB85B000
:10138000757A0DF1100E0EE90F00A5423CBF05F174
:10139000FF34E4B204AB03EB8404304654F8101C71
:1013A000394461F07F01C9B2002205B0BDE8F040C8
:1013B00088E700BF10B5002201210446FFF782FF35
:1013C0004DF2C043C0F20103013BFDD1A37A03B942
:1013D00010BD002220461146BDE81040C6E700BF00
:1013E00043F28403C2F201031B780BB9012070475A
:1013F00000231B78FFDE00BF08B549F24853C1F651
:10140000FF731B68834203D0FFF7EAFF48B908BDAA
:1014100043F28403C2F2010301201A7811431970C8
:1014200008BD00231B78FFDEF8B590F82030C469B2
:10143000102B49F2485305460E461746C1F6FF7376
:1014400020D0186804EBD114844220D142F230033A
:1014500006F07F01C2F2010343F8217043F28403D6
:10146000C2F20103297E1A78012942F001021A70A2
:101470001FD9AA6843F28003C2F201031044186026
:101480000120F8BD1B6804EB11249C4208D0002108
:101490002046FFF7B1FF68B195F82030102B0AD134
:1014A00042F23003F1B2C2F20103204623F8117078
:1014B000D4E70120F8BD2046C8E700BFC368013368
:1014C0008B421ED370B590F82030102B49F2485350
:1014D000044616460D46C069C1F6FF7313D01B685B
:1014E00000EBD110984213D142F2300305F07F0196
:1014F000C2F20103012053F8213023F0704333601E
:1015000070BD002070471B6800EB1120984207D087
:101510000021FFF771FF68B194F82030102BE3D160
:1015200042F23003E9B2C2F20103012033F8113074
:10153000336070BD002070BD40F2207008B5C0F26D
:101540000F00162106F0D6F849F2A823C1F6FF7362
:1015500093F82330B3B143F60860FF21C2F20000D4
:10156000FEF77EFB40F29C00C0F20F0006F0A4FDE7
:101570004FF60F7006F054FD40F2AC00C0F20F00C1
:1015800006F09AFDBDE80840FAF79CBC40F23870BE
:1015900008B5C0F20F00182106F0ACF849F2A823F4
:1015A000C1F6FF7393F82330B3B143F60860FE2110
:1015B000C2F20000FEF754FB40F29C00C0F20F00A4
:1015C00006F07AFD4FF60F6006F02AFD40F2AC00FF
:1015D000C0F20F0006F070FDBDE80840FAF772BCDB
:1015E00040F2547008B5C0F20F000F2106F082F8E7
:1015F00049F2A823C1F6FF7393F82330B3B143F641
:101600000860FC21C2F20000FEF72AFB40F29C00B9
:10161000C0F20F0006F050FD4FF60F4006F000FD3F
:1016200040F2AC00C0F20F0006F046FDBDE80840F5
:10163000FAF748BC40F2647008B5C0F20F001321FD
:1016400006F058F849F2A823C1F6FF7393F8233047
:10165000B3B143F60860FB21C2F20000FEF700FBC5
:1016600040F29C00C0F20F0006F026FD4FF60F304E
:1016700006F0D6FC40F2AC00C0F20F0006F01CFDF4
:10168000BDE80840FAF71EBC40F2787008B5C0F219
:101690000F00102106F02EF849F2A823C1F6FF73BF
:1016A00093F82330B3B143F60860FA21C2F2000088
:1016B000FEF7D6FA40F29C00C0F20F0006F0FCFCE8
:1016C0004FF60F2006F0ACFC40F2AC00C0F20F0069
:1016D00006F0F2FCBDE80840FAF7F4BB40F28C706B
:1016E00008B5C0F20F00102106F004F849F2A82353
:1016F000C1F6FF7393F82330B3B143F60860F821C5
:10170000C2F20000FEF7ACFA40F29C00C0F20F00FB
:1017100006F0D2FC4FF60F0006F082FC40F2AC005F
:10172000C0F20F0006F0C8FCBDE80840FAF7CABBDB
:1017300040F2A07008B5C0F20F00162105F0DAFFE4
:1017400049F2A823C1F6FF7393F82330C3B143F6DF
:10175000C053C2F20003F621986C0368DB6C984713
:1017600040F29C00C0F20F0006F0A6FC4FF20F60A2
:1017700006F056FC40F2AC00C0F20F0006F09CFCF4
:10178000BDE80840FAF79EBB38B5044640F2B87091
:10179000C0F20F00152105F0ADFF49F2A823C1F6F4
:1017A000FF7393F823301BB9BDE83840FAF78ABBC2
:1017B00043F6C055C2F2000548F67523A86C0268CE
:1017C0001268C0F200039A4221D1F32004F09AFC7F
:1017D000A86C036804F07F01DB6C984740F29C0022
:1017E000C0F20F0006F068FC200400F4FE0040F494
:1017F000734040F0020006F013FC40F2AC00C0F26F
:101800000F0006F059FCBDE83840FAF75BBBF32146
:101810009047DDE770B5044640F2D070C0F20F008B
:101820001F2105F067FF49F2A823C1F6FF7393F863
:1018300023301BB9BDE87040FAF744BB43F6C056ED
:10184000C2F2000648F67525B06C03681B68C0F24A
:101850000005AB4224D1F12004F054FCB06C0368C5
:101860001B68AB421FD1204604F04CFC40F29C00A8
:10187000C0F20F0006F020FC04F00F044FF202103B
:101880002404C0F21000204306F0CAFB40F2AC0072
:10189000C0F20F0006F010FCBDE87040FAF712BB72
:1018A000F1219847DAE721469847DFE770B5064609
:1018B00040F2F0700C46C0F20F001221154605F000
:1018C00019FF49F2A823C1F6FF7393F8233013B32D
:1018D000214633462A46A020FAF70EFF40F2442064
:1018E000C0F20F0006F0E8FB681E0002240400F4BA
:1018F000706004F4FE04044344F45044300144F0A6
:101900000D04C0B2204306F08BFB40F2AC00C0F2E5
:101910000F0006F0D1FBBDE87040FAF7D3BA00BF64
:101920002DE9F04F87B0059040F604000491C0F215
:101930000F00102105F0DEFE49F2A823C1F6FF7367
:1019400093F8233023B907B0BDE8F04FFAF7BABADD
:1019500043F6C05BC2F2000BF021DBF848000368DD
:10196000DB6C9847049B002B00F0B8801A4648F2C5
:101970003403C4F20403DBF848000093059B0568B8
:1019800048F6752A4FF420461F461344C0F2000A59
:10199000C4F2060699462B6817F8011B534540F020
:1019A0009580009B1B685C0560D543F21473C2F2FE
:1019B00001031B680BB10120187043F2CC63C2F223
:1019C000010343F2CD651C7801343F2C88BF002011
:1019D00043F2D06894BFE0B20446C2F20105C2F2FD
:1019E00001082A78A24233D1EFF31382002A57D19B
:1019F000EFF31082002A53D1EFF3058EBEF1000FF2
:101A000061D0BEF10F0F05D94EF2F032CEF20002D6
:101A100072441278EFF3118EBEF1000F02D07245BE
:101A200028BF7246402A3BD9B2F5807FD9D143F214
:101A30004172C2F201021278002AD2D103930291BC
:101A4000019005F057FD2A7801A8A2420BC8CBD01F
:101A500043F21075C2F2010508F804100124BC21FC
:101A60002C701870F170DBF848000568B94592D108
:101A7000EB6CF721984740F29C00C0F20F0006F093
:101A80001BFB04990598FAF713FB40F2AC00C0F277
:101A90000F0006F011FB07B0BDE8F04FFAF712BADD
:101AA000327912069DD52A7801323F2A86BF4FF03F
:101AB000000E72465FFA82FE18F80220D2B2F2716E
:101AC00085F800E08DE74FF48072A3E79847DBF8D4
:101AD0004800B94505687FF45EAFC9E7DBF8480008
:101AE0000568C5E740F6180008B5C0F20F001621DA
:101AF00005F000FE49F2A823C1F6FF7393F82330E6
:101B00009BB14FF60F7006F08BFA40F2AC00C0F2BA
:101B10000F0006F0D1FA4FF60F7005F0D3FE40F239
:101B20003810C0F20F0006F0C7FABDE80840FAF717
:101B3000C9B900BF40F6300008B5C0F20F00182147
:101B400005F0D8FD49F2A823C1F6FF7393F82330BE
:101B50009BB14FF60F6006F063FA40F2AC00C0F2A2
:101B60000F0006F0A9FA4FF60F6005F0ABFE40F249
:101B70003810C0F20F0006F09FFABDE80840FAF7EF
:101B8000A1B900BF40F64C0008B5C0F20F000F210C
:101B900005F0B0FD49F2A823C1F6FF7393F8233096
:101BA0009BB14FF60F4006F03BFA40F2AC00C0F29A
:101BB0000F0006F081FA4FF60F4005F083FE40F269
:101BC0003810C0F20F0006F077FABDE80840FAF7C7
:101BD00079B900BF40F65C0008B5C0F20F001321D0
:101BE00005F088FD49F2A823C1F6FF7393F823306E
:101BF0009BB14FF60F3006F013FA40F2AC00C0F282
:101C00000F0006F059FA4FF60F3005F05BFE40F278
:101C10003810C0F20F0006F04FFABDE80840FAF79E
:101C200051B900BF40F6700008B5C0F20F00102196
:101C300005F060FD49F2A823C1F6FF7393F8233045
:101C40009BB14FF60F2006F0EBF940F2AC00C0F26A
:101C50000F0006F031FA4FF60F2005F033FE40F288
:101C60003810C0F20F0006F027FABDE80840FAF776
:101C700029B900BF40F6840008B5C0F20F0010215A
:101C800005F038FD49F2A823C1F6FF7393F823301D
:101C90009BB14FF60F0006F0C3F940F2AC00C0F262
:101CA0000F0006F009FA4FF60F0005F00BFE40F2A8
:101CB0003810C0F20F0006F0FFF9BDE80840FAF74F
:101CC00001B900BF40F6980008B5C0F20F00162118
:101CD00005F010FD49F2A823C1F6FF7393F82330F5
:101CE0009BB14FF20F6006F09BF940F2AC00C0F2DE
:101CF0000F0006F0E1F94FF20F6005F0E3FD40F24E
:101D00003810C0F20F0006F0D7F9BDE80840FAF726
:101D1000D9B800BF10B5044640F6B000C0F20F00BD
:101D2000152105F0E7FC49F2A823C1F6FF7393F8EB
:101D30002330C3B1240404F4FE0444F4734444F097
:101D40000204204606F06CF940F2AC00C0F20F002D
:101D500006F0B2F9204605F0B5FD40F23810C0F2A9
:101D60000F0006F0A9F9BDE81040FAF7ABB800BFC4
:101D700070B5064640F6C8000C46C0F20F001221AE
:101D8000154605F0B7FC49F2A823C1F6FF7393F896
:101D900023301BB9BDE87040FAF794B86B1E1B02E4
:101DA000240404F4FE0403F47063234343F4504317
:101DB000340143F00D03E4B21C43204606F030F931
:101DC00040F2AC00C0F20F0006F076F94EB140F2DE
:101DD0003810C0F20F0006F06FF9BDE87040FAF756
:101DE00071B8204605F06EFDF1E700BF38B5044636
:101DF00040F6DC00C0F20F001F2105F07BFC49F229
:101E0000A823C1F6FF7393F82330CBB104F00F047D
:101E10004FF202152404C0F210052543284606F0AF
:101E2000FFF840F2AC00C0F20F0006F045F928467A
